:020000040800F2
:100000007056002015020008DD93000835580008DE
:10001000F5920008B71D0008990A010800000000C9
:10002000000000000000000000000000C1E6000821
:100030007F1F00080000000063A60008A5F000086C
:100040002F0200082F020008D9F200082F02000832
:100050002F0200082F0200085D210008632100081C
:100060002F0200082F0200082F0200082F020008AC
:100070002F0200082F0200082F020008C51E0008EA
:100080002F0200082F0200082F0200082F0200088C
:10009000000000002F020008692100082F0200085C
:1000A0002F0200082F0200082F020008E1F20008CA
:1000B0002F0200082F0200082F0200082F0200085C
:1000C0002F0200082F0200082F0200082F0200084C
:1000D0002F0200087D0101082F0200082F020008EE
:1000E0002F0200082F0200082DAF00082F02000881
:1000F0002F02000800000000000000002F0200088E
:100100002F0200082F020008C5DC00082F0200089B
:100110002F0200082F0200082F0200082F020008FB
:100120002F0200082F0200082F0200082F020008EB
:100130002F0200082F02000800F002F800F05AF821
:100140000AA090E8000C82448344AAF10107DA4532
:1001500001D100F04FF8AFF2090EBAE80F0013F02A
:10016000010F18BFFB1A43F00103184738130300AF
:10017000581303000A444FF0000C10F8013B13F031
:10018000070408BF10F8014B1D1108BF10F8015BF0
:10019000641E05D010F8016B641E01F8016BF9D1E3
:1001A00013F0080F1EBF10F8014BAD1C0C1B09D13A
:1001B0006D1E58BF01F801CBFAD505E014F8016BAC
:1001C00001F8016B6D1EF9D59142D6D3704700003E
:1001D0000023002400250026103A28BF78C1FBD850
:1001E000520728BF30C148BF0B6070471FB51FBD05
:1001F00010B510BD01F0F8FA1146FFF7F7FF12F045
:1002000075F801F016FB03B4FFF7F2FF03BC01F031
:1002100019FB00000948804709480047FEE7FEE750
:10022000FEE7FEE7FEE7FEE7FEE7FEE7FEE7FEE7A6
:1002300004480549054A064B70470000D5F20008FE
:1002400039010008705000207056002070520020C4
:100250007052002014214160704714207047406A9A
:1002600070470000550200085B0200085F020008AA
:100270007502000810B5044604F1100000F0A8FE55
:10028000C4F8F8000148C4F87C0110BD64020008FD
:10029000F8B5E6B004460D4616461F460A4906A8BC
:1002A00000F05AFB70996F9A0591049200973346BB
:1002B0006E996D9A039102922A466C99019121469A
:1002C00000F060F867B0F0BD70020008F8B5E6B065
:1002D00004460D4616461F46094906A800F03CFB99
:1002E0006F996E9A0491039200976D996C9A02919E
:1002F000019233462A46214600F087F867B0F0BDE8
:100300007002000838B500281CBF01680029184A8F
:1003100023D1184B1C684FF6F0710C404CF240256D
:10032000AC421FBF1B6819404CF27024A14212D18D
:10033000114D296879B911490B68C3F30B03B3F563
:100340008A6F1FBF0968C1F30B0140F283439942D2
:1003500004BF0121117028B905E0094B994204BF7F
:10036000012111704068BDE8324011F08FBD00BF1F
:100370006001002000ED00E0002004E00010005CBF
:10038000000037482DE9F04104460D462168164625
:100390004A681F4690478046B8F5403F2ED12268F4
:1003A0000A999368204698478046B8F5403F25D182
:1003B0002368089A0799D3F80CC02046E047804686
:1003C000B8F5403F1AD12368069A39461F6920467E
:1003D000B8478046B8F5403F10D1236829465D698B
:1003E00032462046A8478046B8F5403F06D12368EC
:1003F0000B9A09999D692046A847804621680A689A
:10040000204690474046BDE8F0812DE9F041044682
:100410000D46216816464A681F4690478046B8F543
:10042000403F2ED122680A9993682046984780461B
:10043000B8F5403F25D12368089A0799D3F80CC036
:100440002046E0478046B8F5403F1AD12368069A17
:1004500039461F692046B8478046B8F5403F10D15D
:10046000236829465D6932462046A8478046B8F58C
:10047000403F06D123680999DD6900222046A8473C
:10048000804621680A68204690474046BDE8F081D2
:100490004FF4403070470000F0B50C4685B011466F
:1004A00000281A461CBF0568002D0B4B11D082B1E5
:1004B00004B971B90D9860B10F9E0E9F0A9B02900E
:1004C000049603970B980C9E009001962046A8472F
:1004D0000346184605B0F0BD0200030010B500F059
:1004E00033FA4FF4403400280EBF034C4FF4C07170
:1004F00001F03CF9204610BD0200030010B504468F
:1005000000F022FA08B9054810BD0021A160D0F81A
:100510007C21116888474FF4403010BD0200030071
:1005200070B504460D4600F00FFA064E40B1D0F803
:100530007C0141688847A84224BF65604FF440367B
:10054000304670BD020003002DE9FF4715000C4640
:1005500000D02CB1064600F0F7F95FEA000801D19F
:100560006448C3E0D8F8F80001684A689047B0F5DD
:10057000003F17D1D8F87C118A68404690478146E1
:10058000B9F1810F80F09E80A94508F1FC0A17D2CD
:10059000D8F8F8000368D3F80CC02A462146E04793
:1005A000B0F5003F40F08E80D8F8F8000368D3F82B
:1005B00010C06A465146E047B0F5003F76D10AE0E8
:1005C000002004E0215C0AF800100098401C009014
:1005D0000098A842F6D34FF0000C4749474A484BD1
:1005E00001AC0098844558D2D3E9007001ADC5E94B
:1005F0000070107800281ABF042086464FF0000EC5
:10060000085854F80E5028443E4D05600127D0F894
:1006100000E08760019D4F681AF80C007D408EEA6B
:10062000050585F0040E65680F687D4085F0FC05C2
:10063000754485F0A30568400AF80C000CF1010C24
:10064000CFE7D3E9004501A8C0E9004510782E4D59
:10065000002814BF4FF0040E4FF0000E01A874469E
:1006600051F80EE00459A6440127CEF80050DEF8F8
:100670000040CEF808704D68019F40687D406C4096
:100680000D68684084F0040480F0FC00041984F0D4
:1006900057040AF80C400CF1010CCC45D1D3D8F822
:1006A000F80001684A689047B0F5003F0AD1D8F8D1
:1006B000F8000368D3F80C804A465146C047B0F5AD
:1006C000003F01D0114811E0002006E05AF8201048
:1006D00081F06A314AF82010401CB0EB990FF5D335
:1006E000B06840F00100B0604FF4403004B0BDE8A5
:1006F000F08700BF020003000C39010860010020F0
:1007000020090008ADBE4ED70DBE75A10100030043
:1007100038B50C46017A1546CA0702D500F014F91F
:1007200008B9084832BDD0F8F80003682146DC68F3
:100730002A46A047B0F5003F01D0034832BD4FF430
:10074000403032BD02000300010003002DE9F841F2
:1007500091B005460E461746402101A801F006F863
:10076000297AC80704D5284600F0EEF8040002D123
:10077000DFF8A4804BE0D4F8F800DFF8A08003682D
:10078000D3F810C06A4601A9E047B0F5003F3ED15A
:10079000D4F8F80001684A689047B0F5003F36D1B8
:1007A000D4F87C118A6820469047D4F8F830024685
:1007B00018461B68D3F80CC004F1FC01E047B0F503
:1007C000003F24D1D4F87C0141688847D4F8F83040
:1007D000024618461B68D3F80CC001A9E047B0F5E3
:1007E000003F14D1D4F8F80002686968936898470C
:1007F000B0F5003F0BD1D4F8F80003681C693A4605
:100800003146A047B0F5003F08BF4FF4403840469E
:1008100012B0BDE8F08100BF020003000100030038
:100820002DE9F841A5B0074688461646402115A88F
:1008300000F09CFF00220492402105A800F096FFE2
:10084000387AC1075ED5384600F07EF8050059D0E9
:10085000D5F8F8002D4C0368D3F810C06A4605A9F6
:10086000E047B0F5003F3CD1D5F8F80001684A6890
:100870009047B0F5003F34D1D5F87C118A682846FE
:100880009047D5F8F830024618461B68D3F80CC0DC
:1008900005F1FC01E047B0F5003F22D1D5F87C011D
:1008A00041688847D5F8F830024618461B68D3F8E7
:1008B0000CC005A9E047B0F5003F12D1D5F8F8000B
:1008C0000268796893689847B0F5003F09D1D5F878
:1008D000F80003681D6904AA15A9A847B0F5003FF0
:1008E00001D020460FE00A4B0A490B4A03960291B9
:1008F000019240461C68049B009415AA796800F098
:1009000051FD00E0054826B0BDE8F081010003007C
:1009100014390108936E030026C703000200030088
:1009200004B0010100170145DD040008FD040008C2
:100930002105000891040008490500081107000876
:100940004D070008210800080168024A914218BFBB
:10095000002070472809000810B5040008BF0024D3
:1009600004D003482060204609688847204610BD0F
:10097000280900082DE9F04F0646D0B00868F56D4B
:10098000D6F860E0726EB76EF36E00BA00906C46F7
:10099000486800BA60600DF14008886800BAA0603D
:1009A000C86800BAE060086900BA2061486900BA06
:1009B0006061886900BAA061C86900BAE061086A2C
:1009C00000BA2062486A00BA6062886A00BAA0620F
:1009D000C86A00BAE062086B00BA2063486B00BACC
:1009E0006063886B00BAA063C86B00BAE063402004
:1009F00058F80C1C58F820CC58F838AC8CEA010197
:100A000058F840CC8AEA01018CEA01094FEAF979E9
:100A1000401E48F8049BEBD187EA020000EA0E0072
:100A2000784010EBF5610098DFF824C44118614468
:100A3000C81882EABE032B404FEAF06153405918B0
:100A4000636859186144CF194FEAB50383EABE01C0
:100A5000014081EABE0111EBF765A1684D196544BB
:100A6000A91883EAB0023A404FEAF1655A40551995
:100A7000E26855194FEAB70282EAB00765440F40B1
:100A800005EBBE0E97EAB00717EBFE6527697D19E7
:100A90004FEAB10782EA0701654401EA0E01EB184B
:100AA000514011EBF36561694D194FEABE0187EAC8
:100AB000010E65440EEA030E15EBB0008EEA070E38
:100AC0000EEBF065D4F818E075446544AA1881EA85
:100AD000B30505404FEAF26E4D40AE44E569AE44C1
:100AE000E64477444FEAB00080EAB30E0EEA020E05
:100AF0008EEAB30E0EEBF765D4F820E0754465443A
:100B0000691880EAB2053D404FEAF16E4540AE44B7
:100B1000656AAE44E6440EEBB3034FEAB70787EAD3
:100B2000B20E0EEA010E8EEAB20E0EEBF365D4F8A9
:100B300028E075446544281887EAB1051D404FEA4E
:100B4000F06E7D40AE44E56AAE44E6440EEBB20280
:100B50004FEAB30383EAB10E0EEA000E8EEAB10E3D
:100B60000EEBF265D4F830E075446544EF1983EA82
:100B7000B00515404FEAF76E5D40AE44656BAE447C
:100B8000E6440EEBB1014FEAB20282EAB00E0EEA81
:100B9000070E8EEAB00E0EEBF165D4F838E075441E
:100BA0006544EB1882EAB7050D404FEAF36E5540F5
:100BB000AE44E56BAE44E6440EEBB0004FEAB10143
:100BC00081EAB70E0EEA030E8EEAB70E0EEBF06561
:100BD000D4F840E07544654481EAB30EAA180EEAE1
:100BE000000E4FEAF2658EEA010E7544DDF844E02E
:100BF0004FEAB000754480EAB30E65440EEA020E77
:100C000015EBB7078EEAB30E0EEBF765DDF848E09B
:100C10004FEAB202754480EA020E65440EEA070EFE
:100C200069188EEA000E0EEBF165DDF84CE07544B4
:100C3000654405EBB3034FEAB70E14270DF1500CD2
:100C4000DFF810528EEA010B82EA0B0B0BEBF36A12
:100C50005CF804BBDA44AA44504483EAB10B4FEA7F
:100C6000F06A8EEA0B0BDA445CF804BBDA44AA445F
:100C7000524480EAB30B4FEAF26A8BEAB10BDA44D2
:100C80005CF804BBDA444FEAB000AA4480EA020BE5
:100C9000D6448BEAB30B0BEBFE6A5CF804BBDA4478
:100CA0004FEAB202AA4482EA0E0B0AEBB10180EAD3
:100CB0000B0B0BEBF16A5CF804BBDA447F1DAA4412
:100CC000282F0AEBB3034FEABE0EBBD33C2F61D3F0
:100CD000502F4DD204EB870CC7F154075E4CA7FB95
:100CE00004A504465D4FA8088EEA010A82EA0A0AB2
:100CF0005CF804BB0AEBF3655D447D192C1983EAAB
:100D0000B10A4FEAF4658EEA0A0A55445CF804AB6E
:100D10005CF804BB55447D19AA1884EAB30A4FEA6B
:100D2000F2658AEAB10A55445D444FEAB4047D197C
:100D300084EA020AAE448AEAB30A0AEBFE655CF86A
:100D400004AB55444FEAB2027D1982EA0E0A15EB54
:100D5000B10184EA0A0A5CF804BB0AEBF1655D4460
:100D60007D1915EBB303401E4FEABE0EBCD12046E1
:100D7000F46D1B19F365336EC9183166716E7144D9
:100D80007166B36ED218B266F16E4018F06650B05C
:100D9000BDE8F08F4EEA010B0EEA010A0BEA020BE6
:100DA0004BEA0A0A0AEBF36554F827A0DFF8B0C053
:100DB000554443EAB10B654403EAB10A0BEA0E0B52
:100DC00028184BEA0A0A7F1C0AEBF06554F827A0A2
:100DD000554440EAB30B654400EAB30A0BEAB10B91
:100DE000AA184BEA0A0A7F1C0AEBF26554F827A0FE
:100DF00055444FEAB00040EA020B654400EA020A9B
:100E00000BEAB30BAE444BEA0A0A7F1C0AEBFE6501
:100E100054F827A055444FEAB20242EA0E0B65444B
:100E200002EA0E0A0BEA000B15EBB1014BEA0A0AC3
:100E30007F1C0AEBF16554F827A055447F1C6544DC
:100E40003C2F05EBB3034FEABE0EA3D340E700BF30
:100E50009979825AA1EBD96ECDCCCCCCD6C162CADD
:100E6000DCBC1B8F00B581B00168074A914200D1FC
:100E700010B9064801B000BD7C2100F077FC4FF4AA
:100E8000003001B000BD00BF700F00080300020079
:100E90002DE9F0410B4A92E8F85188B0694681E8A3
:100EA000F8510268084B9A4200D118B9074808B0B7
:100EB000BDE8F0811422083000F003F908B0BDE865
:100EC000F08100BF500F0008700F000803000200FF
:100ED000152904D20268044B9A4200D108B903488C
:100EE0007047083000F0FCB8700F000803000200E3
:100EF00010B481B013460268074CA24200D118B961
:100F000001B010BC0548704701B000F1240210BCCC
:100F1000083000F0E9B800BF700F000803000200BD
:100F200010B481B013460268074CA24200D118B930
:100F300001B010BC054870470A4601B000F1240119
:100F400010BC083000F024B9700F00080300020044
:100F50000123456789ABCDEFFEDCBA987654321099
:100F6000F0E1D2C30000000000000000000000001B
:100F7000650E0008910E0008D10E0008F10E000861
:100F8000210F00087509000855100008A11000087D
:100F90005D100008F0B5A3B004460B4802900D4662
:100FA00016461F46094B0822402104A800F085F888
:100FB00028980190009733462A46214602A800F05F
:100FC0001BF823B0F0BD00BF700F0008840F0008AD
:100FD00010B5040008BF002408D00548054B206068
:100FE0000822402104F1080000F067F8204610BDF7
:100FF000700F0008840F00082DE9F04104460E46EA
:10100000216817464A681D4690478046B8F5003F5C
:1010100019D1226806999368204698478046B8F50A
:10102000003F10D123683146DE683A462046B0477B
:101030008046B8F5003F06D12368079A29461D6906
:101040002046A847804621680A68204690474046C7
:10105000BDE8F08120225C3000F0DFBAF0B5846892
:10106000A308002204F0030407E000F15C0555F832
:10107000226035BA41F82250521C9A42F5D3002220
:101080000BE000F15C0502EB830755F82360D50007
:10109000C5F11805EE40CE55521CA242F1D3F0BD69
:1010A00030B5C46803690022E31AD5188C5C054486
:1010B000521C082A2C77F8D330BD0360C16002614E
:1010C000704738B5044615460022626023685A68A6
:1010D000904700206061A061A5604FF4003032BDF0
:1010E00081604FF4003070472DE9F84304462079C1
:1010F000D4F80C80450748BF244845D466691D468E
:10110000A8F1010000EAD60306EBC506B6EBC50F51
:10111000666102D2A669761CA6611746A66906EB2F
:101120005576A6610E46E918884225D2A8EB030938
:101130004A463146F81800F070FA226813683946BA
:101140000FE04246384600F068FA23681A683946CC
:101150002046904707E0311811F00300F1D12268D2
:10116000136820469847484600EB0809A9F1010199
:10117000A942F0D3002300E000202A1A3118F81801
:1011800000F04BFA4FF40030BDE8F2830400020097
:101190002DE9FC4F024685B0D0681369DFF86CC1B9
:1011A000DFF86C81A0EB030A506840F00400506047
:1011B000002703A802900DF10C0ED8E9003403A813
:1011C000544DC0E900342878534D00280CBF00234B
:1011D000042399465CF803305EF809402344012655
:1011E0001D601C689E60DCF80430039DDCF80090F4
:1011F000DEF804605D406540484C654089EA0606BB
:10120000474C66407519474C6540D8E9006B03AC04
:101210000028C4E9006B0EBF002404200424029EB1
:101220005CF80000345920183F4C04600126046823
:1012300086600398029E43406340384C7068634068
:1012400089EA0000364C6040034438484340280097
:1012500018BF01205B1E9B41042F2CBFC0B2D80FCA
:1012600002F1140353F8200007F00303C3F1030352
:10127000DB00D8400DF807007F1C082F9DD31546D2
:101280000C466A69AB69E868D20842EA4372401EBC
:1012900000EA0207002302409B420AD8524508D2C6
:1012A0008020E0557F1C574516D2AAEB0701E019B4
:1012B00010E08020E05500E0E355E8687F1C87429D
:1012C000FAD32A68136828469847BAF1000F03D06A
:1012D0005146204600F028FA2A68069E059F93682A
:1012E0006946284698472A68D2F800902146284641
:1012F000C8472B68DA683946284690470EB1A86877
:1013000030604FF4003007B0BDE8F08F0C390108B1
:101310009C140308600100205FC51093048500122F
:10132000FC68017AC0F524FF24AF33D426AF698B63
:10133000F8B501240094002300240DE0009D065D13
:101340000F5D7E40F643761CF60F86F001063540B1
:101350000095641C009DEB189442EFD31846F2BD33
:10136000F8B5002301240094002A11E0009C8518A0
:101370008F1815F8016C17F8015C6E40F643761C67
:10138000F60F86F0010634400094009CE318521ECC
:10139000ECD11846F2BD00003113000861130008BB
:1013A000010000002DE9F84F1D46DDF828900B9F45
:1013B0000D9C4FF0FF3300930E469246D9F800B0D3
:1013C000804632465146D847834664B3D9F8043044
:1013D00032465146404698476FEA0B02521C42EA99
:1013E0000B0200996FEAD2735B1C1940C243009153
:1013F000521C024300996FEAD2735B1C19400091A2
:1014000086F05531484087EA000181F0553121606E
:1014100080F05531C943491C0843009A6FEAD070E7
:10142000401C82430092D9F80800012809D1754078
:10143000E943491C0D4300986FEAD572521C904352
:101440000AE0F11C85EA9102D243521C1543009830
:101450006FEAD5735B1C984386F0AA36009086EA43
:101460000B0686F0AA33F243DB430C98C2F3C0723A
:101470005B1C42EAD3720099D243521C9143009103
:10148000774000998843009987F0AA370F40384386
:10149000BDE8F28F53EA020C00F069802DE9F04BB1
:1014A0004FF00006002B1FBFB3FA83F503FA05F4D3
:1014B00024FA05F65E4012BF1643B2FA82F502FA2C
:1014C00005F4C5F120051EBF22FA05FC44EA0C0410
:1014D000203556EA044C4FEA144418BF641C4FF000
:1014E00000084FF00009904271EB030C39D300293A
:1014F00019BFB1FA81F701FA07F6B0FA80F700FADE
:1015000007F6C7F120071EBF20FA07FC46EA0C06C3
:101510002037B6FBF4FCA7EB0507103F07F01F0BC5
:10152000CBF120062CFA06F60CFA0BFB44BFB346AF
:101530000026202FA4BF5E464FF0000B5BEA060C8E
:1015400008BF4FF0010B19EB0B0948EB0608ABFB8A
:10155000027C06FB02CC0BFB03CCC01B71EB0C0125
:10156000C1E70B46024641464846BDE8F08B13B53D
:10157000084318BF4FF0FF300146AFF30080BDE8CD
:101580001C40704740EA010310B59B070FD1042AA5
:101590000DD310C808C9121F9C42F8D020BA19BA3E
:1015A000884201D9012010BD4FF0FF3010BD1AB1A3
:1015B000D30703D0521C07E0002010BD10F8013BF8
:1015C00011F8014B1B1B07D110F8013B11F8014B1F
:1015D0001B1B01D1921EF1D1184610BD10B5431C42
:1015E00002E010F8011B71B18107FAD14FF001320E
:1015F00002C88C1A8C4314EAC211F9D0C01A0A0628
:1016000003D0C01E10BDC01A10BD0A0401D0801E38
:1016100010BD0902FCD0401E10BD032A40F23080EC
:1016200010F0030C00F0158011F8013BBCF1020F23
:10163000624498BF11F801CB00F8013B38BF11F8A4
:10164000013BA2F1040298BF00F801CB38BF00F8BB
:10165000013B11F0030300F02580083AC0F0088038
:1016600051F8043B083A51F804CBA0E80810F5E71C
:10167000121D5CBF51F8043B40F8043BAFF30080FF
:10168000D20724BF11F8013B11F801CB48BF11F874
:10169000012B24BF00F8013B00F801CB48BF00F844
:1016A000012B704710B5203AC0F00B80B1E81850FC
:1016B000A0E81850B1E81850A0E81850203ABFF43C
:1016C000F5AF5FEA027C24BFB1E81850A0E81850DB
:1016D00044BF18C918C0BDE810405FEA827C24BF2F
:1016E00051F8043B40F8043B08BF7047D20728BFBD
:1016F00031F8023B48BF11F8012B28BF20F8023B0C
:1017000048BF00F8012B704702F0FF0343EA0322B1
:1017100042EA024200F00AB802F0FF0343EA032261
:1017200042EA024200F024B84FF000020429C0F05F
:10173000128010F0030C00F01B80CCF1040CBCF103
:10174000020F18BF00F8012BA8BF20F8022BA1EB55
:101750000C0100F00DB85FEAC17C24BF00F8012B3A
:1017600000F8012B48BF00F8012B70474FF0000232
:1017700000B5134694469646203922BFA0E80C5087
:10178000A0E80C50B1F12001BFF4F7AF090728BF62
:10179000A0E80C5048BF0CC05DF804EB890028BFDE
:1017A00040F8042B08BF704748BF20F8022B11F007
:1017B000804F18BF00F8012B704770477047704783
:1017C00010B500F009F8006810BD10B5044600F02F
:1017D00003F8046010BD0000004870476401002059
:1017E00000487047640100207546FFF7F9FFAE46D8
:1017F00005006946534620F00700854618B020B51D
:10180000FEF716FDBDE820404FF000064FF0000740
:101810004FF000084FF0000BAC46ACE8C009ACE854
:10182000C009ACE8C009ACE8C00921F007018D4649
:10183000704710B50446AFF300802046BDE8104065
:10184000FEF7E1BC01491820ABBEFEE7260002000E
:1018500070470000B0B5044600688168490701D4AC
:101860000020B0BD8168890704D48168464A1140D0
:101870001031816001F09EFE0546206880684007B7
:10188000EED501F097FE401B0328F6D32068806850
:101890004007F2D5714607F0CEFD8E46B0BD00BFC1
:1018A000B0B50168044688688A6880074FF0000078
:1018B00020D412F001021DD0886800F00500012834
:1018C00016D18868304A10400230886003200860D2
:1018D00001F070FE054620688068C0070BD001F05B
:1018E00069FE401B0328F6D320688068C007F2D049
:1018F00007F0A1FDB0BD0020B0BD00BF7CB504461F
:101900000020019021688A68D20707D11E4E88689E
:1019100006F12F02104202D007F08DFD7CBD8868D1
:10192000304040F00100886018480068000204D48C
:10193000607E01280ED100207CBD15481549006845
:10194000B0FBF1F00130019001980028F0D001982F
:101950000138F8E701F02EFE054620680168C90746
:10196000E9D18168C90704D18168314041F00101A2
:10197000816001F01FFE401B0328EED32068006841
:10198000C007EAD1C8E700BFE8FFFF7F0827014092
:1019900058010020400D0300BFB500250446039503
:1019A000CDE9015507F0BEFA144800F0C3FE08B1B6
:1019B00000F0FAFB11480395CDE9014501A900F0BB
:1019C00041FF08B100F0F0FB0C4801F0D7F908B175
:1019D00000F0EAFB094C4FF0FF31204601F076F9A8
:1019E000204601F0F3F9204601F03EF80546204676
:1019F00000F0F4FF284604B0B0BD00BFB44B002097
:101A0000BCB56B4C00204FF47A750DF10602A6218F
:101A100001238DF807008DF806000095204601F09F
:101A2000CBFE642001F0A7FB0DF107022046A621A2
:101A30000123009501F066FE9DF80700BCBD00BFC4
:101A4000F8B50246002001210DF10F038DF80F00BB
:101A50006420CDE90031A62101230290544801F011
:101A600007FF9DF80F0004B080BD00BF70B586B0C1
:101A700014460D460646642006210DF1120201238C
:101A8000CDE9002102904A48A621322201F0F0FE61
:101A9000BDF812003080BDF814002880BDF8160093
:101AA000208006B070BD00BFBCB5FFF7A9FFE528D8
:101AB00003D0284B009008F091F9002000F04EF878
:101AC000082000F04BF8082000F04CF80F4C2E20B6
:101AD0000021A0472720FF21A0470D4D2420297871
:101AE000A0472F20E721A04769782520A047A978A3
:101AF0002620A0472E203821A0472D203821A0479E
:101B00003020BDE8BC40FFF79BBF00BF8D1B000825
:101B1000640000201CB5FFF773FFE52803D00D4BD0
:101B2000009008F05BF92E20002100F02FF80A4CFD
:101B30000320A0470020A0470820A0470D2000F068
:101B400011F82E20C72100F021F80120BDE81C402B
:101B500000F00CB88A9401085D1B00080146312092
:101B600000F014B801462C2000F010B810B504465F
:101B70002D20FFF765FF00F0F70040EAC400C1B276
:101B80002D20BDE8104000F001B80000F8B5024675
:101B90008DF80F104FF47A7001210DF10F03CDE98C
:101BA000003102900248A621012301F0D5FE8FBD2D
:101BB000784C0020F0B589B005AE0C4605460021F2
:101BC0001022304610F0B5FB30463146224610F068
:101BD000B3F99DF914000021B0F1FF3F06DD0F2994
:101BE0000CD007F0ACFCFAE707F0A9FC0F29FBD1F9
:101BF0009DF82300872181EA400002E09DF8230040
:101C000040008DF82300D4F8140110280AD104F202
:101C100001100021102936D0425C735C5A404254B6
:101C20000131F7E79DF914100022B1F1FF3F06DD05
:101C30000F2A0CD007F010FEFAE707F00DFE0F2A6E
:101C4000FBD19DF82310872282EA410102E09DF832
:101C5000231049008DF823108021204480F80111C1
:101C60000021D4F8140101301028C4F81401F4D371
:101C700004F201100021102905D0425C735C5A4027
:101C800042540131F7E70020102803D0211807F053
:101C9000DDFCF9E701AE04F1F1011022304610F04D
:101CA00034FB30462946224610F046F905A80021AB
:101CB000102210F03EFB09B0F0BDB0B50446F13083
:101CC00000211022002510F034FBC4F814512046E6
:101CD0000021F022BDE8B04010F02BBB02460846C0
:101CE000102110F085BA2DE9F04385B00E46D0F8EA
:101CF00014111446804699B308EB0100C1F1100598
:101D000027463146A54238BF2F4600F20110BAB22D
:101D100010F0FBFAD8F81401A5423844C8F81401B1
:101D200046D2102844D30020102804D008EB00012C
:101D300007F08CFCF8E708F1F1050DF10409102219
:101D40004846294610F0E1FA48464946424610F016
:101D5000F3F828464946102210F0D7FAE41B3E4417
:101D600008F1F10701AD112C1AD30020102805D07D
:101D7000395C325C514039540130F7E72846394626
:101D8000102210F0C2FA28462946424610F0D4F834
:101D900038462946102210F0B8FA103C1036E2E717
:101DA00008F20110A2B2314610F0AFFAC8F814419F
:101DB00005B0BDE8F083FEE72DE9F041CCB051B3AA
:101DC000DDF84881B8F1000F25D0074602A81C466F
:101DD00015460E46FFF771FF01A9204600F0EEFB05
:101DE0000446C8B90198411C02A8FFF777FF27B144
:101DF00002A839461022FFF776FF02AF31462A4685
:101E00003846FFF770FF48A83946FFF7D3FE4898D9
:101E1000C8F8000000E0022420464CB0BDE8F08184
:101E2000B8B170B50C4C4FF0FF3200238B420ED08E
:101E3000C55C6A400025082D07D202F00106013575
:101E40007642264086EA5202F5E70133EEE7D043B8
:101E500070BD0020704700BF2083B8EDB0B586B0DC
:101E600000F0C4FF00F0CCFF00F0C4FF032001210C
:101E70000490002002910390059003F0C3FE03F04C
:101E8000C1FE4FF480500E4C019001AD2046294612
:101E900001F0BEFA4FF4005029460190204601F0AF
:101EA000B7FA20464FF48051002201F07DFB204616
:101EB0004FF40051002201F077FB06B0B0BD00BF27
:101EC00000040048014801F063B800BF184C00202E
:101ED00010B51049436C104C01F1640223F0030368
:101EE000C2640268A24238BF04F57E71194414230B
:101EF00081646FF00701A24251FA82F1B1FBF3F164
:101F000028BF0731012201F01F0102FA01F101652A
:101F100010BD00BF1C0802400804024010B5436811
:101F200007490124543003F07F0301F14002013BD3
:101F300001EB830103F0030304FA03F30EC010BDA9
:101F400000090240F0B500F14C0670CE656016B194
:101F5000D0E91645656004688568D0E910600127FE
:101F600000F01C00102D07FA00F070600846636056
:101F700008BF1046A06008BF0A46E260F0BD704787
:101F80001FB504460020022CCDE90200CDE9000077
:101F900003D0032C22D1022000E001208DF80000A4
:101FA000180A8DF804208DF801108DF807308DF88F
:101FB0000800100C8DF80600100A22468DF8050066
:101FC000080C8DF80300080A01218DF8020068460C
:101FD0000CF072FD002818BF0E2000E00A2004B0AB
:101FE00010BD00002DE9F04F8DB050480026DFF8FD
:101FF0003491DFF834A14E4FDFF838B14FF400715F
:10200000CDE90566CDE90366CDE9016606604A487B
:10201000C9F80060CAF800603E60CBF80060066056
:1020200007AC20460FF0FAFE454D444920460023F8
:102030002A460FF0D1FE434C07F019FD424D4FF0F8
:1020400004082660B8F5806F0ED054F8080011F02F
:1020500003F807F083FE07F0FEFD10F03BFD44F8A7
:10206000080008F10408EDE7364806AA03AB07F0BC
:102070008DFD0398324D35490023002638600698BF
:102080002A46C9F8000007A80FF0A6FE304C07F05A
:10209000EEFC2D4D26600426B6F5806F0BD0A059BE
:1020A00010F0DAFF07F05AFE07F0D5FD10F012FD30
:1020B000A0510436F0E7264805AA02AB07F066FDFA
:1020C00002981F4D234900230026CBF800000598F5
:1020D0002A46CAF8000007A80FF07EFE1E4C07F043
:1020E000C6FC194D26600426B6F5806F0BD0A059AA
:1020F00010F0B2FF07F032FE07F0ADFD10F0EAFC81
:10210000A0510436F0E7144804AA01AB07F03EFDE5
:102110000198094908600498044908600DB0BDE8B9
:10212000F08F00BFE8010020E4010020E001002062
:10213000A4330020A8330020AC330020A41B0020CF
:102140007C0C0020B43300200000703FA42300204A
:10215000B43B0020A42B0020B4430020012001F058
:102160004DB9022001F04AB9402001F047B90020E2
:102170007047000010B504460CF0C0FA0649084B41
:10218000064A0012C4E9021306492261216011F0D7
:1021900059F96060002010BD00004842AB03050003
:1021A0000D093E0000007A44EFF3108072B6FEE79E
:1021B000B0F1006F0BD3A64AA64B126803EA822245
:1021C0006FF078431A44824228BF00F019B84FF0EC
:1021D000FF30704780B501F073F810B16FF0040064
:1021E00080BDBE48816841F0404181604CF2FA31C7
:1021F000016001F021F8002818BF6FF0040080BDD5
:102200007FB50546002003904DB10C46FFF7E2FF75
:10221000064680BB01F054F818B1FB262BE0FA26E5
:1022200029E002208B496FF0006300908848006825
:1022300001EA802005F17841B1FBF0F202FB1011B8
:10224000CA0A019262191A44B2FBF0F303FB102090
:10225000C00AA0EBD12001300290684603A900F02B
:1022600091FF6FF00106022808BF0126002808BF71
:10227000064600F0E1FF70B204B070BD40B139B164
:1022800080B592B20EF068FA0020BDE8804000E010
:10229000FA2040B2704700006F4908600020704784
:1022A000B1F1006F0ED310B5694B6A4C1B6804EA9C
:1022B00083236FF0784423448B42BDE8104028BF4D
:1022C000FFF7DCBF4FF0FF30704700BF2DE9F04F44
:1022D00085B0B0F1006F0BD35D4D06465D4C89466D
:1022E0006FF07841286804EA80200844B04204D2A4
:1022F000FF2778B205B0BDE8F08FFA27002EF8D09E
:10230000B9F1000FF5D046EA0200934610F007003D
:10231000EFD1FFF75FFF07460028EAD100F0D0FFBA
:1023200008B1FB27E5E7286806F178416FF0006304
:10233000DA46494FB44604EA8020B1FBF0F202FBD2
:10234000101106EB0B021A44B2FBF0F303FB102052
:1023500032466FF3DF22C40AA4EBD12001300128FA
:1023600088BFC2F5006A4FF000600094CD0AA54214
:1023700068D800EBC5203146CDF80CA0CDE901C5E9
:1023800004900020504507D2D1E900231A400132C1
:1023900006D108300831F5E7CDF810C04D461BE0F6
:1023A0003868002850D004994FF40062E046FFF7E7
:1023B00065FF404639681FFA8AF26FF3DF20084450
:1023C00049460EF0C9F904984FF40061FFF718FF71
:1023D000E0BB3D684FF4006A4FF00008D04518D2CA
:1023E000049805EB080455F80820636800EB08071B
:1023F0000120394600F02AFF00BB58F80500D7E954
:102400000012484061685140084317D108F108089C
:10241000E4E7DDF80CA0DDF804C04FF400600E4FD7
:10242000D144D444ABEB0A0ABAF5006F28BF824608
:10243000029D009C4FF00060013598E7FC2700F0FA
:10244000FBFE56E70027FAE7FA27F8E7FE27F6E74C
:10245000E075FF1F00FCFF03504E0020B0B51F4A7F
:10246000536843F480235360EFF31083EFF3108439
:1024700072B6402420C9013C20C02506FAD110685C
:10248000C003FCD483F31088B0BD00BF70B5134EF9
:10249000044601F08FF805463068C00306D501F008
:1024A00089F8401BA042F7D3032070BD3068C107F4
:1024B00001D0012131604CF2FA31084009D00849BD
:1024C00048603060012070BD01F074F8401BA042EC
:1024D000EAD230684003F7D4002070BD10400058A5
:1024E000544E002080B50CF0EDF8B0F5616F01D9C5
:1024F000FE200DE0B0F5E16F01D2002008E00549B3
:10250000C0EBC01001EB40004FF4E161B0FBF1F013
:10251000C0B280BD1006F9FF10B585480068411CA7
:1025200000D010BD01F050F8044601F053F84440CB
:1025300001F056F8604010BD008871B949F6B0212D
:1025400042F210738A4238BF4FF47A73B2F5616F6A
:1025500038BF6423834228BF1846002808BF0120E3
:102560007047000070B50B4A92F820307BB1002410
:1025700002F11C059C420AD20E78864208D00E1D3C
:10258000A94208BF02F10C0631460134F2E70021EE
:10259000084670BD540C002010B5074A0223043AC7
:1025A0003BB112F8044F013B8442F9D100200A608C
:1025B00010BD0B2010BD00BF0001002010B5084A5F
:1025C0000023126803F11104BB2C06D013441B7CBA
:1025D00083422346F6D107F042B8032010BD00BF66
:1025E000381B002061B1013803280BD8DFE800F068
:1025F000020C12190E48006802690A6001690EE0B7
:1026000009207047052070470948006842690A6040
:10261000416904E00648006882690A6081690162D4
:1026200003E003480068C06908600020704700BFED
:10263000780C0020E0B50B498DF8010091F874206A
:1026400091F8400091F880108DF802200E220029A8
:10265000694608BF0D228DF800200AF06DFEC0B259
:102660008CBD00BF7C850020FEB56846FFF782FD6B
:10267000019810F0ABFE06B080BD0000F0B585B04B
:10268000064613480D461349845730460AF01EFC8F
:10269000014611480023EAB2476A0120072E0BD1F8
:1026A0000525CDE90053CDE902204FF47A700023CF
:1026B00004FB00F2002007E00825CDE90053CDE936
:1026C0000220012022460123B84705B0F0BD00BF1B
:1026D000CC390108AC390108C43A01080348016843
:1026E00002689142FBD1C843704700BF08280040F0
:1026F000B0B504460E4801684A1C08D009BA6160AA
:102700004168E1704268100E110C120A0CE000F0F2
:102710005BFF054600F064FF054400F05BFF010E1F
:102720006560020CE170010A6170A2702070B0BD9A
:102730008075FF1FF8B504460020009094F85400FF
:10274000012801D1022544E0012084F854002046EC
:10275000FFF7A6F8054620688268A16DD20728D148
:1027600021F4817148F203030231A165C168C26896
:102770009A4301EA030732490023C2600022082B72
:1027800029D086680E4006F1004686608668B6F15C
:10279000FF3F07DC009E01360096009EB6F52E3FF7
:1027A000F4D30CE0D0F8B460013306F07F06324475
:1027B000E5E741F01000002184F8541008E0002003
:1027C000012584F85400A06D40F0100020F00200B4
:1027D000A0652846F8BD83680B4043F00103836081
:1027E000D0F8B43023F07F0343EAD202C0F8B4201B
:1027F0008268114041F00201816000F0DBFE064674
:1028000020688168C90712D000F0D4FE801B03281D
:10281000F6D320688068C007F2D0A06D012540F093
:102820001000A065E06D40F00100E065D1E7C168EF
:102830003943C1600121A06D61F30100BBE700BF16
:10284000E8FFFF7FF8B50022009290F85420012A9B
:1028500001D10221B3E0012280F85420026893687C
:102860005B0711D403694C6843F00403022C11D1B7
:10287000544CA34219D10B68574CD94361EA040167
:10288000946A2140916211E0816D41F020018165DF
:10289000012191E04B4DAB421AD1144654F8285F08
:1028A0000B681E466FF39F4635E00B68B3F1FF3FA0
:1028B00000F38180F349464C0A68A3426BD0454C33
:1028C000A3426BD0414CA34275D102F0A07267E0E5
:1028D0000B689D0393FAA3F5B5FA85F604F01F057E
:1028E00008BFC3F3846606FA05FC076ED0F81CE047
:1028F0000F26AE40B74347EA0C07BEEB940F0766BE
:102900000BD99C0EF64304F00F0404FA05F51446A7
:1029100054F8287F3E4035432560546989682A4D24
:1029200001EA032124EA032429402143B3F1FF3FB4
:10293000516140DCD34A254915688B4208BF15F424
:10294000000105F0E07411D021498B4208BF15F059
:1029500080712BD01F4E0021B34208BF15F48003B5
:102960002AD107F040FA41F4800123E007F03BFA56
:1029700041F400011160BF49BF4A0968B1FBF2F19F
:102980000C2201EB410102EB81010091009991B110
:1029900000990139F9E702F4400201E002F0C07247
:1029A0000B6823F0E0731A440A6004E007F01BFA96
:1029B00041F0807111600021002280F85420084607
:1029C000F8BD00BF0400008000FFFF03001000B04E
:1029D000004000B8002000B4FFFF030070B558B1FC
:1029E0000446806D40F00200A0652046FEF732FFED
:1029F00020B1054620680CE0012530E007F0B2F96F
:102A0000054608B90120A0652068994A81681140EF
:102A10008160416840F29F3200269143416002602C
:102A2000104AC1681140C160016921F04041016153
:102A3000416921F007014161016A01F0F021016261
:102A4000816A86628F48016821F0FE71016020462C
:102A500000F01AF9E665266684F85460A6652846F3
:102A600070BD00BF00023E830068006C704700002C
:102A70002DE9FC4104460020019044B3254655F859
:102A8000580F30B9204600F00BF9002084F85400AC
:102A9000E06521688868C00013D48868744A1040D3
:102AA000754A00F18050886072480068B0FBF2F00F
:102AB000022202EB40000190019810B10198013808
:102AC000F9E78868C00005D406F0B5FC03E00120F2
:102AD000BDE8FC8100208A682B68C2F3800203F005
:102AE0001003D2182A6803D042F010010120BBE085
:102AF00022F4817202322A608A68D2072CD104F152
:102B00000808237E98E8C00146EA8333667E43EADC
:102B1000C633A67E43EA46333B43276B002F28F09B
:102B2000004718BF43F48053B8F1FF3FC8BF4FF4CC
:102B300000173B4394F82C7043EA470394F8207045
:102B4000012F0ED15EB1A66D46F02006A665E66D9A
:102B500046F00106E66504E0D4F810802CE043F46A
:102B60008033666A26B106F4E0763343A66A3343BF
:102B7000CE68424F3E403343CB606368E66C03F05F
:102B800040473E4394F83C70012F0AD104F1400EB7
:102B90009EE880503E4346EA0C0646EA0E0646F0A2
:102BA00001060F69364A3A403243B3F1004F0A61D9
:102BB00018BFB3F1404F1ED1D4E90D324E6926F053
:102BC00007061E434E61B8F1000F4E6926F07006ED
:102BD00046EA02124A611AD0B8F5001F2CD1226EC3
:102BE0000026202E19D022FA06F707F00F070F2F24
:102BF0000BD00436F5E7B3F1804FDDD09A0C214BB2
:102C00001E6862F395461E60D6E7042E05D10A467B
:102C100052F8286F66F00F060DE0E6691C2707EBF7
:102C200086066FF00F0706F01C0607FA06F6164335
:102C30000A4652F8287F1660496901F00701994257
:102C400006D100210122E165A16D62F301010BE0D3
:102C5000A06D40F0100020F00200A06554F85C0F59
:102C600040F00101012025462960BDE8FC8100BF3C
:102C7000E8FFFF6F58010020400D03000102FEFF36
:102C800002FCFF1F0827014000680E49884200D05F
:102C900070470D48016821F400710160704700BF62
:102CA00081B000680749884209D10748016841F4AA
:102CB00000710160006800F400700090009801B09D
:102CC000704700BF00240140600000582DE9F0412A
:102CD000044640690D46082801D1082704E0206811
:102CE000C068C00733D1042700F064FC80466E1C26
:102CF0002068016839420FD1002EF9D000F05AFC4B
:102D0000A0EB0800A84201D8002DF1D1206800688E
:102D10003842EDD106F06FBDA16D41F40071A1659F
:102D2000C16811F4406F21D1A17EF9B9016809078A
:102D30001CD58168490711D4416840F2011221F085
:102D40000C014160A16D91430131A1650EE0A06DC0
:102D500040F02000A0650120BDE8F081A16D41F0A8
:102D60002001A165E16D41F00101E165217E09B914
:102D70000C2101600020BDE8F081000010B5044680
:102D800000688068400703D494F85400012801D1FA
:102D9000022010BD06F0FEFE08B106F09CBF2168BF
:102DA000A06D40F60172084B90431C2200F5807024
:102DB000A0650020E0650A6084F854008A681A4023
:102DC00004328A6010BD00BFE8FFFF7F10B506F037
:102DD00054FE01D1022010BD06F0EBFB20B906F035
:102DE000C1FF08B906F03BFF06F075BF064806F0C4
:102DF000C0BD00BF0448016821F0040101607047B4
:102E0000014806F050BB00BF042004E050B3B0B549
:102E100090F82510022927D1016800F140041CCC4C
:102E20000D6803F01C0325F00E050D60256825F4E0
:102E3000807525600C6824F001040C60012101FA02
:102E400003F35360D0E913235360426D32B113682A
:102E500023F480731360D0E91623536080F82510A3
:102E6000002104E0012107E00421C16301210022C7
:102E700080F82420BDE8B04008467047B0B590F80F
:102E8000251002292BD10168D0E91032846C0D681D
:102E900025F00E050D600D6825F001050D60216817
:102EA00021F48071216002F01C01012202FA01F17B
:102EB0005960D0E913134B60416D31B10B6823F4B5
:102EC00080730B60D0E916134B60002180F824104A
:102ED00080F82520826B2AB19047002102E004216E
:102EE000C16301210846B0BDF8B54FF0010C0028C0
:102EF00046D00368254A7E4F0446196802F580656E
:102F000021F00101196020490E1DB3423CBF00258C
:102F1000C4F2020538BF07F580671F441420B7FBD1
:102F2000F0F08700C4E910570025B3421D6038BF98
:102F3000111D1C2202EA80000CFA00F008602046F5
:102F4000FEF7C6FF606804F148030ECB0138032882
:102F50000D60536007D82046FEF7E0FF04F15402ED
:102F600007CA05604A60E563C4E91555E565C4E92B
:102F70000B55C4E90D5584F8245084F8255000E021
:102F800001252846F8BD00BF0404024000000240AD
:102F9000F0B5D0E910230168042403F01C0316687F
:102FA0000D689C40344201D06F071BD402249C4022
:102FB000344201D0AF071FD426FA03F4240735D5D5
:102FC0002C0733D50C6824F00E040C60012101FAA3
:102FD00003F353600022C16380F8242080F8251099
:102FE000416B1FE00B689B0603D40B6823F00403BE
:102FF0000B605460016B15E00A68920606D40A68FB
:1030000022F00A020A60012280F82520002280F8BE
:103010002420074A02F17C03994288BF02F58062AE
:103020001460C16A11B1BDE8F0400847F0BD00BFAF
:1030300004000240B8B3F8B5044602202B4984F8D6
:10304000250004F10806206801F1080268CE9042CC
:10305000274A38BFA1F5806138BF02F58062142786
:103060000244B2FBF7F29200C4E9101247F6F07284
:1030700001689143016045EA0301626931431143EC
:10308000A2691143E2691143226A114302681143A4
:1030900001602046FEF71CFFA068B0F5804F04D108
:1030A0000020606002E001207047606804F148037E
:1030B00000F07F0501380ECB03280D60536009D85E
:1030C0002046FEF72BFF04F15402002307CA0360D9
:1030D0004A6003E00020C4E91500E06500200121FA
:1030E000E06384F8240084F82510F8BD0004024051
:1030F000F8FBFDBFB0B5044690F82400012801D1CB
:103100000220B0BD06F0C3F913D1022084F82500D7
:103110000020E0632068056825F001050560204671
:10312000FEF710FF2068226B01684AB141F00E01E2
:103130000CE0002084F824008020E0630120B0BD72
:1031400021F004010160016841F00A010160A16CF5
:103150000A68D20303D50A6842F480720A60616D7E
:1031600019B10A6842F480720A60016841F00101F5
:1031700001600020B0BD81B00090009801B00CF05B
:10318000DFB800002DE9F84FDFF82CA105469AF8CA
:103190000000012802D10220BDE8F88F01200024A0
:1031A00089468AF800004FF47A70CAF80440FFF7A5
:1031B0006DF9C8BB2868414B1D4A04289B4607D1BE
:1031C0001968901C0843186006F05DF95B4627E01B
:1031D0004FF0FF301749C9F8000068688846C400FE
:1031E0000646A968084486420FD21868174600EAC6
:1031F000080020431043186006F045F938B96868A4
:10320000083401363A465B46EBE7002002E05B46B5
:10321000C9F80060196840F2FA320024914319603D
:1032200053F8141C53F8141C8AF80040BDE8F88FBA
:103230000200010005FCFEFF2048016841F000414A
:1032400001600068C043C00F704700BF2DE9F8431C
:10325000194F04463878012802D10220BDE8F883CE
:1032600001204FF00009984616460D4638704FF47D
:103270007A70C7F80490FFF709F9C8B90F49012C13
:103280000AD1086840F0010008602E60BFF36F8F1C
:10329000C5F804800D4604E028460D463146FFF788
:1032A000DDF84FF47A70FFF7F1F82968A14329603F
:1032B00087F80090BDE8F883544E00201440005871
:1032C0000648C168B1F1FF3F01DD002070470449A5
:1032D000016004490160C068C00F70470840005891
:1032E00023016745AB89EFCD2DE9FC4FA64A4FF08E
:1032F000000890424FF0070208BF02220025002379
:103300000092019131FA03F608BFBDE8FC8F01225B
:1033100002FA03F616EA010C56D0072208F00C094F
:103320004FEA930E02FA09F4994AB0F1904F52F81D
:103330002E7007EA040A07D0964ADDF800B09042E2
:1033400008BF4FF0010B01E04FF0000B0BFA09F73B
:10335000BA451AD18D49D1F8807027EA0C07C1F817
:103360008070D1F8847027EA0C07C1F884700F6868
:1033700027EA0C070F604F6827EA0C074F60844963
:1033800051F82E70A74341F82E7003212C4601FA04
:1033900005F705680F213D43056008F01C0501FA9B
:1033A00005F56FF0030101EA53020244116AA943D3
:1033B000254611628168B94381604168B14341602B
:1033C000C168B943C160019908F1040802350133AD
:1033D00098E700BF012818BF704780B50648012153
:1033E0000170202000210DF047FA02200021BDE8E5
:1033F00080400DF041BA00BF0C4E002003490A681E
:10340000024208BF70470860FFF7E4BF0C0800588D
:103410002DE9F84F5C4A5E4F4FF000094FF0010B69
:103420004FF0000890424FF0070208BF022200232D
:1034300000920C6834FA03F208BFBDE8F88F0BFA6B
:1034400003F214EA020A00F098804E6806F0030CBA
:10345000ACF10104012C19D80324856804FA08F49E
:1034600025EA040ECD6805FA08F545EA0E058560E3
:10347000C6F3001505FA03FE456825EA020242EA92
:103480000E026FEA040E42605A000CE0032202FAB8
:1034900008F2BCF1030F6FEA020E424603D1424626
:1034A0004FF0030C1FE0C4688D6804EA0E049540D9
:1034B0002C43BCF1020FC46015D109F01C040F2588
:1034C00005FA04FC6FF0030505EA53060644356A65
:1034D00025EA0C0C0D6905FA04F444EA0C04346284
:1034E0004E6806F0030C04680CFA02F204EA0E04BB
:1034F000224316F4403F02603FD009F00C06072239
:1035000002FA06F49A0857F82250A543B0F1904FFA
:1035100005D0204CA042009C08BF012400E00024FC
:10352000B440BC462C4347F82240184A174612685C
:103530004D6842EA0A04EE0258BF22EA0A043C60DF
:10354000AE027A6842EA0A0458BF22EA0A047C60A2
:10355000EE03D7F8802042EA0A0458BF22EA0A04A0
:10356000C7F88040AD03D7F8842042EA0A0458BF68
:1035700022EA0A04C7F88440674609F1040908F101
:103580000208013355E700BF000800480008005852
:103590000800014000040048426902EA0103914327
:1035A00041EA0341816170471823002A08BF28239C
:1035B000C150704703480078012808BF0BF0F0BEE7
:1035C00000207047341B002001480068704700BF8E
:1035D0009075FF1F01480068704700BF9475FF1F7A
:1035E00001480068704700BF9875FF1F90F84120A0
:1035F000202A03D190F84020012A01D1022111E0B4
:10360000242280F841200268136823F0010313602C
:10361000136823F48053136013681943734605F04D
:1036200082FF9E460846704790F84120202A03D129
:1036300090F84020012A01D1022110E0242280F8D4
:1036400041200268136823F001031360136823F418
:10365000706343EA0121734605F065FF9E46084604
:10366000704790F84100704700B3B0B5044690F839
:10367000410018B906F0ADFB00F0E4F9242084F80D
:103680004100D4E90003D4E90212056823F0706315
:10369000012A25F0010505600361836823F40043D6
:1036A000836005D141F40041816009E00120704749
:1036B00041F40441022A816004BF4FF4006141607B
:1036C00041680F4A04F1100511434160C16821F4BB
:1036D0000041C1602ECD114341EA0321C160216A3E
:1036E00029430160016841F00101016000202021AF
:1036F000606484F84110206384F84200B0BD00BFCC
:10370000008000022DE9F84305F09BFF02D106F08E
:103710005EFA02D1022706F00DBB06F0FDF98146E4
:10372000009006F076FB0028F5D1222006F084F9FF
:103730008848618DB1F5807F02D306F054F901E02D
:1037400006F063F92046414602F07EF9089F002505
:10375000FF26608D10B3204639464A4602F0BCF978
:1037600008BB05F0E4FFF4D10028F2D02046802108
:1037700000223B46CDF8009002F07CF998B906F0A3
:10378000FEF905D306F019FB009502F05DF9E0E7BC
:1037900006F059FA009502F057F9DAE72046394663
:1037A00006F083FA08B10127B5E720682021A44B71
:1037B00006F082F8AFE700BF2DE9F84305F041FFBE
:1037C00002D106F004FA02D1022706F0B3BA06F0DD
:1037D000A3F98146009006F01CFB0028F5D12120BA
:1037E00006F02AF92148618DB1F5807F02D306F0F9
:1037F000FAF801E006F009F92046414602F024F902
:10380000089F0025FF26608D10B3204639464A46A2
:1038100002F0BFF908BB05F0ACFFF4D10028F2D0EC
:103820002046802100223B46CDF8009002F022F98C
:1038300098B906F0A4F905D306F0BFFA009502F096
:1038400003F9E0E706F0FFF9009502F0FDF8DAE78A
:103850002046394606F029FA08B10127B5E7206865
:103860002021774B06F028F8AFE700BF002000804A
:103870002DE9FE4F05F0E5FE0CD1DDF830B0BBF1CF
:10388000000F09D0DDF83480B8F1000F04D006F045
:103890009EF907D1022502E006F045FA01252846E7
:1038A000BDE8FE8F06F04EF98146009006F0B1FAB1
:1038B0000028F4D122200E9905F017FFCDE9001958
:1038C0002046514602F074F810B184F84050E5E704
:1038D000618D2048B1F5807F02D306F084F801E0C5
:1038E00006F093F82046514602F0AEF80027FF2676
:1038F0002046042100224346CDF8009002F0BAF899
:103900000028CBD105F013FF14D198B120468021B7
:1039100000224346CDF8009002F0ACF80028BDD15B
:1039200006F02DF902D306F080F901E006F066F901
:1039300002F08AF8608D0028DAD12046414606F070
:10394000B4F90028AAD1206820213D4B05F0D9FF09
:10395000A5E700BF002400802DE9FE4F05F071FEB1
:103960000CD1DDF830B0BBF1000F09D0DDF83480A8
:10397000B8F1000F04D006F02AF907D1022502E0C1
:1039800006F0D1F901252846BDE8FE8F06F0DAF8E9
:103990008146009006F03DFA0028F4D121200E99CE
:1039A00005F0A3FECDE900192046514602F024F8A7
:1039B00010B184F84050E5E706F0E1F805D3FF20A8
:1039C000514606F081F9204608E0608D00214FF055
:1039D000007320850091C2B22046514602F034F8AF
:1039E0000027FF26204641464A4602F0D2F800282A
:1039F000C8D105F0BEFE14D198B120468021002226
:103A00004346CDF8009002F035F80028BAD106F010
:103A1000B6F802D306F009F901E006F0EFF802F07B
:103A200013F8608D0028DDD12046414606F03DF9AF
:103A30000028A7D120682021014B05F062FFA2E7F2
:103A400000E800FEF0B593B004460EA81421FDF77F
:103A50008DFE68463821FDF789FE2068324988428C
:103A60002AD0324988425DD14FF44030402605903B
:103A70006846009600F028F908B1FEF795FB022091
:103A800002F0CEF8022002F0CBF804200025012736
:103A90001224129011951097CDE90E64244E0EA9B0
:103AA0003046FFF7B5FC80201195CDE90F471E2465
:103AB0001F254FF400171BE04FF440200690802094
:103AC0000090684600F000F908B1FEF76DFB012098
:103AD000012402F0A5F8002021254FF480074FF0C3
:103AE0009046CDE91040122020240F904FF4C05092
:103AF0000E90042012900EA93046FFF789FC38463C
:103B000002F0A8F828460121002200F049F82846D2
:103B100000F038F820460221002200F041F820464B
:103B200000F030F813B0F0BD0058004000540040E1
:103B30000004004880B5032000F04EF800F04CFA75
:103B40003A4908600F2000F007F808B1012080BD55
:103B500000F004F8002080BD00207047704700008E
:103B600000280CD400F01F010122400902FA01F1E3
:103B7000034A42F82010BFF34F8FBFF36F8F704797
:103B800080E100E0002808D400F01F010122400974
:103B900002FA01F1014A42F82010704700E100E00A
:103BA00070B5134B4FF0FF351B68C3F30223DC1EC7
:103BB00083F0070338BF002405FA04F6B243042B50
:103BC00028BF042305FA03F39943A1401143BDE83C
:103BD00070400CF07BBF00BF05494FF6FF030A6839
:103BE0001A4060F30A22034810430860704700BF80
:103BF0000CED00E00000FA0521483222016821F4B2
:103C000080410160F24909685143094AB1FBF2F170
:103C10004A1E43698A4203D213F400711146F7D158
:103C200040690321800501EAE070704758010020D7
:103C300040420F001248016841F480410160704722
:103C40000F49022301280A6863F302020A601D4932
:103C50000A6842F004020A600FBF30BF40BF20BFB5
:103C600020BF05F01BBC00BF0548006800F4C06021
:103C7000704700BF0248016841F4807101607047DD
:103C80000004005810B50C460D49096801F4007194
:103C900018B139B9FFF7CEFF04E019B1FFF7ACFF57
:103CA00000B110BD0748012C016821F0040101603A
:103CB00004BF30BF10BD40BF20BF20BF10BD00BF3C
:103CC0001404005810ED00E0F8B504468078544E16
:103CD000C00742D0FFF7CEFFFFF76CFC0546D6F8D1
:103CE000F403C00506D4FFF765FC401B0228F6D993
:103CF000032533E0606BD6F8841001F440718142F3
:103D000024D0D6F88410D6F8842042F48032C6F845
:103D10008420D6F8842022F48032C6F8842021F44E
:103D2000407289070146C6F884200FD5FFF742FC90
:103D3000054641F28837D6F88400800705D4FFF79E
:103D400039FC401BB842F6D9D2E7616BD6F8840043
:103D500020F440700843C6F8840000252068C1079D
:103D600002D0616805F091FE810702D5A16805F0D7
:103D70008CFE810605D52169F26F22F44062114361
:103D8000F167810502D5216A05F073FB410502D573
:103D9000616A05F06EFB010502D5A16A05F069FBB9
:103DA000410603D5606901F063FF2068010603D571
:103DB000A06901F05DFF2068C10503D5E06901F04D
:103DC00057FF2068C1060CD5E168F26F22F44072FB
:103DD0000A43B1F5807FF26703D1316841F0807109
:103DE000316001040AD5216BF26F22F040420A4390
:103DF000F26719B9316841F08071316040040CD527
:103E0000E06AF16F21F040510143B0F1005FF167CA
:103E100003D1306840F4803030602846F8BD00BFE0
:103E20000C0000582DE9F843002800F09F80674FF0
:103E300005460C46386800F00700884211D2386801
:103E400020F00700204305F01DFE0646386800F00C
:103E50000700A04205D0FFF7ADFB801B0228F5D973
:103E600056E02868B946704F810711D5A8683968AF
:103E700021F0F001084305F005FE06463868C0034E
:103E800005D4FFF797FB801B0228F7D940E028688C
:103E9000410616D56869D7F8001121F00F0141EAF3
:103EA0001010C7F80001FFF785FB0646D7F80001A0
:103EB000C00305D4FFF77EFB801B0228F6D927E05C
:103EC0002868410711D5E868396821F4E0610843A2
:103ED00005F0D8FD06463868800305D4FFF76AFB75
:103EE000801B0228F7D913E02868010714D5286938
:103EF000396821F4605141EAC00005F0C3FD06466F
:103F00003868400307D4FFF755FB801B0228F7D918
:103F10000320BDE8F8832868C0071CD1D9F8000049
:103F200000F00700A04224D9D9F8000020F00700D3
:103F30002043C9F80000FFF73DFB05464846D9F885
:103F4000000000F00700A04213D0FFF733FB05F09C
:103F50000CFDF3D930E068684FF0B04198B1032808
:103F60002CD002282ED1096889030FD40120BDE886
:103F7000F88300F031F81649086016480068BDE87B
:103F8000F843FFF7E9BD09688907EFD5396821F0E3
:103F90000301084305F076FD064641F2883868685B
:103FA000396801F00C01B1EB800FB7D0FFF702FBCD
:103FB000811B03204145F2D9BDE8F88309688901D6
:103FC000D4D5E3E709684905D0D5DFE700400058BC
:103FD000580100206C00002080B500F029F812493B
:103FE0003C22096802EA9101024A5158B0FBF1F003
:103FF00080BD00BF4839010880B5FFF7EDFF0A49D1
:104000000A4A0968C1F3022152F82110C84080BD54
:1040100080B5FFF7E1FF0449044A0968C1F3C221F2
:1040200052F82110C84080BD0800005888390108A6
:1040300010B5364951F8042C086812F00C0205D06E
:104040000C2A15D100F00300012811D14FF0B04027
:104050000368006800F008001B0705D4B8B9D1F860
:104060008800C0F303201CE0B0B9D1F8880011E04B
:104070002748042A1ED0082A1BD14FF0B0421268EC
:10408000D2025CBF44F60000C0F2E81012E04FF02C
:10409000B0400068002004E04FF0B0400068C0F37A
:1040A00003101C4B002A53F82030184618BF00207C
:1040B00001E00020002351F8042C02F00C020C2A2D
:1040C00022D1086800F003021148022A0CD0032A0A
:1040D00009D14FF0B0421268D2025CBF44F6000032
:1040E000C0F2E81000E018460A680B68096801246D
:1040F000C2F3062204EB51715043C3F302120132A2
:10410000B0FBF2F0B0FBF1F010BD00BF0C000058A6
:104110000024F400843A01082DE9F047002800F05B
:104120005981DE4C8246606800F00C08A06800F0FF
:1041300003099AF80000800627D49AF80000C00707
:1041400070D0B8F1080F63D0B8F10C0F08BFB9F107
:10415000030F5DD04FF0B041DAE901020B6823F4A0
:1041600080131A43B0F5803F0A6009D0B0F5041FF0
:1041700040F096814FF0B040026842F400120260B5
:10418000086840F48030086097E1B8F1000F1DD056
:10419000B8F10C0F08BFB9F1010F17D04FF0B046BE
:1041A0003068DAF82010002900F0348140F0010076
:1041B00005F005FA05463068800700F13A81FFF7FF
:1041C000F9F905F0D2FBF6D9BDE8F0874FF0B04120
:1041D0000868800704D5DAF82000002800F0FA808B
:1041E000DAF828000968090747BF4FF0B0410968AD
:1041F000D4F89010090901F0F001884240F2D4800F
:1042000006F02AFE002840F0E58005F01EF9E4E003
:104210004FF0B0400068800304D5DAF804000028AD
:1042200000F0D8809AF80000800730D5B8F1040F6C
:104230001BD0B8F10C0F08BFB9F1020F15D04FF029
:10424000B0463068DAF81010002900F0468140F4DA
:10425000807005F0B4F90546306840050FD4FFF7CB
:10426000A9F905F082FBF7D9AEE74FF0B04000683E
:10427000400504D5DAF81000002800F0AB80DAF829
:104280001400216821F0FE4141EA006020609AF8A4
:10429000000000072CD49AF8000040074FD4DAF849
:1042A0002C0010B3B8F10C0F40F0C680012800F0CC
:1042B0009180DAF83010A06800F003028A4240F0E2
:1042C0008980DAF8341000F070028A4240F082806F
:1042D000DAF8381000F4FE42B2EB012F7AD1DAF8A6
:1042E000441000F06040884274D10020BDE8F0879F
:1042F000D4F89010DAF8180000287AD0DAF81C0008
:1043000001F01002904200F08D8101F00302022AB8
:1043100060D0C90700F07F81D4F8900020F0010040
:1043200005F03EFC0546D4F89000800740F171810D
:10433000FFF740F9411B03201129F4D944E7D4F8D1
:10434000FC03C0050ED4FFF795FCFFF733F90546D3
:10435000D4F8FC03C00505D4FFF72CF905F005FBE4
:10436000F6D931E7DAF80C00002800F0C58085287E
:1043700001D0052805D1D4F88C0040F00400C4F821
:104380008C00FFF717F905F040FA40F00100C4F87F
:104390008C00D4F88C00800764D4FFF70BF9411B24
:1043A0000320B142F5D90FE74FF0B0410A6842F05F
:1043B00008020A600A6822F0F00202430A60DAF892
:1043C0002410226822F47F4242EA0121216006F093
:1043D00043FD10B10120BDE8F087FFF7FDFD9B49CB
:1043E00008609B480068FFF7B7FB00287FF4ECAE3D
:1043F000A3E621F0010005F0D3FB0546D4F89000B8
:1044000080077FF548AFFFF7D5F8411B032011293E
:10441000F4D9D9E620F0010005F0D1F8054630685E
:1044200080077FF58AAEFFF7C5F805F09EFAF6D94A
:10443000CAE605F00AF880E64FF0B0460228316877
:1044400021F08071316071D1FFF7B4F80546306812
:10445000800140F18180FFF7ADF8411B03200A295C
:10446000F5D9B1E6DAF80C0040F00400852840F0F8
:104470009980FFF79FF805F0C8F940F08000C4F874
:104480008C00D4F88C0000053FF509AFFFF792F8D7
:10449000411B0320B142F4D996E600BF0400005846
:1044A0004FF0B0460028316821F480313160316826
:1044B00021F40011316000F09E80FFF77BF8054683
:1044C0004FF0B046306880033FF5ACAEFFF772F8AE
:1044D000411B03206429F5D976E620F4807005F0AD
:1044E0006EF80546306840057FF5D1AEFFF762F8FB
:1044F00005F03BFAF6D967E6FFF75CF80646D4F814
:104500008C0041F2883920F08000C4F88C00D4F887
:104510008C0027460405FFF74DF80546002C55D5BD
:10452000A91B03203C464945F1D94DE6A0684949FD
:1045300020F00300A060A0680840A060FFF73AF8F0
:104540000446306880017FF5D0AEFFF733F8011BD9
:1045500003200A29F5D937E6A0683F490AF1300758
:104560000840EECF0843104340EA032028434FF0B1
:10457000B04530433843A060286840F08070286020
:10458000A06840F08050A060FFF714F80446286847
:1045900080013FF5AAAEFFF70DF8011B03200A29A1
:1045A000F5D911E6FFF706F805F02FF920F08000A5
:1045B000C4F88C00D4F88C0000057FF570AEFEF7CF
:1045C000F9FF411B0320B142F4D9FDE5D7F88C0077
:1045D0003C4641F2883620F00100C7F88C00D4F840
:1045E0008C0080077FF55BAEFEF7E4FF411B0320E4
:1045F000B142F4D9E8E5FEF7DDFF054630688003F7
:104600007FF510AEFEF7D6FF411B03206429F5D9D4
:10461000DAE5DAF81C00D4F8901021F01001084314
:10462000C4F89000D4F8900040F0010005F0B8FA0A
:104630000546D4F8900080073FF52DAEFEF7BAFF8F
:10464000401B1128F5D90320BDE8F0875801002050
:104650006C000020FFFFFEEE8C80C111704700004F
:10466000034850F821007047014840F82120704766
:1046700000B1004090F82C200221012A0DD080F8D2
:104680002D10C049734605F00DF89E4642F02002F9
:104690000A60734604F01EFF9E460846704700BF3E
:1046A00080B50AF023FE0130BDE880400AF02ABE42
:1046B00010B5044621480168490604D540218160AF
:1046C0002046FFF7EDFF012084F82D0010BD00BF4C
:1046D00090F82C200221012A12D080F82D10A9492F
:1046E000734604F0DFFF9E4642F080020A60A74A4C
:1046F000136843F480231360734604F0EBFE9E4678
:10470000084670470CF000B970B50C4D0446286897
:10471000216B01EA0006F00704D00120A8602046C2
:10472000FFF7F0FFB00704D50220A8602046FFF78E
:1047300095FF012084F82D0070BD00BF5428004073
:10474000B0B590F82C300222012B2ED08D4BCA240C
:1047500080F82D20DC605324DC606FF40854B1F540
:10476000807F08BF6FF488541D682C401C6034247F
:10477000B1F5807F08BF2C24E55825F00045E550B1
:1047800008BF01225A64FF22DA600022012380F868
:104790002C2080F82D306FF00203B1F5807F08BF28
:1047A0006FF00103016B194001631046B0BD00BFFB
:1047B00070B590B3044690F82D0028B9002084F815
:1047C0002C00204600F03EF802207C4D84F82D009D
:1047D000CA20A8615320A861204606F0BFFBC8B9D3
:1047E000E8681749261D0840E8604ECEA0693143AD
:1047F0000843E9680843E86043EA02406860D4E996
:1048000009012A6822F4F85210430843286004F092
:1048100046FF20B1FF21A96170BD012070BD606914
:10482000D4E90712EB6823F060431A4311430843AD
:10483000E860FF20A861012084F82D00002070BDF1
:10484000BFFF8FFB10B590B0044601A83821FCF7DC
:104850008DFF20681749884229D14FF480700E904F
:104860004FF48030019001A8FFF72EFA08B1FDF750
:104870009BFC11480022816B41F400418163016877
:1048800041F4806101600021006800F480600F90B5
:104890000F980220FFF784F90220FFF773F92A200E
:1048A00000210022FFF77CF92A20FFF76BF910B0F6
:1048B00010BD00BF00280040580000582DE9F84FF7
:1048C00004F080FE5CD084F82D0001202D4F05F00F
:1048D0006BF901D1002029E072B16869B0F1803F25
:1048E00007D0B0F5000F04D03968490601D4002183
:1048F000E97004F0DDFD19E03868400602D40026B6
:10490000EE7001E0E87886052878DFF87CB0D5F80D
:1049100014A0D84780466878D84705F069FA05F0B2
:10492000A6F9296A41EA080141EA006005F0B4F8F5
:104930000ED105F01AFA19BFB862A869D5E90601C7
:104940000843F86268680121B8654FF488500DE0AB
:1049500005F0C5F919BF3863A869D5E90601084310
:10496000786368680221F8654FF408503A6810438C
:1049700038600648026842F40032026004F050FFDA
:10498000BDE8F88F1828004039AF000880080058AB
:10499000B0B50A4D286820F020002860FEF70AFE16
:1049A00004462868800607D4FEF704FE001BB0F515
:1049B0007A7FF6D90320B0BD0020B0BD0C2800409E
:1049C000014804F028BF00BF10E000E0012904D036
:1049D00041B9CF48816880200847CD4881684FF4AD
:1049E00080700847704700BFC94881684020084769
:1049F0002DE9F04105F07BF902D16079012802D15F
:104A00000220BDE8F08104F06EFDED4905F0B5F936
:104A1000394609F009F920460021002709F004F978
:104A2000AF4204D205F02AF901370136F8E705F064
:104A30003CF8724604F000FF964618BF0120BDE81E
:104A4000F08100BF2DE9F04105F051F902D1607904
:104A5000012802D10220BDE8F081012520461E4632
:104A600017468846657109F00DF948F01000414677
:104A7000942818BF00252571D14D286820F40040E6
:104A80002860204609F0D0F836B117F8011B2046FF
:104A900009F0CAF8013EF7E72868B8F1840F40F43E
:104AA0000040286002D0204609F010F9724604F058
:104AB000C3FE964618BF0120BDE8F0819448816886
:104AC0002020084792488168102008477CB504469A
:104AD00000200DF1060212210223ADF80600204647
:104AE000FFF786FF9DF807609DF80650F00702D09B
:104AF000204600F009F9B00702D5204600F0F6F88C
:104B0000700702D5204600F091F8300702D5204604
:104B100000F0F6F8F00602D52046FFF7D3FFB00606
:104B200002D52046FFF7CAFF700602D52046FFF7E0
:104B30005BFF300604D505F001012046FFF746FF74
:104B4000A80702D5204600F0D5F80DF10602204650
:104B500002210223FFF776FF7CBD0000BCB510B335
:104B60000446807920B900206071204600F046F8A4
:104B700002201E4A6423A0711D48815821F400417F
:104B800081501C490968C1EBC101C1F34C41594333
:104B90000191019949B1019B013B019383585B0449
:104BA000F7D4002503E001251DE00125A560D0F81C
:104BB000882042F40042C0F888200F4A136843F46A
:104BC00080531360026842F4006202604FF4006296
:104BD000026131B1206808F0E7FF0020A0600120E9
:104BE00020710120A0712846BCBD00BF8CFCFFFFD6
:104BF000080400585801002090080058E0B50A4801
:104C00000022016841F0010101600021006800F00C
:104C10000100019001983220FEF7C2FF3220BDE86A
:104C20008C40FEF7AFBF00BF640000583848816871
:104C3000042008472DE9F84305F059F802D16079BE
:104C4000012802D10220BDE8F88304F04CFC5C4945
:104C5000DFF8708104F092FE1E21C04720463946DD
:104C6000C047204600210027C047AF4204D205F0CC
:104C700005F801370136F8E704F0ABFC724604F0A2
:104C8000DBFD964618BF0120BDE8F8832DE9F84307
:104C900005F02DF802D16079012802D10220BDE88B
:104CA000F88304F020FC4649DFF8188104F066FE22
:104CB0001D21C047390A2046C047F9B22046C047E7
:104CC000204600210027C047AF4204D204F0D6FF9F
:104CD00001370136F8E704F07CFC724604F0ACFDC5
:104CE000964618BF0120BDE8F88300BF08488168D8
:104CF00002200847064881684FF40070084700BF4B
:104D00000348816808200847014881680120084756
:104D1000A00200202DE9F04104F0E9FF02D1607902
:104D2000012802D10220BDE8F08104F0DCFB244917
:104D300005F023F80E2108F077FF2046394608F0E9
:104D400073FF1DB105F05AF8013DFAE704F0ADFE1E
:104D5000724604F071FD964618BF0120BDE8F0814F
:104D60002DE9F84304F0C3FF1ED10F4661790220FC
:104D7000012922D0A07101201D46164660712046EF
:104D800008F080FF0E49DFF83C8004F0F7FD0D21AC
:104D9000C047390A2046C047F9B22046C04735B15E
:104DA00005F02CF8013DFAE70220BDE8F88304F095
:104DB00010FC04F041FD18BF0120BDE8F88300BFDE
:104DC0009004005829DC0008014804F06CBB00BFC7
:104DD00010E000E0704770477047000070B590F831
:104DE0003C300222012B23D080F83D200122334C9D
:104DF00080F83C20026855689368A24203D14E684F
:104E000025F4700535430E6825F070053543A24240
:104E1000556002D0B2F1804F04D1896823F080033D
:104E2000194391600022012180F83C2080F83D1058
:104E3000104670BD58B110B504F0ECFE03D104F07B
:104E40006FFD00F006F804F09FFF04F0CBBB0120DB
:104E5000704780B50068B0F1804F18BF80BD012059
:104E600000F0F8FE1B2003210022FEF799FE1B2014
:104E7000BDE88040FEF786BE90F83D10012918D1AC
:104E8000022180F83D100168C86840F00100C86048
:104E90000A48814202D0B1F1804F0CD18868084A9B
:104EA000734604F068FE9E4602D0B2F5803F02D100
:104EB00070470120704704F0C0BE00BF002C0140C5
:104EC00007000100016841F21113CA6822F00102D3
:104ED000CA600A6A1A4208D10A6A40F244431A4276
:104EE00003D10A6822F001020A6004F0E8BE000063
:104EF00010B504F03AFE4ED084F83D000120274B57
:104F000084F83C00206882681A4082600A68C2B156
:104F1000102A16D0202A14D0302A12D0402A17D0B6
:104F2000502A1DD0602A23D0B2F5005F2BD0B2F5F5
:104F3000805F2DD0702A2FD104F0CEFC41F0770194
:104F400025E08168164B1940114341F007011EE02E
:104F500004F0F3FE2068124A81681140473116E0E0
:104F600004F0EBFE20680E4A8168114057310EE0D4
:104F70004B68CA6819460AF0BEFA2068084A816878
:104F80001140673103E004F0A7FC41F480418160E7
:104F9000002004F08DFE10BD0120FAE78800CEFF4E
:104FA00088FFCFFF704710B5044600680169890784
:104FB00014D5C168890711D56FF002010161012183
:104FC00021778069800702D004F069FE03E004F0D5
:104FD000AEFE04F067FE00202077206801694907D3
:104FE00015D5C168490712D56FF00401016102218E
:104FF0002177806910F4407F02D004F050FE03E076
:1050000004F095FE04F04EFE002020772068016930
:10501000090714D5C168090711D56FF008010161AE
:1050200004212177C069800702D004F038FE03E034
:1050300004F07DFE04F036FE002020772068016930
:10504000C90615D5C168C90612D56FF010010161F6
:1050500008212177C06910F4407F02D004F01FFEC0
:1050600003E004F064FE04F01DFE002020772068B9
:105070000169C90709D0C168C90706D06FF00101ED
:105080000161204600F03AF820680169090609D557
:10509000C168090606D56FF0800101612046FFF75F
:1050A0009AFE20680169C90509D5C168090606D5B7
:1050B0006FF4807101612046FFF78CFE2068016962
:1050C000490609D5C168490606D56FF0400101615E
:1050D000204600F019F820680169890602D5C168E8
:1050E000890600D410BD6FF0200101612046BDE8A3
:1050F0001040FFF771BE7047704700000148012162
:1051000001807047981B0020704710B504F041FCE7
:1051100001D1022010BD2420C4F884002068016859
:10512000026822F0010241F000510260012284F87D
:1051300080204FF000526266016020460AF07CFB3E
:105140000020202184F88000C4F8841010BD90F85D
:105150008010012901D102210FE0012180F8801087
:10516000016851E8001F026841F0020142E80013A3
:10517000002BF5D1002180F8801008467047704759
:105180007047B0B504F005FC01D10220B0BD04F0B9
:10519000BCF922F0606204F09BFC04F049BAB0B59F
:1051A00004F0F7FB01D10220B0BD04F0AEF922F00B
:1051B000604204F08DFC04F03BBABCB504F0E9FB9E
:1051C00001D10220BCBD2420C4F8840020680368FB
:1051D00023F001030360012384F88030836823F403
:1051E00040130B43836059B9436891B223F0100315
:1051F00019434160C2F30741426861F31F62426094
:10520000016841F001010160FEF7D4F903466FF037
:105210007E404FF4800100220025009020460AF0D5
:1052200047FF08B1032003E02020C4F884000020D9
:1052300084F88050BCBD70477047704770B5044615
:10524000006840F60F05C269016883682A426BD086
:10525000A54D01EA0506A54D1D4076196ED0D6076D
:1052600009D0CE0507D501260662D4F88C6046F039
:105270000106C4F88C60960709D5DE0707D0022620
:105280000662D4F88C6046F00406C4F88C605607B9
:1052900009D5DE0707D004260662D4F88C6046F0F4
:1052A0000206C4F88C6016070BD501F020063543C2
:1052B00007D008250562D4F88C5045F00805C4F8DD
:1052C0008C5015050AD54D0108D54FF400650562CF
:1052D000D4F88C5045F02005C4F88C50D4F88C508C
:1052E000002D6ED092060AD501F0200103F0805205
:1052F000891804D0216F11B1204688472068D4F85E
:105300008C10806801F0280100F04000401852D055
:1053100020460AF08BFB2068816849065DD504F0C1
:1053200092FA4FD02068FAE7950607D501F02005DC
:1053300003F08056AD1901D0216F13E0E56E012D09
:1053400003D1D50601D5CD064CD4D50201D55D02D9
:1053500029D415060BD501F0800503F400035B1971
:1053600005D0616F69B32046BDE870400847530619
:1053700001D54B060DD4100201D5480057D4D001F9
:105380001FD5B1F1FF3F1CDC2046BDE87040FFF7A0
:10539000F7BE50E8000F216820F0400004F013FC35
:1053A0003BD02068F5E74FF4801101622046BDE84C
:1053B0007040FFF741BF2046FFF73FFF0020C4F8D1
:1053C0008C0070BDE06F40B149498163FDF756FD27
:1053D0000028F6D0E06F816BC6E72046BDE870403C
:1053E000FFF72BBF102101628168490624D4B4F86D
:1053F0005E10B4F85C20B4F85E30002BE1D0511A96
:105400000A04DED050E8000F226820F4907042E8D1
:105410000003002B48D02068F4E7002060672020BC
:10542000C4F884002046BDE8704000F095B92046DD
:10543000BDE87040FFF7FFBEE16F0A6853689DB298
:10544000002DBED0B4F85C108D42BAD2A4F85E3004
:105450001268920623D450E8000F216820F480706F
:1054600004F0B1FB01D02068F5E7206850E8020F96
:10547000216820F0010004F088FAF6D1206804F0D9
:10548000E2F9FBD12020C4F888000020E06604F097
:1054900032F8FCD1E06FFDF7B9FCB4F85C10B4F859
:1054A0005E00081A81B21AE01248226852E8022F00
:1054B0002368024043E80225002DF6D12020C4F8DD
:1054C000880000202067E066206850E8000F22680E
:1054D00020F0100042E80003002BF5D189B22046ED
:1054E000BDE87040FFF74BBE200100040100001032
:1054F00089F90008FEFFFFEF10B548B10446D0F867
:10550000840008B904F07FFC04F087F8012801D179
:10551000012010BDA06A08B104F08BFA04F06EFA05
:1055200021F02A01816004F0D3F8BDE810400AF0B0
:10553000F9B9000010B5044600688C49884218BFCC
:1055400010BD0948016821F4003101604FF090401E
:105550000C21FDF7C9FEA06FFDF7C6FC2520BDE8B4
:105560001040FEF7FDBA00BF58000058F0B595B0E6
:1055700004460FA81421FCF7F9F801A83821FCF71C
:10558000F5F820687949884252D12A4802250195C8
:10559000039001A8FEF798FB08B1FCF705FE26482A
:1055A00003270026C16841F40031C160C16801F4DD
:1055B000003114911499016841F001010160006803
:1055C00000F0010014900720129713900420CDE9F9
:1055D00010560F9014980FAD4FF090402946FDF7EC
:1055E00017FF0820CDE9107629460F904FF0904024
:1055F000FDF70EFF114D124B142280201021C5E93A
:105600000032C5E90216C5E904062846C5E9066662
:105610002E62FDF70FFD08B1FCF7C6FD2520022123
:105620000022AC62A567FEF7BBFA2520FEF7AAFAB6
:1056300015B0F0BD04000C004C000058184C0020C0
:1056400058000240B0B5D0F88830202B05D131B1D8
:105650002AB190F88030012B03D10220B0BD012087
:10566000B0BD0023074C04F063F902D05C6824024B
:1056700003D40AF09DFC0020B0BD04F089F8F8D0F6
:105680000368FAE70080004010B504460068374917
:10569000884218BF10BD0848436833B1D4F88C0065
:1056A00018B90548012100229847034920460122E4
:1056B000BDE81040FFF7C6BFC4010020F8B504469E
:1056C000D0F88400202806D161B3134652B394F871
:1056D0008000012801D10220F8BD00250120A4F896
:1056E0005630C4F88C5084F880002120A4F854303F
:1056F0002165C4F88400A06FB0B1144A144E154F50
:10570000C0E90B76C0E90D2522682832FDF7F2FCCE
:1057100050B11020C4F88C00002084F880002020B4
:10572000C4F884000120F8BD2068402184F880502E
:10573000016250E8020F216840F0800004F025F972
:1057400001D02068F5E70020F8BD00BF99F90008F6
:1057500027FA0008EFF9000800680449884218BFDA
:105760007047034801680020084700BF004400401C
:10577000A01B002070470000F8B52B4F05460C46D3
:1057800097F80401022802D02848C06A804701F037
:10579000A5F8064628B1022001F0B5F8002001F076
:1057A00096F897F80401012813D101F09DF830B163
:1057B000002001F0ACF8002001F0A0F8012601F073
:1057C00091F830B1002001F0A0F8002001F092F82B
:1057D00020E0FEB9164E96F8941496F81E0431B1E6
:1057E00008B186F84544204601F044FA10E008B1BB
:1057F00086F84554284601F03DFAF86A0BF074F833
:10580000D6F8B413884205D306F566700BF010F98C
:1058100004F07BFA97F804010549022818BF062016
:1058200081F89404F8BD00BF7C850020C43A0108CB
:105830007C140020FEE700688169890701D50021FA
:1058400081628169C90703D1816941F001018161E8
:10585000704700002DE9F047044600688A4600279B
:105860008169C90601D4002146E0102190460AF161
:1058700001064FF020090025C161816901F0200176
:10588000294334D10025002EF7D0FDF793FEA0EB7D
:1058900008012068514503D80025BAF1000FECD16A
:1058A000436894F8421082695B0409D412F4004200
:1058B00006D0202904D004F04CFAFDF77BFE804688
:1058C0000025206881698906D7D4FDF773FEA0EB17
:1058D00008001A28F5D3606C012540F020006064B0
:1058E00084F8419084F8407084F84270E9E70DB97B
:1058F0002021C161012104278269D30505D54FF418
:10590000807147F00107C1610121530505D492055B
:1059100009D469B90020BDE8F0874FF480610837E9
:10592000C161910504D54FF4007147F00207C161D0
:1059300004F094F82068884A416811404160606C26
:105940003843714603F03CFF8E460120BDE8F087E6
:1059500010B586B00446642006210DF11202012321
:10596000CDE9002102900E48A6213222FDF780FFEA
:10597000BDF812000DF066FD0A4941F82400BDF89B
:1059800014000DF05FFD084941F82400BDF8160031
:105990000DF058FD054941F8240006B010BD00BFC8
:1059A000784C0020A41B0020A4230020A42B00205E
:1059B0002DE9FC410446234815461E46DAB2002371
:1059C000009003F0D0FEDDE9088704F0FDF910B186
:1059D0000120BDE8FC81012E03D004F0A5F80028C9
:1059E000F6D104F0AFF94021009700F043F8002809
:1059F00018BF0120BDE8FC812DE9FC410446114897
:105A000015461E46DAB24FF08073009003F0ABFEED
:105A1000DDE9088704F0D8F910B10120BDE8FC8168
:105A2000012E03D004F080F80028F6D104F08AF9A2
:105A30008021009700F01EF8002818BF0120BDE863
:105A4000FC8100BF0020008070B500686FF39F21CB
:105A5000049D074E1943446841EA0241294324EA60
:105A6000555421F0004134402143416070BD00BFD6
:105A7000009C00FC2DE9F843DDF820801D46164609
:105A80000F4681465C1CD9F8000080693840C01B75
:105A9000B0FA80F04009B0421AD1002CF3D0FDF7E3
:105AA00089FDA0EB0800A84201D8002DEBD1D9F860
:105AB000440040F02000C9F84400202089F841004B
:105AC000002089F8400089F842000120BDE8F883F1
:105AD0000020BDE8F883000070B515460E46044668
:105AE0002068806940071DD404F034F890BB20681A
:105AF0008169890611D4FDF75DFD401BB04201D8D4
:105B0000002EEDD1606C40F020006064002084F82D
:105B10004000202084F841001CE08169490703D53A
:105B2000218D09B1002070BD81690022C9064FF0A6
:105B3000000102D51022C261042262642022064DB7
:105B4000C26143682B40436084F8412084F84010D0
:105B500084F84210012070BD00E800FE70B51546C3
:105B60000E46044620688069800610D403F0F2FFD8
:105B700058B9FDF71FFD401BB04201D8002EF1D1EE
:105B8000606C40F0200003F01BFE012070BD00207F
:105B900070BDF8B515460E4604464F1C2068806956
:105BA000800712D403F0D6FF68B9002FF6D0FDF7B6
:105BB00001FD401BB04201D8002EEFD1606C40F0D7
:105BC000200003F0FDFD0120F8BD0020F8BD00001D
:105BD00081B005490A6802430A60096808400090DC
:105BE000009801B0704700BF4800005881B01849C4
:105BF0000A6802430A60096808400090009801B0F2
:105C0000704700BF81B01248016841F00201016095
:105C1000006800F002000090009801B0704700BFDB
:105C200081B00B490A6802430A6009680840009085
:105C3000009801B0704700BF81B005490A6802436F
:105C40000A60096808400090009801B0704700BFE2
:105C50004C00005881B005490A6802430A6009688F
:105C600008400090009801B0704700BF58000058ED
:105C7000064A6FF47F2161EA101100F47F40136837
:105C8000194041EA00101060704700BF88000058BA
:105C90002DE9F04190B0734D0146142205F140000A
:105CA0000AF05AFD0020287003F02EF995F84020E4
:105CB0004068D040C00708D005F10C0005F12C0168
:105CC00001F0FCFA40B1FF26C8E0734B0020002130
:105CD00001220AF073FCFEE727208DF81C0007A8BC
:105CE00001F02AFFF0B128208DF81C0068680069D7
:105CF00040B107A801F03AFE686840F27C510269A1
:105D00000898904727208DF81C0007A801F014FF81
:105D100058B901208DF81C0007A801F027FE9DF856
:105D2000200010B10120687001E0687800B3686855
:105D3000C16909B10020884706208DF81C0007AC16
:105D400003F0D0FE48480899016327208DF81C0015
:105D500003F0C8FE089890F8401090F8042190F8DD
:105D6000060185F8401085F8412085F8420014E0CE
:105D70000020089005208DF81C0007AC204601F09B
:105D8000DBFE6868C06880473749089008630620D2
:105D90008DF81C00204601F0CFFE02208DF81C007B
:105DA00007AC03F09FFE304E0899082206F11C0054
:105DB0000CF0ABFA03208DF81C0003F093FE089959
:105DC00006F1240008220CF0A0FA08F0BDFE96F8B7
:105DD000300096F8311096F8322096F833300026CD
:105DE000CDE90032CDE9021020A3022000210022DB
:105DF0000AF0E4FB0120974F4FF00F088DF82000C8
:105E000020468DF81C80B84710208DF820608DF852
:105E10001C002046B84704208DF81C0095F842006D
:105E20008DF820002046B84738208DF81C00286DDA
:105E300008902046B84795F840008DF8148005A9D1
:105E400007F07AFA002818BF012085F846001420D0
:105E500000F084FA95F8460002F09AFF70B210B094
:105E6000BDE8F0811C0300207000002023232323C1
:105E7000232320446576416464723A202020202048
:105E8000253032583A253032583A253032583A25A2
:105E90003032580D0A0000004B950108FEB509206C
:105EA0008DF8040001A802F073F8D349059A002880
:105EB0008A6018BF4FF0FF3006B080BD10B58AB0C1
:105EC00038B1044600208DF8040001A801F04EFD11
:105ED00008B1FF2003E09DF808002070002040B2C8
:105EE0000AB010BDE8488068704700BF10B58AB09E
:105EF00038B1044620208DF8040001A801F036FDD9
:105F000008B1FF2006E09DF80800DF49207081F805
:105F10004400002040B20AB010BD00BF21B10128EA
:105F200004D028B94C4802E0FF2002E00248086093
:105F3000002040B2704700BF0100010280B501F0AF
:105F40001BF9002818BF6FF0010080BD2DE9F84350
:105F50000A46CD49D0F818C0DFF844E0DFF84480A5
:105F6000DFF84490486090E83800D0E90F7641F8B7
:105F70001C2F0E4A41E9042941E9028E0C4A406C6B
:105F8000C1E9017601F10C0639C60020C1E9072CF0
:105F900000F0C0F8002818BF4FF0FF30BDE8F883CC
:105FA00085930008F9920008799200084192000850
:105FB000E1930008F0B58FB0E74E01220C460228AD
:105FC0008DF8282096F844108DF82D1008D1E1485E
:105FD00002218DF82C10C471817102F0BFFE2DE0FA
:105FE000DC484FF480738DF82C20C471A0F8053084
:105FF00001717078C0B91F208DF80810154F8DF809
:10600000040001AD2846B84720208DF8040096F81A
:1060100044008DF808002846B8470F480290292010
:106020008DF804002846B84702F098FE01208DF84C
:1060300008008DF8040001A801F07EFD70780128A9
:1060400008BF002C02D00AA801F0A2FF0E98B06091
:106050000FB0F0BD397B00080004000180B58AB0A4
:1060600001208DF8040001A801F080FC9DF80810C3
:10607000B0FA80F0002918BF0121400908400AB099
:1060800080BD0000B0B58AB0FFF758FF044650BB92
:1060900003F0ACF9811C15D090B9AF4C6068406931
:1060A00070B127208DF8040001A801F05FFC606842
:1060B0004FF4B0614269029890470025002403E044
:1060C000FF2400E0F824012503F09EF9002818BF02
:1060D0004FF0FF343DB930B99F484068C16909B1FC
:1060E00001208847002460B20AB0B0BDB0B59A4D17
:1060F0000024052C08D005EB8400406D10B1C06869
:10610000804708B90134F4E70020052C38BF01208E
:10611000B0BD00BFB0B508B1FF201AE00C4605467F
:1061200000F01CFB0028F7D08B4901EB8502496881
:106130005065094A8B6B8262084AC2628A69896C1F
:10614000C0E90C3106494261F22243682046984773
:10615000002040B2B0BD00BFB55F00089D5E0008E2
:1061600042090020F8B57C4F0C4605460026052E56
:1061700008BFF8BD07EB8600406D78B1032D0DD840
:10618000DFE805F002040608816904E0C16902E065
:10619000016A00E0416A09B1204688470136E6E716
:1061A0007CB502F097F86C4C0025052D10D004EB5F
:1061B0008506706D50B1042D08D8016931B1806831
:1061C00020B1804710B1706D006980470135ECE760
:1061D000FFF78CFF60B92078012809D194F84310AB
:1061E000002568460022CDE9005500F04FF800B1C7
:1061F0007CBD25707CBD00BF1C03002010B58AB09B
:10620000044601F0EFF908B1FE240DE0FFF726FF88
:10621000012808D100208DF8040001A801F0A6FB98
:1062200028B1FF2400E0FD2460B20AB010BD9DF843
:106230000800A04226D0022C14D0012CF1D00CBBB7
:1062400000240028F0D08DF8084001A801F074FC6B
:106250000028E6D140484068016B99B10020002435
:106260008847E1E70028DCD102208DF8080001A86A
:1062700001F062FC0028D4D137484068016B09B1B5
:10628000022088470024CFE71C0300202DE9F041BD
:1062900086B014460E46054601F0A4F908B1FE2169
:1062A00053E0FFF7DBFE012818D12A4F002E694684
:1062B00087F83C6018BF01268DF80460264E96F8DA
:1062C00044008DF81200687802F04EFC60B10020A6
:1062D0004FF0F90803908DF804000DE01D4988790E
:1062E000C979FFF767FE25E0297868784FF0000844
:1062F0008DF8081069680391D5E90012ADF8100017
:10630000C7E9111296F8441087F83E1001A82146FB
:1063100001F07AF905991128B16011D8FE21DFE862
:1063200000F00B140F0F0F0F0F090F0F0F110F0FAE
:1063300014141413FD2108E000204146307004E0DD
:10634000FF2102E0FA2100E0FB2148B206B0BDE8DF
:10635000F08100BF700000201C03002080B58AB0CF
:10636000029023208DF8040001A801F0E5FB00282D
:1063700018BF4FF0FF300AB080BD80B500F0E2FEDC
:10638000002818BF6FF0010080BD0000BCB588B1C7
:1063900081B1E44B18600120996283F825204FF009
:1063A000FF310022187700200090181D0B4B0AF0D7
:1063B00077FA03E0DB48002101770160D94C002522
:1063C0000021202204F13000A5850BF0B2FFA4F8D3
:1063D000505084F82E506577BCBD00BF819E0008E8
:1063E000D048007F704700BFCE48407F704700BF55
:1063F0002DE9F0478AB0CB4C217F002900F08E8137
:10640000C17809B9827B12B1A28D0132A285E0293F
:1064100040F08481417B002900F08081002184F8D4
:10642000261081680A78222A3AD8DFE812F0230081
:106430006201BF00C500CC00D900E000EC00F8000C
:1064400014012D0172017201720172017201720157
:1064500072017201720172017201720172017201A4
:1064600072017201720172017201720172013001D6
:1064700034013801A16A01200022062384F8260095
:106480000A7094F826104A1C84F82620A26A5354F5
:1064900094F826104A1C84F82620A26A50542BE156
:1064A0007D2A00F004817E2A00F01A817F2A40F0C4
:1064B00030812A208DF8040001A801F057FA94F8E1
:1064C0002610A26A7F239DF80CC09DF80DE09DF870
:1064D0000E809DF80F909DF808A09DF809609DF82A
:1064E0000A70481C84F826009DF80B00535494F859
:1064F000263021685D1CCA7884F82650A56AEA54C3
:1065000094F826308A785D1C84F82650A56AEA54EF
:1065100094F826304A785D1C84F82650A56AEA541F
:1065200094F826200978531C84F82630A36A9954DD
:1065300094F826104A1C84F82620A26A505494F835
:106540002600411C84F82610A16A0F5494F82600F6
:10655000411C84F82610A16A0E5494F82600411CB0
:1065600084F82610A16A01F800A094F82600411CC6
:1065700084F82610A16A01F8009094F82600411CC6
:1065800084F82610A16A01F8008094F82600411CC6
:1065900084F82610A16A01F800E094F82600411C56
:1065A00084F82610A16A01F800C0A5E05E48012128
:1065B000826A022090479FE04878012184F85110B8
:1065C00084F8520098E004208DF8040048780028F0
:1065D00018BF01208DF8080001A801F0ADFA8BE08A
:1065E0004878002818BF012002F0D2FB84E04878E8
:1065F0000A2800F281802168496800297CD04BA2DA
:1066000052F8200051E04878411E012974D8013821
:1066100018BF0120216884F82400896844E0A26A38
:106620000121082384F8261013700122037B94F8BB
:106630002550AB4238BF1D46AA425DD2836894F80C
:10664000265001325B5C6E1C013184F82660A66A1C
:1066500001337355EAE70120092184F82600A06A76
:10666000017094F8260094F82C20411C84F8261020
:10667000A16A0A5494F8260094F82D20411C84F84D
:106680002610A16A0A5437E00020A08534E00420D7
:106690008DF8040020E02448C06A80472CE0487848
:1066A000216884F83100C96831B3884724E0007B51
:1066B000072821D1B1F80100ADF808004879B1F8F8
:1066C000032042EA004064225043039005208DF8E5
:1066D000040088798DF8100001A801F059FC0BE046
:1066E00000208DF8080039208DF8040001A801F081
:1066F00023FA012084F8500094F8260048B10434AD
:106700004FF47A7120460AF045F920460AF05AF90A
:1067100004E0201D0AF08CF9002060770AB0BDE883
:10672000F08700BF2C020020C800002000000000FD
:106730008813000010270000204E00003075000074
:10674000409C000050C3000060EA0000C0D401007B
:1067500080A9030000530700704770472548704721
:106760007CB5234E707F38B30AF0B4F8356A04461E
:10677000FFF7B8FB284484422ED996F8260058B378
:106780008DF80100E02096F8241001228DF8000019
:10679000B06A01906846FFF779FD40F00400C0B28E
:1067A000FE2814D1351D4FF47A7128460AF0F2F80C
:1067B00028460AF007F90EE096F8510060B1002073
:1067C00086F8510096F85200FFF718FD04E000200B
:1067D00086F826007077346296F8500030B10020B9
:1067E00086F850000348406B00B180477CBD00BF75
:1067F0002C020020C80000202DE9F04F89B08A4605
:106800000546447B90F80EB090F90C8040681299D0
:1068100000270860687800284CD0CDE901230220C9
:10682000E97B8DF81C00287C8DF81E1007A906F066
:1068300083FD29896A684FFA80F94E468A4228BF4B
:106840000127C145B8BF4646688943189A420AD312
:106850000A208DF81C00287C07A906F06DFD04466F
:10686000688929896A6801EB40039A421FD3511A4B
:10687000B1FBF0F202FB1010C8B9C1450ADB287861
:1068800030B102208DF81800287C03A906F05EFDC7
:106890004FF0010B2120E97B8DF81D608DF81C0065
:1068A000287C8DF81E1007A906F046FD0646DDE996
:1068B000012301E05FFA88F68AF80060147083F81B
:1068C00000B0384609B0BDE8F08F0020704770472F
:1068D000704770477047704700207047002070472E
:1068E000002070470020704700207047002070474C
:1068F000022070477047002070477047704770470C
:106900007047002070477047704770477047704766
:1069100070470220704700002DE9F843002940D05D
:10692000824F91468046002207F1080007EB0215CE
:10693000002605F10803102E0CD0845D0136002CD2
:10694000F9D0741E0F2C05D810300132202AEDD159
:10695000022627E0386800B93B60786800B1036020
:10696000002605F10D001FFA89F27B60C5F8109032
:1069700085F80C801E600BF0C8FCA8F1050041F200
:1069800039020021C0B20D2822FA00F038BF0121DF
:1069900008402875D7F8080248440130C7F80802B3
:1069A00000E001263046BDE8F88300BF811E0020CC
:1069B000112913D8DFE801F013090B090D0F0B0B98
:1069C0000912120F12120D09111105207047022031
:1069D000704701207047062070470420704703204D
:1069E0007047000028B15149D1F808120160002019
:1069F00070470120704700BFB0B54C4C00214FF4E8
:106A00000372002520460BF094FC0020C4E90055D9
:106A1000B0BD00BF50B180B544490B68834207D078
:106A200043B11A461B688342FAD104E00120704743
:106A300002680A6000224B68834208BF4A600AB1BC
:106A400003681360836800220260D1F80822DB43E8
:106A50001A44C1F80822002110220BF06AFC002021
:106A600080BD00BF10B5314804683CB120462468A1
:106A7000017B0029F9D1FFF7CDFFF6E7002010BD1B
:106A800070B52A48084D012406685EB13046366864
:106A900001791129F9D804FA01F12942F5D0FFF75B
:106AA000B9FFF2E7002070BD200702002DE9F04198
:106AB00042B3884631B31D4D0746164600202D6867
:106AC000B5B1AB68C1B27A1A01339A4210D32A79B0
:106AD000441C56FA84F07254691D2A890BF015FC87
:106AE000287A2044EBE72C682846FFF793FF2546D9
:106AF000002DF8D10D48D0F80802C8F80000002099
:106B0000BDE8F0810120BDE8F08100BF58B100214F
:106B100001700649096821B10A7B002AFAD00121D7
:106B20000170002070470120704700BF340A002028
:106B300010B55D4A92F8201004290ED84B1C82F83B
:106B40002030936800681C4644F8040B02F11C00D6
:106B5000834208BF02F10C0494600020052938BF6D
:106B6000012010BD504890F82000704780B54E4974
:106B700091F820202AB14968FBF7F4FC08B140786D
:106B800080BD012080BD00BF2DE9F843DFF81891DA
:106B900004460025E84699F82070BD4228BFBDE8AC
:106BA000F883D9F804008678017842782170627001
:106BB0002EB1D9F8000081682046884706E0C078E9
:106BC0008DF801208DF800108DF8030000F02CF8EE
:106BD00016B94046FFF7ACFF0135DEE710B5324C81
:106BE0000021142284F8201004F10C01C4E90001F2
:106BF000A1600846FF210BF09CFB012084F82100D6
:106C000010BD00BF80B528494968FBF7ABFC0028E0
:106C100018BF012080BD00BF234890F8201000203D
:106C2000042988BF0120704710B51F4991F8200042
:106C300058B14B68421E81F8202001F11C021C1D36
:106C4000934208BF01F10C044C60002818BF0120DA
:106C500010BD00BF10B50446134890F8202042B183
:106C6000426808461146FBF77DFC10B101214470D3
:106C7000817010BD70B50C4991F8202081F8210079
:106C800082B1D1E90152012301F11C04EE78687050
:106C900006B9AB702E1DA54208BF01F10C063546A2
:106CA0009642F3D170BD00BF540C002004280FD1D0
:106CB000F8B5002004217F22CDE90200CDE90000D3
:106CC000684607F0F9FE002818BF0E2004B080BD0A
:106CD0000A20704709B10A207047F8B50021012841
:106CE000CDE90211CDE9001102D120208DF800007C
:106CF00068460021042207F0DFFE002818BF0E209E
:106D000004B080BDBCB50D46002101912AB101A996
:106D10001446FBF767FC10B1BCBD0920BCBD01984F
:106D2000411C05D081B2691A012903DB084408E03F
:106D3000256007E041B100F580304FF6FF718843D0
:106D4000284420600020BCBD20600720BCBD00009E
:106D500030B1A4490968C968013101600020704759
:106D6000092070472DE9F0438DB002B30E46F1B112
:106D700004AC0746212115462046FAF7F7FCDFF858
:106D8000C09300202B680DF10F018DF80F00D9F88A
:106D90000000B0F804802879CDE90004029138465B
:106DA0003146424607F06AFF28B10E2000E0092074
:106DB0000DB0BDE8F0832A79286804A90BF0A5FA84
:106DC000284601F03AFA08B10F20F1E7287AE9885D
:106DD00041EA0046D9F8000081688E4201D10320C3
:106DE000E6E786609DF80F000021FFF773FF00289B
:106DF000DED10420FFF75AFF0028D9D1E87AB5F890
:106E00000910434641EA0045032031462A46FBF774
:106E1000B7F80028CCD1022031462A464346FBF77A
:106E2000AFF80028C4D1D9F800109DF80F30002029
:106E30004FF0FF328B70C1E90302C1E90522B7E7C9
:106E4000B0B580B1BE4D00212822002428600BF08F
:106E500070FA28680549FF220160C46010301421CF
:106E6000FAF75AFC00E008242046B0BD00010101F9
:106E700090B11CB504460020019001A807F03CFF2A
:106E8000AF48BDF804100068E1828180204601F01F
:106E900032FF18B110201CBD092070472046132274
:106EA000012350F8181B0090002007F0FFFD08B1E7
:106EB0000E201CBD204601F01EFF002818BF012037
:106EC00000011CBDF0B587B04BB39D4E0446306841
:106ED000C068A04201D9062022E01D460FD2AB684F
:106EE00095F82810686A95F820700022CDE90024F2
:106EF0000322002F08BF022203F052FB80B928466C
:106F000001F092FE08B110200AE0296839B1287911
:106F1000043882B2B2F5807F04D90D2000E0092048
:106F200007B0F0BD0023AF6805F12C0C8DF81640BA
:106F30008DF81B008DF81A308DF81130CDF80D301A
:106F40004923CDF800C08DF80C30230E8DF8127057
:106F50008DF81930230C8DF81830230A8DF817306E
:106F60003B0E8DF815303B0C8DF814303B0A8DF834
:106F7000133003A8022307F099FD08B10E20CFE7D4
:106F8000284601F051FE0028BDD13068C4600020C1
:106F9000C6E700BF10B5044607F0D6FE08B10E20C4
:106FA00010BD0CB1002010BD65480021006880783C
:106FB000FFF790FE0028F2D10420FFF777FE0028AB
:106FC000EDD1EFE75E49096808600020704700BF17
:106FD00028B15B4909681C31016200207047092013
:106FE000704700BF780C00202DE9F04FCBB0549FC4
:106FF0007FB3064600200DF11C088B461C46154643
:10700000079010464146FBF7EDFA08B1062021E053
:107010000798A04201D30130F8D1384601F0B2F808
:1070200008B10F2016E006A93046FBF7B5FA88B97B
:10703000B868584511D1D7F800A0BAF1000F08D0B0
:107040003879061F1FFA86F9B9F5807F07D90D2018
:1070500000E009204BB0BDE8F08F0220FAE7039072
:1070600006984FF48872417880780291F96A059009
:107070004046049100210BF05CF9012000214A46B2
:107080008DF826408DF822B08DF82B608DF8210008
:1070900049208DF82A10CDF81D1051468DF81C009E
:1070A000200E8DF82900200C8DF82800200A8DF87C
:1070B00027004FEA1B608DF825004FEA1B408DF832
:1070C00024004FEA1B208DF8230008F110000BF07C
:1070D0001CF90398DDE9042300F10C01404607F098
:1070E00067FE0146012818BF0E200029B2D197F88B
:1070F0002020012397F82810786ACDE900345B46F8
:10710000002A029A08BF022203F04AFA0028A1D1FD
:10711000681E032812D8DFE800F002060A0E0848AD
:10712000006804610AE006480068446106E004481B
:107130000068846102E002480068C461002089E7B9
:10714000780C0020B0B501F00FFE08B10120B0BDF1
:107150004F4C1B4D04F55A70A84704F56070A847C2
:1071600004F56670A847FFF7B5FB06F03DF9154832
:10717000C06A80470020B0BDB0B5454C104D04F545
:107180005A70A84704F56070A84704F56670A847D0
:1071900004F20440A847FFF79DFB0A48C06A8047F5
:1071A0000020C4F8400300F011F80748424940F2BB
:1071B0007C520BF0AAF80120C4F840030020B0BDB7
:1071C000310A0108C43A01080080002070B5F64E6B
:1071D000D6F8400300B170BDF24D24212846FAF7DD
:1071E0001FFE696A884201D1002401E0012468621F
:1071F00005F1280002F066FAE96B88421CBFE863DB
:10720000023405F14000E021FAF70AFED5F820111A
:1072100088421CBFC5F82001043405F59270BC21DA
:10722000FAF7FEFDD5F8E01188421CBFC5F8E00171
:10723000083405F5F2700021FAF7F2FDD5F8E411F3
:1072400088421CBFC5F8E401103405F5F4704FF412
:107250005E71FAF7E5FDD5F8601588421CBFC5F8E8
:107260006005203405F2645002F02CFAD5F8781548
:1072700088421CBFC5F878054034D6F8480300287A
:10728000A9D0C1680029A6D02046BDE870400847B3
:107290007C14002010B561B10446084609F024FBB7
:1072A00001460020A14203D9BE4981F83A000120DD
:1072B00010BD002010BD00BF7C8500202DE9F04FDF
:1072C0008BB0002800F04D810D46002900F0498167
:1072D00004460068002800F044816068002800F03F
:1072E0004081A068002800F03C81E068002800F0A0
:1072F00038811046174606F02EF8002800F0368137
:107300002046FFF76BFCA74E002140F27C524FF065
:10731000000A30460BF00DF8DFF85C8E00214FF4C8
:10732000A46240460BF005F8A04886F804A186F850
:10733000407086F880A08DF820A0C6F818019C48FF
:10734000079006F5F470069006F5F270059005A911
:10735000384605F0FBFF0F200DF12409DFF854B289
:107360008DF8240096F840004946D847002818BFF9
:10737000012086F8080149460A208DF8240002F011
:1073800074FA86F8CC00062049468DF8240002F0F5
:107390006CFA86F8CD00102049468DF8240002F0E2
:1073A00064FAC6F8900096F84000112749468DF817
:1073B0002470D847C6F89400122049468DF824005E
:1073C00002F053FAC6F89800132049468DF82400BD
:1073D00002F04BFAC6F89C00142049468DF82400B0
:1073E00002F043FAC6F8A000162049468DF82400A2
:1073F00002F03BFA86F8A500172049468DF82400D4
:1074000002F033FAC6F8B000C6F8A80018204946C2
:107410008DF8240002F029FA86F8B40086F8AC0052
:107420001D2049468DF8240002F01FFA86F8B800A6
:107430001E2049468DF8240002F017FA86F8B9009C
:107440001F2049468DF8240002F00FFAC6F8BC0050
:10745000202049468DF8240002F007FAC6F8C00043
:107460000B2049468DF8240002F0FFF9A8F800042B
:107470000C2049468DF8240002F0F7F94FF001097D
:107480000621A8F802040A2006F1900C06F14C0E21
:10749000C8F8485386F8A49086F88C10C6F888007F
:1074A00086F84810706486F80B9186F860909CE826
:1074B0000F108EE80F1005F097FF88F895A4C8E923
:1074C000D0943D4B3D4C08F55A704FF0FF310022EF
:1074D00086F80591C6E90BAACDF800A0A047384B65
:1074E00008F560704FF0FF310022CDF800A0A047F2
:1074F000344B08F566704FF0FF310022CDF800A044
:10750000A047314B08F204404FF0FF310022CDF884
:1075100000A0A04702A807F015FEDDE902012D4AF0
:107520002E4C2D4BC6E944013648C8E9D3242849DE
:107530002B4CC0F800A02548C8E9D5132168C8F82D
:107540005C0308F553708847A96806F5927007F048
:10755000E9FA38B9134D2846FFF772FC40B11127FC
:1075600000E0032738460BB0BDE8F08F0927F9E7A4
:10757000FFF742FA08B11327F4E705F1D800FFF747
:1075800027FD0028EBD16069E66AA46D80470AF008
:1075900061FF95F80501A047B0470120002788F852
:1075A0009604DFE77C8500207C14002000040001A5
:1075B000A01A002039D30008D1A30008A1080108AF
:1075C000BDA1000801A20008E5A00008F19E000886
:1075D000959E0008519F00080D9F0008A59F000878
:1075E000C43A010807480078C00709D1DD48D0F83F
:1075F000401329B990F89604012801D10020704762
:1076000001207047880200202DE9F04F95B0002836
:1076100000F02281044600200E4601272061FFF77A
:10762000E1FF002840F08E81A089DFF84C8B00211B
:1076300094F80EB0257814220790D4E901A008919F
:107640000021099008F244400AF073FEDFF82C9BF9
:1076500088F8457499F8040199F81C2199F80A11E1
:1076600080F0020082F00202294310430843000622
:1076700008BF012506950496E8B2032804D0012826
:107680000CD090B940200AE009995046E0224FF012
:10769000010A4FEA114BCDE907120BE08020CDF82B
:1076A00014A04FF0010A089007E04FF0000B4FF0D4
:1076B000000A002009900020059099F87410022714
:1076C00099F840008DF82C708DF82E100BA905F05C
:1076D00033FE46B24FFA8BF18E42B8BF0E4699F890
:1076E0001C2199F8091199F8063182F001050D4322
:1076F00018BF3046002B08BF30464646BAF1000F8F
:1077000000F01D811BB1012A08BF002912D199F890
:1077100074108DF8280099F8400005228DF82A1081
:107720000AA905F059FE002800F096809DF828006F
:1077300089F83900D6F89C14D9F88400FFF7AAFD1F
:1077400099F81C11D9F8280099F8392099F838A02F
:107750000029129000F0828099F8071111B90021D8
:10776000C9F830100E9001204B4603928DF840204E
:107770008DF841A08DF83400D6F800040F9013F86E
:10778000600F13F8201C1A7D93F8A4508DF8420066
:1077900013F8260C8DF8441093F8A6108DF84320AA
:1077A000012DA3F128024FEAC11BA3F1270108BF55
:1077B0000BF1100B002818BF0BF1200B5FFA8BF0B8
:1077C000C0098DF8350012A800900DA8FFF714F835
:1077D000099902900020079D86F81E043080CDE9AB
:1077E000130006F59C70002908BF0D46AAB280461A
:1077F0000AF08BFD0899022786F83752B7EB511F24
:10780000B17008D0480907282AD0042840F08380A6
:10781000012086F81E04029886F80D1186F8305172
:10782000C6F82C8160F3861B059886F814B186F89B
:107830002801FF2086F80C01042086F80401B01C02
:10784000C6F80801D9F8D400C6F8100114A8FFF74B
:107850007FFAA0B112275EE0032773E007275FE0FD
:107860000998002852D0280650D00999F01CEAB295
:107870000AF04BFD96F837020130308046E014984C
:10788000A6F81601C6F850040020A6F8480413A86C
:10789000FFF7A8F808B113273DE01398B0B399F9A2
:1078A0003900FAF7C7FE96F83772139D9FB10F2D76
:1078B00011D806F58C7213A90F20FFF7F7F80028EE
:1078C000E9D19DF84C100BF0F00001F00F010844D5
:1078D00086F814011AE0D34606F5946A13A95246B5
:1078E000FFF7E4F82FB1102D03D30028DA46D2D1E8
:1078F0000CE010B11327DA460DE00020C6F82CA1E9
:10790000DA4686F82801139886F83001049806F0C4
:1079100033FF0746D0B1039889F838A089F83900B9
:107920001FB1002086F81E0409E00698002786F89B
:10793000440496F8950440F0010086F89504D6F8C2
:1079400098042061384615B0BDE8F08F12980027E2
:1079500089F83A70C9F82800FFF784F80028DFD0CA
:107960001327DDE77C140020022070471CB5002897
:1079700000F0458004460078392800F25880DFE89E
:1079800010F03A004000440047004A004E00520008
:107990005600560056005600560056005600560037
:1079A0005A005E006200640068006C0070007500A0
:1079B00077008100850088008B008E009100940084
:1079C000A200A600AA00AE00B200B500B900BC003B
:1079D000C000C2005600C4005600560056005600B3
:1079E00056005600560056005600560056005600E7
:1079F0005600CC00D1004E4890F8040195E00320D9
:107A00001CBD4B4890F81C018FE007F071F887E02F
:107A100007F072F884E0464890F8060185E0444893
:107A2000D0F8D0007CE04248D0F8D40078E020467E
:107A3000FEF75EFF1CBD3E4890F8050175E03C482E
:107A400090F8800071E01C2013E03948D0E919104B
:107A50000AE03748D0E92A1006E03548D0E91B1083
:107A600002E03348D0E92C10616054E0192000E0B6
:107A70001A208DF800002E48694690F8400005F065
:107A80005BFC4DE02A4890F860004EE02848C06C4E
:107A900046E02748006D43E02548406D40E024481B
:107AA000806D3DE02248C06D3AE0214902208DF80A
:107AB000000091F8400091F874108DF802106946AA
:107AC00005F03AFC31E01A4890F8CD002DE0184856
:107AD00090F8390029E0164890F8380025E014485D
:107AE00090F8CC0021E01248406C19E0104890F862
:107AF00048001AE00E48C06F12E00D48D0F8C000F0
:107B00000EE00B480CE00B480AE00948D0F81801D9
:107B1000606005F017FCA06008E00548D0F884001C
:107B2000606003E0024890F80B01207100201CBD4A
:107B30007C850020008000207FB5002800F0B78100
:107B4000DFF834660446D6F84003810700F1158259
:107B50002178392900F25F81DFE811F03A003E0018
:107B600047003E014B00510057005D006300690073
:107B70006F0075007B00810044014E0158015D01DA
:107B8000640187009B007F01BE00C000CF00D800C9
:107B9000DC00E0009101E4005D01E8009501FA00DD
:107BA0000C011E01AB01B2012401BD015D012901DF
:107BB0005D015D015D015D015D015D015D015D01D5
:107BC0005D015D015D015D015D015D013401390112
:107BD000207907F003FA21E12079022800F067817B
:107BE000DFF87C1F81F81C016DE1606807F092F8F6
:107BF000F5E02079DFF8681F81F8060163E160682D
:107C0000DFF85C1FC1F8D0005DE16068DFF8501F4D
:107C1000C1F8D40057E16168002900F048810020D4
:107C2000E4E06168002900F042810120DEE0616843
:107C3000002900F03C810220D8E06168002900F0B2
:107C400036810320D2E06168002900F030817F2076
:107C5000CCE06168002900F02A818020C6E06168DC
:107C6000002900F024818120C0E0C64D01F035FFDD
:107C70008DF8040095F840008DF8051001A905F075
:107C8000ABFB002800F01381D4E90101C5E92A010A
:107C900019E1BC4D01F021FF8DF8040095F840007A
:107CA0008DF8051001A905F097FB002800F0FF8072
:107CB000D4E90101C5E91B0195F80401022840F04F
:107CC000028195F81C01002800F0FD80AF48C06AD1
:107CD000804702F0F1FBF6E0002000E001208DF883
:107CE0000C0060680290A74890F8400002A904F0D8
:107CF000C0FF002800F0DB80E5E02079411E0E295E
:107D000000F2D5809F4981F86000DCE060689D4901
:107D1000C864D8E060689B490865D4E06068994908
:107D20004865D0E060689749C865CCE02079954CFB
:107D300006228DF8040094F8400001A905F04CFBE0
:107D4000002800F0B4809DF8040084F8CD00BAE06B
:107D500020798C4C09228DF8040094F8400001A988
:107D600005F03AFB002800F0A2809DF8040084F89A
:107D70003800A8E02079834C0A228DF8040094F89A
:107D8000400001A905F028FB002800F090809DF834
:107D9000040084F8CC0096E06068F8494864C1F8B3
:107DA000880090E06068F549C1F8C0008BE0A079D8
:107DB00001287CD86068F149C1F818016068FFF7B4
:107DC00001F915E06068ED49C1F884007BE0207995
:107DD000EA4981F80B0176E0606806F0A7FF002809
:107DE00065D170E06168002961D08220FFF7D2F888
:107DF000002868D01120C1E02079E04981F8050110
:107E0000DF49CC6A896D8847A0475CE02079DB496F
:107E100081F8800057E02046FFF7A6FD002840F0DB
:107E2000AD8050E0D54D01F058FE8DF8040095F876
:107E300040008DF8051001A905F0CEFAB8B36068CE
:107E40000022019095F8400001A905F0C5FA70B331
:107E5000D4E90101C5E9190135E0C84D01F03DFE45
:107E60008DF8040095F840008DF8051001A905F083
:107E7000B3FAE0B1D4E90101C5E92C0123E060685F
:107E8000BE4988651FE02079BC4C052294F8741027
:107E90008DF8040094F840008DF8061001A905F053
:107EA0009BFA20B19DF8040084F839000BE0032010
:107EB00064E02079B14981F8480081F88C0002E043
:107EC0006068AE49C86796F8950440F0400086F8AF
:107ED0009504002052E001284FD12B4C242120464C
:107EE000F9F79EFF616A88424AD104F1280001F047
:107EF000E9FBE16B884243D104F14000E021F9F74E
:107F00008FFFD4F8201188423AD104F59270BC2139
:107F1000F9F786FFD4F8E011884231D104F5F27008
:107F20000021F9F77DFFD4F8E411884228D104F24A
:107F3000645001F0C7FBD4F87815884220D18F4CEB
:107F4000114D40F27C52204629460AF0DEF92846BF
:107F5000002140F27C520AF0ECF940F20120A6F830
:107F6000FA0396F81F0486F8E803E06EC6F8EC03FF
:107F700094F8750086F8F803A5E7012004B070BDF9
:107F80001720FBE77C85002000800020C43A010810
:107F9000F0B587B004460020ADF8160044B120616A
:107FA000FFF720FB10B9FEF737FE28B1012500E0EE
:107FB0000325284607B0F0BDFEF7D4FD30B96E4862
:107FC0000021142200F58B600AF0B3F96A4E0021FB
:107FD00002258DF81B1096F8950440F0040086F8F1
:107FE0009504012086F85904ADF8190020788DF821
:107FF000180001380C2800F28080DFE800F0077ECE
:108000007E4D517E7E7E5F7E6370760096F84003E3
:108010008006CBD420790225012800F08C8002282C
:108020006BD105F0E1F9554F94F9051000220025B8
:1080300097F8400004F009FE87F8390007208DF812
:108040001900002006F0CAFFFF2086F80451A6F8A8
:108050000C01B01CC6F8080106F04EFD014606F5FD
:10806000877008220AF051F906F042FD014606F534
:108070008B7008220AF049F9002006F07DFB0028E9
:1080800071D0054694F9051097F84000012204F0DC
:10809000DCFD87F8390030E00DF11601022027E001
:1080A000374B94F90C10A068A288DB6B9847D6F880
:1080B000400340F00200C6F8400354E00DF1160101
:1080C0000D2015E001258DF81B50FEF705FCA0B929
:1080D0000020FEF718FC0020FEF7F9FB43E02748DC
:1080E00090F80401D8B1022507E00DF11601122025
:1080F0000022FEF711FCB0B31325D6F898042061D6
:10810000FEF730FD00287FF454AF002086F81E04EF
:1081100096F8950400F0FB0086F8950449E7257968
:1081200005F00700FEF7F2FB8DF816500DF1160171
:1081300010200122DDE7114F00208DF8105087F844
:10814000090197F8400001A905F000F9207987F8A6
:108150001C014FF48070ADF81900D6F8480300698F
:10816000804701F0D2FDD6F89804206106A8FEF7FA
:10817000DFFC00251DE700BF7C1400207C8500206B
:10818000C43A0108B0B5002855D00168044600295A
:1081900051D0087860714878A0608A7840EA02205F
:1081A000A060CA7840EA0240A0600A7940EA026012
:1081B000A0604A79227302F00F028879E081CB79BE
:1081C000083140EA0320E08104F110000AF09DF834
:1081D0000020217984F8280084F82000207B00F01A
:1081E0000F0202F10803C81A05280EDB25680932C0
:1081F000606A891AEB5C84F820300B1FA918DAB288
:1082000084F828300AF081F821792068084410F8B1
:10821000041CE16210F8032C41EA0221E16210F82B
:10822000022C41EA0241E16210F8010C41EA0060CF
:10823000E0620020B0BD0220B0BD10B578B3016887
:10824000044661B311F8010B03226071A01D0AF00E
:108250005CF8216804F10900032204310AF055F8A2
:108260002168C879E0600A7A40EA0220E0604A7A30
:1082700040EA0240E0608A7A40EA0260E060C87A40
:108280002074087B6074207921280AD104F112003F
:108290000D3110220AF039F821681D2006E0022075
:1082A00010BD112801D9012010BD0D200A5C0B184A
:1082B00040F0020062625B7842EA032262620B5C79
:1082C000084442EA03426262407842EA0060606227
:1082D000002010BD2DE9F04F99B0DFF88068EFF372
:1082E0001080EFF3108172B60023F178B6F8012008
:1082F00096F80090336080F3108842EA014049EA22
:108300000020002800F099815FEA896058D5DFF8E5
:10831000A05A95F80401022803D0DFF84808C06A83
:108320008047DFF8687A07F56074D7F8B01301F07A
:10833000D5F901F0EAF907F56674D7F8B41301F03E
:10834000CDF901F0E2F997F81E0488B115208DF8F7
:10835000200095F8400008A904F0EEFFD7F8B41308
:1083600007F20444014401F0B9F901F0CEF902E04A
:10837000002087F845047068E8620B9097F81F04A6
:108380008DF8280006A806F0DDFED5E94430DDE9C9
:108390000612009016A806F001FFDDE91601CDE9EE
:1083A0000D01D7F8200495F81C110C9095F84000A9
:1083B000002918BF01218DF829100AA904F0F9FF3E
:1083C0005FEAC96040F10181DFF8C0B9DFF8E04938
:1083D0000020317896F81480778AF568B6F810A0F6
:1083E0000690CBF82C048BF84804ABF826048BF8E5
:1083F00029048BF824048BF83C04CBF83404CBF824
:108400003804CBF84004CBF82F04D4F8D40001F0A2
:10841000FE018BF89284ABF8907431709BF8941441
:108420000590DFF840078BF89314C06A80479BF8EB
:10843000930418B90BF5667008F0FAFA284651460D
:10844000FEF75FFA20B18BF88484ABF88274BCE04D
:1084500094F80401012816D1FEF746FA38B100203D
:10846000FEF755FA0020FEF749FA042009E0FEF76E
:1084700039FA40B10020FEF748FA0020FEF73AFA38
:1084800005208BF893042C784FF0FF3000EB54104C
:10849000062824D8DFE800F004232C2329236300D6
:1084A000BAF1100F55D9DFF808798DF82CA00A958C
:1084B00097F81C0100284CD106F01EFB0AAD0146BE
:1084C000FF202A46FEF74EFC002800F0B381012071
:1084D000FEF798FB002800F0EC810720E6E1012080
:1084E0008BF8250402F0BEF84FE001208BF824043D
:1084F000DFF8BC2892F8751092F8400092F88020BE
:108500008DF85A109BF828148DF859100E21002A66
:1085100008BF0D218DF8581016A904F00DFFAAF11F
:108520000D0100B209B221EAE171814211DCBAF118
:108530000B0F0ED9FF208DF82CA00A958DF8500056
:108540000BF50E7013900AA8FFF71CFE002800F030
:10855000598101208BF8250402F084F835E00BF5F1
:108560000E78AAF10104691CA2B2404609F0CDFEC2
:1085700003208BF83044CBF82C84ABF824049BF810
:10858000950440F002008BF89504DFF824789BF8FE
:10859000930401280AD89BF81E0448B19BF84804AC
:1085A00030B1002001F09EFD9BF89304022805D015
:1085B0009BF8950440F020008BF8950497F804018F
:1085C000022818BF06208BF894045FEA097026D5AC
:1085D000DFF8DC57022495F8040102284FF002006E
:1085E00008D0DFF88005C06A804795F804010228AA
:1085F00018BF0620DFF8945785F89404022085F808
:108600004544FEF737FB95F81E0410B1012085F8AC
:108610001D0495F8950440F0200085F895045FEA64
:10862000497003D505200621FDF7A6F85FEA897099
:1086300003D503200421FDF79FF8FEF760F9DFF86A
:108640004C4794F89514880640F1B380002084F8D4
:108650009604D4F84003020644BF20F08200C4F818
:10866000400311F0050F0AD00B20FEF7CBFA94F867
:10867000951420B111F0010001D148072DD448070D
:1086800011D50120FEF7BEFA38B10120FEF76EFACF
:1086900038B9002084F81C0403E00520FEF7B2FA84
:1086A00008B101F0BDFB94F89504C1073FD094F8E0
:1086B0004414032902D0012912D071BBDFF8F0164F
:1086C00094F81C2491F860108A4219D2810724D5AD
:1086D00094F89314022913D31FE001F0A1FB2AE0C0
:1086E00094F81D1419B3DFF8C81694F81C2491F8F7
:1086F00060108A4204D281070FD594F8481461B102
:1087000004F55A7008F094F9D4F8400320F02000E2
:10871000C4F8400306F040FC09E000F0DF0000214F
:1087200084F89504002084F81D1401F051FE94F89B
:108730009514D4F84003A8BB01F0010001F0040532
:108740002A1804D085F0FE02114084F89514012106
:1087500084F8961428B1D4F84403016804F2444024
:10876000884765B104F58B60FEF70EFAFEF7FAF95B
:1087700028B194F8950440F0040084F89504FEF7BD
:10878000BFF894F8950400F0DF01D4F8400384F8B2
:10879000951438B900208DF828000AA8FEF7B6F91C
:1087A00094F8951441F04001012084F8960484F86F
:1087B0009514080709D501F0F70001F063FAC268C3
:1087C00004F26C40904794F89514880707D501F09F
:1087D000FD0001F057FA426804F22440904794F8F3
:1087E0009404022808BF01F067FE94F8950441063E
:1087F00005D500F0BF0084F89504FEF7E7FC19B03A
:10880000BDE8F08FD64890F8040101286BD1FEF73F
:108810006BF8002854D00020FEF779F80020FEF70E
:108820006DF89DF8341004208BF893040C98C1F374
:10883000001156E00021BDF831200D9887F81A117B
:108840009DF8331042EA0141C7E934109DF8380021
:1088500000F00F01C0F3021087F861009DF83900A5
:1088600087F8701087F868104FF47A71002808BFF5
:10887000012010FB01124843C7E91402AAF11100BC
:108880008DF8600005F1120017909BF81F048DF819
:10889000580097F8400016A904F0DEF9022087F886
:1088A0001C010120FEF7AEF918B100200121FEF7EE
:1088B000D1F99BF8950440F008008BF8950466E622
:1088C000FEF710F878B10020FEF71FF80020FEF741
:1088D00011F805208BF893049DF83400C0F30011C3
:1088E0000C98FEF711F80C989DF834C08246CBF82E
:1088F00038045FEA0C7004D09DF8480060B1002095
:1089000012E09DF8500070B19DF848000321002846
:1089100008BF0221049108E09DF85000012110B128
:108920008BF8251418E601200490DFF884E4600930
:10893000002301272C2103900693FC072AD003FB78
:1089400001E01A4601230027D0F8DC505545F4D148
:1089500090F8DA00012300270028EED02C2002FB3B
:1089600000E0D0F8F81090F8DB209EF804010968C8
:108970000228069102D103208BF893041CF0600FAB
:10898000049808BF03287FF4E4AD002A7DD0012AB3
:1089900003D021E0DDF814A000229EF81A014FF464
:1089A0008031B1EB004F07D1049802270AAD28B1FE
:1089B000032818BF012701E00AAD03270120029216
:1089C0000590BDF8361006AA3846FEF79BF960B14F
:1089D000072801D1082000E001208BF82504069823
:1089E000CBF87004CBF83404B6E5069B05985146E5
:1089F0003A460095FEF7F8FA18B102282CD10A2061
:108A0000A8E502980022EA4F8BF825248BF8302441
:108A1000CBF82C248BF845248BF826040698CBF849
:108A20007004CBF834049DF83400C0F300118BF8C7
:108A30002914C0F340118BF848148BF832149BF8BA
:108A40009314012903D80123BA6287F80A31002C54
:108A50002C4603D0022221E00B207BE5039A052A55
:108A600019D197F81A31012287F83A200BB9159BD2
:108A70007B6302298BF8242414D3D7F88400CBF825
:108A80004004B068CBF89C0414E0012005920AADC4
:108A90000427029095E7002287F83A2001298BF8F5
:108AA000242407D89BF84414012901D1800601D55C
:108AB000FDF7E6FF0499DFE801F0021922309DF886
:108AC00034109BF8933404F110004FFA88F201F04F
:108AD0000F0101F089FE012013998BF831049DF8F4
:108AE0004800CBF82C148BF8270420E09DF83410B4
:108AF0009BF8933404F1100001F00F0104E09BF89F
:108B000093349DF8501013984FFA88F201F06CFEE0
:108B10009DF848008BF827040DE013999DF8480054
:108B2000CBF82C1401218BF827048BF831149DF815
:108B300050108BF83014E0280AD197F80B0138B99F
:108B40000020ABF83004CBF82C04E0208BF827048D
:108B50009BF8950440F00200AFE600BF88020020B9
:108B60007C850020C43A010870B58AB0054690485B
:108B70000C460026029690F8CD20816A8DF80F20D1
:108B800090F8CC2004918DF80E20804A92F81C3485
:108B90008DF80D308CB3069190F806118DF82230C7
:108BA00090F840308DF814608DF81510D2F800144C
:108BB00090F839208DF824300DF10D03079190F8CD
:108BC000381090F874008DF820200DF10E028DF809
:108BD00021108DF8230004A80DF10F01009005A8C5
:108BE000FDF70AFE9DF90F00F9F724FD607002A859
:108BF000FDF7F8FE18B1132013E0032011E00298EE
:108C00000F2802D86178884203D9002020700820FC
:108C100007E00A1A284422700022884288BF0122F5
:108C2000D0000AB070BD00BFB0B598B1044600686E
:108C300080B1227B94F828300925217902F00F02B7
:108C4000002B08BF08252A441A4404328A4203D95B
:108C50000220B0BD0120B0BD617901702068A1681B
:108C60004170A1682068090A817020686189C1701B
:108C70002068E17A01712068217B41712068A17B25
:108C800081712068E17BC17104F11001227B2068B1
:108C9000083002F00F0209F038FB207B94F828100E
:108CA00000F00F0000F1080539B1206894F8201099
:108CB0004155013594F8282000E000222068616ABF
:108CC000284409F022FB94F828002168E26A28442D
:108CD0000A542168E26A0144120A4A702168E28D4E
:108CE00001448A70216894F82F2001440430CA702E
:108CF00020710020B0BD10B538B10446006820B125
:108D00002179172903D2022010BD012010BD6179FD
:108D100008220170A11D2068013009F0FFFA2068C7
:108D200004F10E010822093009F0F8FA2068A17D4B
:108D300041742068E17D81742068A169C174A169D2
:108D40002068090A01752068618B41752068E17E01
:108D5000817517202071002010BD00000B480021F4
:108D6000C0F840130020704780B5FEF73BFC30B1DF
:108D70000648D0F84003013818BF012080BD0348E1
:108D80000121C0F84013002080BD00BF7C140020EA
:108D9000BCB5074D04468DF804000F2295F840003D
:108DA00001A904F019FB08B185F80841BCBD00BF5A
:108DB0007C8500202DE9FC474FF000090020CDF80C
:108DC000049001AC2146FDF7A9F801202146FDF7EA
:108DD000A5F8DFF8ECA03B4B3B4C4FF4FA710022B6
:108DE000CDF800900AF12400A047384B0AF13C006E
:108DF0004FF4FA710022CDF80090A0470AF1540513
:108E0000334B4FF4FA710122CDF800902846A04769
:108E10000020F9F741FA08B1F9F7C6F9DFF8B48094
:108E20002D4B4FF4FA610022CDF80090404607F038
:108E300037FD2A4A2A4F01200021B847294A02203B
:108E400000210226B847284A04200021B847274AB3
:108E500008200021B84700F059F825484FF08171EB
:108E6000FDF774F8234C04F11000FCF711FF2846BD
:108E700007F0A8FD9AF80300002818BF0126304625
:108E80000021FDF797F804F02FFD1B4A2020002158
:108E9000B8471A4A40200021B847194A102000213B
:108EA000B847216808F13004164B0022CDF8009035
:108EB000204607F0F5FC204607F084FDBDE8FC875E
:108EC0008403002065A40008A1080108ADA10008E2
:108ED000619E0008F00300204DA20008A161000877
:108EE00081070108E1ED0008D9EF000825EF00082F
:108EF00008010020000000207DD80008D1D900081A
:108F00005DDB000875A4000805487047044800218F
:108F100001220323C0E90032C0E90211704700BFFB
:108F2000FC4D002010B51348002107224FF4805358
:108F3000114CC16480F83C10C0E90C3282630122FC
:108F400080F82C10C0E909114FF0004380F8201080
:108F500081760183C2610422C0E90043C0E90211A5
:108F6000C0E90412F9F784FD18B1BDE81040F9F723
:108F70001BB910BDB44B00200024014080B5042073
:108F8000FCF726FE0120FCF723FE0F200221002221
:108F9000FAF706FE0F20BDE88040FAF7F3BD0000A7
:108FA0002DE9F04186B02D4D002402204FF002083B
:108FB000CDE90444A8470420A84701200127A84779
:108FC0000320274D0394274E02904FF6FF70019027
:108FD00001AC28462146B04705F580602146B047E0
:108FE0004FF090402146B0471F480022016821F011
:108FF00002010160016821F00401016028464FF47C
:109000003A41FAF7D1FA4FF4041003972146CDE91B
:1090100001804FF09040B0474FF48810CDF80C809D
:109020002146CDE901704FF09040B0470F4C06202B
:1090300000210022A0470E4D0620A847072000214E
:109040000022A0470720A847162000210022A047A1
:109050001620A84706B0BDE8F08100BFED5B000810
:1090600000040048113400084C000058A13B0008DF
:10907000853B000810B50F4C0F4A104B0120002112
:10908000C4E90032C4E9021004F110001421F8F719
:109090006DFB2046FAF7E8FA50B906480021FAF7C6
:1090A000A5FA28B903480021FAF7BEFA00B910BDA5
:1090B000F9F77AF8784C00201A0910200054004083
:1090C00080B506F097F8BDE88040FFF773BE4FF01B
:1090D000FF3007F065BB000080B58CB001A82C21E3
:1090E000F8F744FB174800224FF480714FF080439B
:1090F000C0E90422C0E90623C0E908211F218160DC
:1091000011490160FBF754FB08B1F9F74DF80D4820
:10911000FBF7DEFA08B1F9F747F84FF48070002248
:109120000B904FF00050079000200690029008909E
:10913000044801A9FBF7C2FB08B1F9F735F80CB0F8
:1091400080BD00BFDC4C00200028004080B50548F1
:1091500008210160FBF702FD18B1BDE88040F9F776
:1091600023B880BD144D0020B0B588B0184C194DFF
:10917000164800224FF0804140F2E7330792CDE9D4
:109180000522CDE90322CDE9012224688261B4FBE6
:10919000F5F4013CC0E90014C0E902230261FBF7C9
:1091A00049FE88B94FF480500490084804A9FBF7A1
:1091B0009FFE48B9002003900190044801A9FBF7E5
:1091C0000DFE08B908B0B0BDF8F7EEFF204D002045
:1091D0005801002040420F0010B5174C174B4FF4B8
:1091E000E1320C200021C4E90032C4E90211C4E9D3
:1091F000041004F118001421F8F7B8FA2046FCF71F
:109200007BF908B1F8F7D0FF0B480021FBF7C7FF47
:1092100008B1F8F7C9FF08480021FBF7B2FF08B111
:10922000F8F7C2FF0448FBF770FF18B1BDE8104023
:10923000F8F7BABF10BD00BF6C4D002000440040DD
:10924000B0B5044663480121A278E378257900F897
:10925000341F61788272037645724170E168C160A3
:10926000216941765C494968896A8847002021461E
:10927000BDE8B040FCF776BFBFB5044655480122B3
:1092800000238DF8073002726278427202B1BFBDCE
:1092900023798D78E27803740B78C97885744E4D04
:1092A0008DF808200176216943744161217B8DF896
:1092B0000910A16803916968CA6A00F1080102A84F
:1092C00090476868806B10B1217E01B18047012012
:1092D0002146FCF747FF0DF10700FCF7EFFD607931
:1092E0000128D4D19DF807000028D0D10120287092
:1092F000BFBD00BFFEE7000070B58AB0354D044623
:109300000021354E284600F8341F6178417071689D
:10931000896A884702202146FCF724FF20780B2821
:1093200013D0042818D0012829D106208DF8040074
:1093300001A8FEF71BFB02982863281DFCF7D6FD49
:10934000607870B1FF20687111E06078B8B10AB040
:10935000BDE87040FCF7A2BD0120687620896883D3
:109360000DE00020687196F84100FCF747FF706837
:10937000416A18488847607808B905F071FC0AB05E
:1093800070BD00BFB0B50446124800226378A578CE
:1093900002722278437205740B788D78C978017651
:1093A000616843748574416142F004010E2906D05E
:1093B00009494968CA6A00F1080100209047032062
:1093C0002146FCF7CFFE2078062802D10248012171
:1093D0000170B0BD700000201C030020FEE70000FB
:1093E0000D490A8810430880704700BF80B50A48BD
:1093F000008830B1FFF7B8FC002818BF6FF00200FA
:1094000080BD6FF0010080BD80B503480021018060
:10941000FFF7A4FC002080BD9C1900208202810D72
:10942000002310464FF47A72F8F734B84FF4006115
:109430000022FAF7B9B8A06D40F01000A065E06D09
:1094400040F00100E065012070474FF0B040016836
:1094500041F008010160DAE90912036823F0F00322
:109460001A430260206820F47F4040EA0120206017
:1094700070474FF6FF72F36F62EA01021A4042EA48
:109480000141F16770474FF47A70F8F7FFBF012090
:1094900084F8240094F8250001287047086820F01B
:1094A000040008607047016821F002010160704704
:1094B00029786A78AB78EE7840EA0140296A40EA78
:1094C0000220184340EA8650084395F8241040EAE9
:1094D00001607047FF22CA600021012280F82C1031
:1094E00080F82D20704701201D4616460F466071FA
:1094F000204604F0C7BB206850E8000F216820F028
:10950000100041E80002002A70472420C4F88400BB
:1095100020680568026822F001020260012284F8D6
:109520008020826870471160116841F0010111606C
:109530000021202280F8401080F8412070477218E6
:109540005278D30943EA4000705401311046704705
:109550000220002100224047084611461A462346B1
:10956000704702200021012207F028B841EA0020BC
:109570000AF10401C9B21BF8011040EA014064215C
:1095800048437047012304F043BE4FF0FF3070475B
:1095900002200021012207F011B8014620460AF0FE
:1095A00039B920464FF48071FBF7CAB82046F8F766
:1095B000DDB8012084F854002046F8F74BB930603C
:1095C000F9F7F8BF0D4690F82C1004460220012947
:1095D0007047D9F8000040F40040C9F80000204668
:1095E00004F074BB012084F8480084F83E0084F83D
:1095F0003F0084F8400084F8410084F8420084F879
:10960000430084F8440084F8450084F8460084F858
:10961000470084F83D00002010BD2420C4F88400D9
:109620002068016821F001010160204606F0D0BBEE
:10963000206820210560002084F88000C4F8841090
:10964000B0BD044690F8410020287047013091F8E1
:10965000F12091F801315A4081F8F120704710193A
:1096600001380860002010BD0AF10201E0B2C9B261
:109670001BF800001BF8011040EA01200AF1030169
:10968000C9B21BF8011040EA01406421704713463B
:109690000A46014670470022002304F029BD2046F7
:1096A00001F084BCCA22CA605322CA600A687047AB
:1096B000016851E8021F026821F4000142E8021328
:1096C000002B70471421F8F7ABBB29460AF0A2B86B
:1096D000016841F00101016020467047204607F013
:1096E00059B9014628460AF095B8002532463B464E
:1096F00084F84100402084F842006564C4F824B036
:109700006563A4F82A8088467047204607F05AB956
:10971000304609F02BBF04460068D0F81CA0016851
:109720008268B4F86050D4F88830222B70472068E3
:10973000616A406A0870608D01386085606A013036
:109740006062208D411E21850904608D704751465D
:1097500009F00CBF51E8001F026821F4907142E843
:109760000013002B70472046FCF76EB9294609F01C
:109770009FBC616A206811F8012B8262608D0138FC
:1097800060856162208D411E21850904608D7047CE
:1097900053E8003F046843F0806344E80035002D3F
:1097A0007047594609F0E2BE28460AF033B8042152
:1097B0000162D4F88C0040F00200C4F88C007047BD
:1097C0006064202084F84100002084F8400084F880
:1097D00042007047414609F0C9BE02220262D4F835
:1097E0008C2042F00402C4F88C20704700F1180469
:1097F000204607F01DB9002084F85400A06D40F009
:109800000400A0650320BDE8F0810546D4F88C0073
:1098100041F288367047016841F0020101607047EB
:10982000FF20F8600020226B84F82C001143216394
:10983000012184F82D107047002001216071A0687B
:10984000A1710028704750E8020F216820F0400005
:1098500041E80202002A7047B3185B78DF0947EA43
:109860004101B15401321946704796F840005847FB
:10987000012204F0FBBE002004F0E8BD394609F0E7
:1098800017BC01220262D4F88C2042F00102C4F815
:109890008C207047B0F85C10FBF771BC394609F0BA
:1098A00065BE2020C4F88800C4F870B0E06E0128BE
:1098B0007047214609F0AEBF0027C16142681A40D7
:1098C000426084F8411084F8407084F84270704718
:1098D0000146304609F09EBFD1E90123C9681A4309
:1098E00042EA0121826822F47F421143816081684B
:1098F0007047494609F03ABE886940F0080088611F
:1099000070470025C16142681A40426084F84110E6
:1099100084F8405084F842507047294609F026BE2A
:10992000002084F83C0020467047314609F01EBEF6
:10993000C366012380F880300368A3427047044661
:1099400007F060B9C9F800400760BDE8F88F21460C
:1099500009F00CBEB4F85C102046FBF710BC514671
:1099600009F0A6BB012004F0CBB8411B032002295B
:109970007047016821F0010101607047086889465D
:1099800020F4004008602046704741E80202002AA7
:109990007047044690F8800001287047C9B21BF850
:1099A00000001BF801107047016000200021A06535
:1099B00094F8560004F067BD0146204609F078BBD4
:1099C000834699468A4600244FF00108704728468E
:1099D00009F0CCBD51E8001F026841F4807142E8F3
:1099E0000013002B7047FF21FF224FF08073218569
:1099F000009070470146304609F05ABB2068416824
:109A000021F49041416081687047618D4FF000738F
:109A100021850090CAB27047314609F0FBBE02F0C2
:109A2000010901F480784FF0000B7047414609F0BE
:109A30003FBB204605F022BF84F84100102084F887
:109A4000420000206064668560636562704780F84C
:109A50008010016982F480520A4370472046FBF768
:109A6000EABE514609F0D6BE314609F021BB284670
:109A70004FF40072214607F0DBBC044690F8540016
:109A8000012870473860F9F795BDF26F22EA11425C
:109A900089B21143F1677047CA21F9605321F96017
:109AA0003968AA6AB2F5807F7047D8F8000040F4A0
:109AB0000040C8F80000204604F008B9016851E8E9
:109AC000001F026841F0400142E80013002B70477C
:109AD00011438160204605F0AFBE207A072295F839
:109AE000751070472046FDF741BF214600F11C0567
:109AF000284606F04FBF05463846394609F036BDC0
:109B0000191D03F108020C331B8812680968838150
:109B1000826041600020704701271E461546884636
:109B200084F84070F9F746BD2068290A3A468162F8
:109B300020464146FCF72DB8204609F017BD2846BF
:109B400009F0B6BA01251F4616468A4684F84050E9
:109B5000F9F730BD204631462A46FBF77BBE594611
:109B600009F058BE404609F055BE90F83C20044626
:109B70000220012A704702400020062A7047608DAB
:109B8000B0F5807F7047494609F044BE4FF48071BC
:109B900007F065BC012084F854002046F7F7AEBEFC
:109BA000C4F89000F9F706BD84F82C0057F80C0CA7
:109BB00000F44079B9F5807F7047C2EBC202C2F36E
:109BC0004C425A43704741E80002002A704794F81B
:109BD000400001287047C0B21BF8000070474FF4E6
:109BE00000510160201D06F023BFD6E900070146A1
:109BF00009F0BCBC4FF07C5109F0B8BC608D5146F7
:109C00004FF000732085C2B220460097704741464E
:109C100009F000BE044690F83D0000287047384621
:109C200009F0A4BC384609F043BA268500972046BF
:109C30005146FF224FF080737047086840F00100E2
:109C4000086000207047608D41464FF0007320850A
:109C5000C2B22046704700222B4609F015B8A06D0D
:109C600040F2011188430130A0650020704740EAAE
:109C7000080040EA060895F8240058472046314677
:109C800003F0A4BF04F5926184F89504D4F844036A
:109C90007047012001F02ABD394609F0BBBD2046BE
:109CA000FBF780B92046FBF727BA4A46FBF756BFB9
:109CB000002184F83C10012184F83D1070470121F7
:109CC00080F83D1000207047FF224FF08073208500
:109CD000002000907047002184F8541010BD21F43A
:109CE0000851396002217964B9F5807F70470446D4
:109CF000807901287047016851E8021F026821F04D
:109D0000010142E80213002B704796F8950440F0D9
:109D1000200086F89504704740F2FF1004F07CBCE8
:109D2000214609F0C5B94FF40070606470472046C1
:109D3000FBF7E1B93846BDE8F8834B68CA681946B5
:109D400005F0C8BB2068E9B2002243468162204684
:109D50007047416841F480414160704702460B46BC
:109D600008F0EABE2046F7F79BBD21F48851396020
:109D700001217964B9F5807F70470868884620F42E
:109D800000400860204670470220211D84F83D00F5
:109D9000206805F067BB016851E8001F026821F0E8
:109DA000100142E80013002B70470122FCF7B4BDFC
:109DB000504606F8387F04F031B820464146FF226D
:109DC0004FF0807326857047204641463A46FBF7A0
:109DD000E0BE002084F840002046704700200021AB
:109DE000002206F0EBBB116821F0E07121437047BF
:109DF0004AEA084141EA0028A878584716F8011BAA
:109E0000204603F011BF002084F880002046FBF7B5
:109E1000ADBB20464FF4004101221923FBF72ABEB7
:109E2000D4F8400320F00200C4F8400370477047A4
:109E300070470000B0B510B10446407900B1B0BD24
:109E4000D94D05F1540006F0F3FDDB48FFF7EEFABB
:109E5000A079A87094480068BDE8B04000F0ECBA62
:109E6000D5484FF40061F9F797BB00BF01200021EE
:109E700006F002BD704700008B490877704700BFAD
:109E80000248012141770248406900472C02002026
:109E9000C80000202DE9F0410F4F1C4615460E4624
:109EA000804606F017FD3C757D823E82C7E90208B8
:109EB000387840F0110038700848D0F8480310B1E5
:109EC000006900B1804706A3022000210122BDE8FD
:109ED000F04106F073BB00BF880200207C14002014
:109EE0004D4143207278446F6E650D0A00000000FA
:109EF0003748017841F004010170D348D0F8480395
:109F000010B1006900B10047704700BF80B50A4832
:109F1000017841F0020101700848D0F8480310B1FF
:109F2000006900B1804706A3022000210122BDE89C
:109F3000804006F043BB00BF880200207C14002054
:109F40004D414320727854696D654F75740D0A0058
:109F50001CB506F0BFFC0D4C6060684605F0D2F8F9
:109F60000B48DDE90012C0E9CE122178D0F8480391
:109F700041F02001217010B1006900B1804705A3B4
:109F800002200021012206F019FB1CBD88020020DE
:109F90007C1400204D4143207478446F6E650D0A97
:109FA0000000000080B50A48017841F00801017006
:109FB0000848D0F8480310B1006900B1804706A3F3
:109FC000022000210122BDE8804006F0F7BA00BF60
:109FD000880200207C1400204D414320747854698D
:109FE0006D654F75740D0A000A46B149F8F758B906
:109FF000B0B5E64CA34D94F82800A86094F8290069
:10A000004D2804D1A868C0EB001080000DE094F842
:10A010002900482804D1A8684FF46161484304E04E
:10A0200094F82900532801D1A868A860A8680B28D3
:10A030002CBFA8680A20A860A87820B1A8684FF4AF
:10A040007A71484300E0606800F0F6F994F82C005B
:10A05000287094F82D0028710020142806D02218AA
:10A060002918013092F850200A74F6E794F8260077
:10A07000012817D194F82F00032813D194F8300049
:10A080000A4908700A4994F831000870094994F89F
:10A0900032000870084994F833000870BDE8B040F9
:10A0A00003F078BAB0BD00BF0000002064000020BB
:10A0B0006500002066000020B0330020B0B590B0ED
:10A0C0006D46044640212846F7F750FBB049284624
:10A0D000402206F041FB204629464022F7F79DFA30
:10A0E00010B0B0BD10B5D14C04F2044006F0A0FC95
:10A0F00094F81E0410B1012084F81D04D4F848031C
:10A1000020B1006910B1BDE81040004710BD00BF8C
:10A11000F8B5E1B3D64C0E4605464FF40041012296
:10A120002046F9F741FAE24F07F13C0006F04AFCFD
:10A130006DB3307858B3686848B3297802290ED0D7
:10A14000142917D0032922D1697801291FD1007859
:10A15000022822D0012822D0C8B9002020E095F999
:10A160000120D1B2012912D0002A10D4BDE8F84054
:10A1700006F00AB86978012909D100784FF4006126
:10A1800010F001007871204602D1002201E0F8BDF4
:10A190000122BDE8F840F9F707BA022000E00120EB
:10A1A000BDE8F840FCF72AB884030020ED484FF4DE
:10A1B00000410022F9F7F8B90004004810B5D5496C
:10A1C0000020A1F8CA0391F81F0481F8B803D04811
:10A1D00090F8612090F8753090F8804090F81C015C
:10A1E00081F8CC0381F8BB2381F8C83381F8C943D7
:10A1F00001F5607001F56E71BDE8104003F08AB999
:10A20000C44991F89404E8B14FF48070A1F8E203D6
:10A2100091F81F0481F8D003BD48426EC1F8D423E1
:10A2200090F8752081F8E02390F8802090F81C01C8
:10A2300081F8E40381F8E12301F5667001F574719A
:10A2400003F068B9704700BF7C140020B0B598488F
:10A25000C07818B90820002106F00EFBC14C0A4D49
:10A260004FF4004100222046A84720464FF40071D9
:10A270000022A84720464FF4006100222B46BDE88B
:10A28000B040184784030020A935000870B5084E77
:10A290000C4605464FF400613046F7F789FF00B1E0
:10A2A00070BD304629462246BDE87040F8F70EB82A
:10A2B00000F00308B0B590B06D46342105F10C04F0
:10A2C000FFF774F96648202180F82F1090F82420B9
:10A2D0008DF8002090F825208DF8012090F8262098
:10A2E0008DF8022090F827208DF8032090F8282080
:10A2F0008DF8042090F829208DF8052090F82A2068
:10A300008DF8062090F82B208DF8072090F82C204F
:10A310008DF8082090F82D208DF8092090F82E2037
:10A320008DF80B1000218DF80A201C2905D0421849
:10A3300092F8302062540131F7E790F84C10002277
:10A340008DF8281090F84D108DF8291090F84E10C7
:10A350008DF82A1090F84F108DF82B1005F12C0174
:10A36000142A05D0831893F850308B540132F7E744
:10A37000074C4FF400612046F7F71AFF20B96946F1
:10A3800020464022F7F7A2FF10B0B0BD0000002029
:10A3900000F8030880B5FBF7D1FD18B9FBF75EFEA6
:10A3A000012800D080BD06F0A3FB000080B568B195
:10A3B000007858B16B484FF400710122F9F7F4F8B6
:10A3C0003B482430BDE8804006F0FCBA80BD00BFA9
:10A3D000B0B5B34C04F55A7006F02AFBD4F840032C
:10A3E000B04DD4F89C1420F02000C4F84003D5F8F8
:10A3F0008400FCF74FFF28B9012004F0BDF908B133
:10A400000B2800D1B0BD092084F8450495F8390027
:10A4100084F8460494F81C0484F849040920FCF7E5
:10A4200029FCBDE8B04004F0B7BD00BF7C1400209B
:10A430000B49C874704700BFB0B5094D002808BF6C
:10A4400042F2107068601B48FFF7D0F96968204637
:10A4500006F0A0FA2046BDE8B04006F0B3BA00BF4F
:10A46000000000203F484FF400710022F9F79CB82B
:10A470000004004810B50E4C01200021607002203D
:10A4800006F0FAF90B48303006F09CFAA07808B1D3
:10A49000207C00B110BDE068042802D8E0680130DB
:10A4A000E06010200021BDE8104006F0E5B900BFD3
:10A4B00084030020F00300207CB57A4E784D736C45
:10A4C00096F8482096F9701096F8400005F57A74D1
:10A4D000009402F021FF40F2012096F81C1105F5CE
:10A4E0008562A5F8FA0396F8400085F8FC1321462A
:10A4F00002F052FF58B195F8280485F86E0406481A
:10A50000416B0020884795F8FB0385F894047CBDD7
:10A510007C8500207C140020C43A0108704780B577
:10A52000FAF752FC00200121BDE88040F9F7AABBF0
:10A5300010B50C4C4FF6FF7100222046F9F734F8A5
:10A5400004F580604FF6FF710022F9F72DF8FAF755
:10A550003BFC0548012101600120BDE81040F9F7EE
:10A560006FBB00BF00040048880400587047FAF72A
:10A5700027BA000080B5FAF723FA08F0F9F9FEF7D8
:10A5800079FDFEF7F1FD0448F9F76EF80348BDE8E0
:10A590008040FAF771BC00BF784C0020204D0020AD
:10A5A0002DE9F04F89B0002853D08A460646DDE9F0
:10A5B000121000244FF001089146CDF80D4004948C
:10A5C000CDF80940CDE90744CDE90544CDF8054073
:10A5D0008DF804808DF80A308DF80910010E8DF881
:10A5E0000E008DF81110010C000A8DF80F00180EE6
:10A5F0008DF810108DF80D00180C8DF80C00180A4D
:10A600008DF80B0005AF0FFA8AFBBBF1010F22DBBF
:10A610008DF8138001A810214A463B4604F00EFA3B
:10A62000D8B9BBF1100F4FF01000A8BF834608F156
:10A630000108E0B20021CAB2934506DDBB5C0244CA
:10A640000131B55C6B40B354F5E71034AAF1100A40
:10A65000D9E7092002E0002000E00E2009B0BDE8A3
:10A66000F08F704710B50E4CD4F8400340F08000D6
:10A67000C4F8400394F81E0410B10020FFF732FD27
:10A6800094F8950440F0220084F89504054890F869
:10A690000401022818BF062084F8940410BD00BFEE
:10A6A0007C1400207C8500202DE9F04F93B012A986
:10A6B000044604F025FA002848D1042C07D825A325
:10A6C000DFE804F00E03090B0D0040A308E07F2C27
:10A6D0000BD126A304E031A302E036A300E029A3B6
:10A6E00002200021002205F069FF1298817990F87C
:10A6F00001E090F8028090F8039090F804A090F8A0
:10A7000005B090F808C0827AC37A047B457B867BCB
:10A71000C77B1191C1791091417A007C09920A930B
:10A720000B940C950D960E972E4B002208910F90CE
:10A73000CDE900E802A8002180E8000E11980590FC
:10A740001098CDE9060C022005F038FF13B0BDE8E3
:10A75000F08F00BF232323232323204170704B65F8
:10A76000793A2020202020200000000023232323EA
:10A770002323204D434B454B65793A202020202050
:10A7800000000000232323232323204D43526F6F17
:10A79000744B65793A2020200000000023232323F6
:10A7A0002323204E776B534B65793A2020202020BD
:10A7B0000000000023232323232320417070534BE8
:10A7C00065793A2020202020000000002323232345
:10A7D0002323204E776B4B65793A202020202020C0
:10A7E00000000000E59401082DE9F04F93B000252A
:10A7F000012B8DF84B50ADF8485000F2848283460F
:10A8000002F03F00DFF81095884605260DF14B0752
:10A810000024079000200890A246E4B2444580F04E
:10A8200072821BF80400FCF7C1F82044404500F296
:10A830006A821BF804000238112800F264820AF1CF
:10A840000104DFE810F012009200A100AF00E70061
:10A85000F30024012B007000600260023A016002E4
:10A8600060028E01A301B701D5010420FCF7CAF9EB
:10A870000028D1D000200421FCF7ECF9E0B2DFF889
:10A8800090140AF103041BF8000081F860040AF137
:10A890000200FFF7A0F981F86104BDE7E0B28DF88E
:10A8A0002C501BF80000C0F340118DF82D10C1068C
:10A8B00002D501218DF82C1000F00F000AF10204DE
:10A8C0008DF82E0099F840000BA902F07FFD0130B1
:10A8D000A2D09DF82D009DF82E109DF82C5089F8DF
:10A8E00075000FF2384089F87450405C08F0C2FDE2
:10A8F000C9F8780002208DF83A5000258DF838000C
:10A9000099F840000EA902F017FD99F9391040B2EC
:10A910008842B8BF084689F8390012A909200022E8
:10A92000FBF7FAFF78E703200AF102018DF84B00EC
:10A93000E0B2FFF733F88DF838000AF10300C0B237
:10A940001BF80000FEF712FE0F9099F840000EA9C8
:10A9500002F0ECFC0AF1050400288DF84B003FF5ED
:10A960005BAF8DF848000A208DE008988DF82C50D8
:10A970008DF837508DF836508DF83550C00700F0FF
:10A9800051810AF10504BBE1E0B201211BF800008E
:10A9900000F00F0089F8070101FA00F0A9F80C0196
:10A9A000042083E007208DF84B00E0B21BF8000084
:10A9B000C0F3021100F00F008DF839100AF1020106
:10A9C0008DF838000AF10300C0B2FEF7E7FFFEF78A
:10A9D000CDFD0F9099F840000EA902F0E4FC00F0C4
:10A9E00007010AF105048DF84B0007290ED19DF8E7
:10A9F00038109DF8392089F8701089F868100F997F
:10AA000089F86120C9F86C10C9F864108DF8480005
:10AA1000052038E0BE48D0F84803002800F0F68052
:10AA20000168002900F0F2808847F0E003200AF175
:10AA300002018DF84B000EA8C9B20F950B90E0B241
:10AA40001BF801101BF800008DF830000AF105001A
:10AA5000FFF7C1F88DF840000AF10300C0B21BF8FF
:10AA60000000FEF783FD0E9099F840000BA902F05C
:10AA700082FC0AF1060400288DF84B003FF5CCAEAD
:10AA80008DF84800072012A9FFF78FF9C4E6E0B25D
:10AA90004FF47A721BF8000010F00F0008BF01306D
:10AAA00010FB02215043C9E91401082012A9002219
:10AAB000FBF732FF0AF10204AEE60920FCF7A2F828
:10AAC000002800F0138100200921FCF7C3F80AF1E7
:10AAD0000500FFF780F806900AF10400FFF77BF805
:10AAE00003900AF10300FFF776F80290E0B21BF83A
:10AAF00000400AF10200C0B21BF800500EA804F09A
:10AB000001FB0E980299069A05900F9804908048D0
:10AB1000D0E9CE30009044EA0520002540EA01400B
:10AB2000039940EA01607B4901444FF47A70504335
:10AB3000020A09A804F032FBDDE9093000900EA8F2
:10AB4000DDE9042104F0B0FADDE90E0104F006FBB2
:10AB5000FBF7BFFE6E4901200AF1060481F83C04B0
:10AB60005AE60C20FCF74EF800283FF455AE0020C2
:10AB70000C21FCF76FF8664890F8940400F0FE0092
:10AB800004283FF449AEFBF7B8FE45E6FEF76CFD3E
:10AB900041430AF10400FFF71EF800F00F00FBF735
:10ABA000AAFE8DF84800112012A9FFF7FEF80AF15D
:10ABB000050431E60D20FCF725F800283FF42CAE03
:10ABC00000200D21FCF746F80AF10201E0B24F4ADD
:10ABD000FEF7E4FE926840EA01200AF10301C9B2DF
:10ABE00080B21BF80110FBF773FE0AF1040413E6B0
:10ABF000FEF73AFD4843FBF768FE8DF84800132046
:10AC000012A9FFF7D2F80AF1040405E6FF2007991C
:10AC10008DF84800062002228DF8491012A9FBF792
:10AC20007BFEF9E54FF0FF3A99F8382099F80611C4
:10AC300099F8393099F8740099F860508DF84420EB
:10AC4000D9F818218DF8421000298DF843300DF104
:10AC500036018DF8410099F840008DF845500E926C
:10AC60005AFA84F20BEB0203A8EB02020F9308BF1F
:10AC7000052200910DF135018DF840200DF13703CB
:10AC800001910EA90BAA02F06AFB8DF84B0000F0AF
:10AC90000700072812D199F939109DF92C00884234
:10ACA00002DD012189F8091189F839009DF8370082
:10ACB00089F838009DF8360089F8600000259DF875
:10ACC0003500EAB2B0FBF6F1914205D903203946CE
:10ACD000FFF76BF80135F2E70444601EC1B241454D
:10ACE00008D21BF8010003289ED004E0084880F831
:10ACF0003C5491E50446E0B2404538BF013C002594
:10AD00000120089088E513B0BDE8F08F880200208C
:10AD10007C140020803DD5127C850020080A0C0D93
:10AD20000E10121415181A1B1D1E212410B51448DC
:10AD3000007808B1F7F756F91248006808F09AFB56
:10AD4000114C214608F012FC08F05CFB0F4908602A
:10AD50000F48006808F08EFB214608F007FC08F059
:10AD600051FB0C4908600C48006808F083FB214641
:10AD700008F0FCFB08F046FB0849086010BD00BF66
:10AD8000B0330020A433002000007A40DC01002012
:10AD9000A8330020D8010020AC330020D4010020CB
:10ADA000032816D8B0B5C5004FF48070274C4FF477
:10ADB0008071E840C2B22046F8F7F6FB06484FF42F
:10ADC0000051E840C2B204F58060F8F7EDFBBDE841
:10ADD000B0400020704700BF00000101162100288C
:10ADE00008BF0F21084670470220704770B586B033
:10ADF000002402200594FAF71FFF0420FAF71CFF35
:10AE00000320CDE903400120104C02904FF48070E4
:10AE1000019001AD20462946F8F7FAFA4FF40050A8
:10AE200004F58066294601903046F8F7F1FA30467D
:10AE30004FF400510022F8F7B7FB20464FF4807121
:10AE40000022F8F7B1FB002006B070BD00040048F6
:10AE5000012070470020704770B53C21234A01EA69
:10AE60009000204908582049096801F00F0152F864
:10AE70002110B0FBF1F01E49B0FBF1F4F8F7F4FE3D
:10AE8000B0F5007F09D11D49002003280FD031F80B
:10AE9000102094420DD90130F7E71649002003280D
:10AEA00005D031F81020944203D90130F7E700258E
:10AEB00002E0114951F82050114E306820F007008F
:10AEC0002843FEF77CFB0446306800F00700A842E8
:10AED00006D0F8F76FFB001B0328F5D3032070BDE5
:10AEE000002070BD843A0108080100584839010863
:10AEF00040420F001E3901082439010818390108A1
:10AF00000040005870477047FEF73FBB0020704775
:10AF100000207047FEF739BBFEF737BB704770471C
:10AF20007047FEF732BBFEF730BB00000148F9F76F
:10AF3000EBBB00BFDC4C00200928014698BF09216B
:10AF4000CAB20A23B2FBF3F202EB8203A1EB430382
:10AF5000591A084440EA0210C0B270472DE9F04186
:10AF6000114E80463068400619D43068002701240D
:10AF700040F080003060F8F71DFB05463068E14383
:10AF800041EA9010C0070BD1F8F714FB401BB0F555
:10AF90007A7FF3D90327002488F82D70EEE7002785
:10AFA000F8B2BDE8F08100BF0C280040B0B5124DEA
:10AFB000044655F80C0C20F0800045F80C0C28686D
:10AFC000800606D4F9F7E4FC70B1032084F82D0064
:10AFD000B0BD286820F020002860F9F7D9FC28B11E
:10AFE000032084F82D0002E00020B0BD0020296875
:10AFF00041F020012960B0BD1828004001207047B1
:10B0000080B502F01DFF0438C0B2032805D80449FA
:10B01000C00021FA00F0C0B280BD002080BD00BF9A
:10B020000201000380B502F05FFF033080BD000025
:10B03000F8B5F94EEA4F00253446BD65C7E901551C
:10B040007D7001C4184802F0ABFFBD8103F05DF9CB
:10B050000020002103F015F801200021042203F054
:10B0600065FA4FF6FF704FF6FF71FEF714FB00F024
:10B07000F9FF0E4B20464FF0FF310022009505F0FE
:10B080000FFC009506F11C05094B4FF0FF31002223
:10B09000284605F005FC204605F0CAFC2846BDE818
:10B0A000F84005F0C5BC00BFD5B30008FDB30008EB
:10B0B000E5B300087CB58D4C00208DF807000090AA
:10B0C000B4F85400411E072927D9102800F0B08099
:10B0D000202800F0AF80402800F0BE80802800F0DB
:10B0E000C780B0F5807F00F0CC80B0F5007F40F0E5
:10B0F000E68091A3FEF74CFA02F0A2FE042840F08D
:10B10000CA80C4487E4CFEF76AFDFEF7B4FB206897
:10B11000002800F0D4804068CFE0DFE801F004169A
:10B12000D052D0D0D07FBB48754CFEF758FDFEF70B
:10B13000A2FBFFF7EDFE012808BFFFF7E4FE206841
:10B14000002800F0BC800068B7E0B2486C4D4FF4B6
:10B150008051016005F11C0005F06AFC607880B93F
:10B16000FEF789FB40F60210002103F08DFA40F64D
:10B17000441002F061FF40F0020140F6441003F079
:10B1800083FA72480DF10701FF2202F095FE04F1E7
:10B19000240002F059FE2868002800F0908086689C
:10B1A000002E00F08C8094F82400012840F0888064
:10B1B00094F9313094F930209DF807106348B04776
:10B1C0007CBD59A3022000210122002505F0F6F9DB
:10B1D000A06D002873D0574EC0F3074140F603100E
:10B1E000B04794F8591040F60410B04794F858103E
:10B1F00040F60510B04740F6021002F01DFF40F087
:10B20000010140F60210B04740F2622040F2622194
:10B2100000220023A56502F06BFF7CBD3FA3FEF773
:10B22000B7F9FFF773FE012849D1FFF777FE7CBD20
:10B2300037A30EE0324D05F11C0005F0F9FB6078F4
:10B2400008B9FEF718FB2868C8B3C068B8B38047D0
:10B250002CA3FEF79DF97CBD25A3FEF799F9607834
:10B2600008B9FEF708FB2648006840B3006924E0EF
:10B27000FEF701FB2248006808B38169F9B100209C
:10B2800007E0FEF7F8FA1E480068C0B18169B1B165
:10B29000012088477CBD02F0D3FD05280FD15D4811
:10B2A000174C4FF48051016004F11C0005F0C0FB05
:10B2B000FEF7E1FA206810B1C06800B180477CBD9C
:10B2C000E06B694602F06CFD00984FF47A7194F9D6
:10B2D000292000F5FA7090FBF1F09DF8071043B2B9
:10B2E00028688468EE48A0477CBD00BF3C1B002056
:10B2F0004952515F4352435F4552524F520D0A002B
:10B30000AC020020484452204B4F0D0A00000000C0
:10B31000484452204F4B0D0A0000000053594E4341
:10B32000204F4B0D0A000000505245204F4B0D0A94
:10B330000000000089E600084952515F52585F54EE
:10B34000585F54494D454F55540D0A009F19002030
:10B350002DE9F0418AB01C4615468846074600F0A4
:10B360008AFE0020002600F0C1F9384602F0DEFF18
:10B37000012041464FF416720023CDE908600320F6
:10B38000CDE900800020CDE90266CDE90466CDE973
:10B39000066600F0F3F9002000F052F8FFF742FED5
:10B3A000F7F7E9FE05F096FA0646304605F09CFAF6
:10B3B0000746A04203D202F0CBFDA842F5DD0025EE
:10B3C000A74228BF012500F056FE28460AB0BDE876
:10B3D000F0810000E849A1F85400FFF76BBE00BF00
:10B3E0003C1B00200B484FF480510160B4480068BA
:10B3F00010B1C06800B10047704700BF05484FF466
:10B4000000510160AE48006810B1406800B10047CB
:10B41000704700BF28040048AC02002080B500201F
:10B420000021FEF738F9BDE8804002F05FBD02F070
:10B4300003BE02F00DBE80B502F08AFD80BD0000A3
:10B44000B0B50446FFF762FD012802D1FFF762FDA7
:10B4500005E040F2622040F26221FEF71CF92CB1B7
:10B460009748FEF742FB284605F0ACFA8A484FF4AD
:10B470008051C14CFEF798FA61786FF07F40A26866
:10B48000002908BF9001BDE8B04002F07FBF00BFB7
:10B49000B0B50446FFF73AFD012802D1FFF73AFDA7
:10B4A00005E040F2622040F26221FEF7F4F82CB190
:10B4B0008348FEF71AFB284605F084FA76484FF4D5
:10B4C0008051AD4CFEF770FA61786FF07F40A26852
:10B4D000002908BF9001BDE8B04002F06BBF00BF7B
:10B4E0002DE9F84F8B46814640F2012040F20121C0
:10B4F000FEF7D1F868484FF40051DFF8A0810160F1
:10B50000012198F8560002F0BEFF98F8000098F864
:10B51000511081F0060180F0010050EA010640F66A
:10B52000890018BF012602F087FD00F0FB0040EA09
:10B53000860140F6890003F0A7F898F80000042877
:10B5400000F29180DFE800F0031503181F00FFF7F9
:10B55000DDFC012824D10DF1030248465946FFF7CE
:10B56000E0FC002800F08B804FA3FEF711F8BDE847
:10B57000F88F88F81FB015E00221404600F80E1F32
:10B5800080F80CB010E0464800215A464B468AB17C
:10B590001E78013AF64303F8016B00F8011BF6E749
:10B5A00088F816B008F10E0002F042FE48465946EF
:10B5B000002256E03A4E4FEACB0700200721002236
:10B5C000974215D0C2F3C70421EA0203013219F8E9
:10B5D000044024FA03F321EA020403F00103584073
:10B5E000C3B2A340C2F3C704355D2B433355E7E72D
:10B5F000C10145460BF1010941EA8011C0B2B0FA20
:10B6000080F0400941EA401006F80B00022005F8DE
:10B610000E0F284685F80C9002F00AFEDFF884A091
:10B62000F1200021D047F0200021D047D5F83A4042
:10B63000E121642C08BF7021F320D0470421642C41
:10B6400008BF1D21F220D0474FEA5B11F420D047FC
:10B65000B81CC1B2F520D0475FFA89F130466FF0CF
:10B660007F4202F005FD1648D8F80410041D20465C
:10B6700005F090F9204605F0A5F9BDE8F88F9DF892
:10B68000030088F8160008F10E0002F0D1FD9DF8C5
:10B69000031048468CE700BF180400483C1B0020FC
:10B6A0009F19002089E60008526164696F53656E36
:10B6B00064204F76657273697A650D0A0000000098
:10B6C000AC02002002F032BE012802D1DA48C17774
:10B6D00005E0D948427D012A18BF70478175C548E9
:10B6E0000170D5480E3002F0A3BD00BFB0B5D24DF9
:10B6F00004462870FFF714FC052C14D8DFE804F08A
:10B70000050B1303030502200EE00020002402F0C5
:10B71000E3FD6C7306E0012002F0DEFD287B697B0F
:10B72000814206D1B0BD032002F0D6FD002068732F
:10B73000B0BD6873002818BF0120BDE8B04000F01C
:10B7400001B800BF10B50446BB4844730473FEF74C
:10B75000A0FA14214FF4E860002C18BF342102F045
:10B7600093FF242140F24170002C18BF4421BDE812
:10B77000104002F089BF00BF3C1B00202DE9F04FB4
:10B7800085B0DDE91185DFF87CBA179C1F4691462C
:10B790008A4606468BF80140B8F1000F08BF4FF00B
:10B7A000FF35FFF7AFFB9349002C10980F9C0D70ED
:10B7B00018BF0020002E6AD0012E00F0B080052EA8
:10B7C00040F0148100900120884602F053FE0920C9
:10B7D00000275E468BF844004FF44870CBE90F9089
:10B7E000FEF7E6FA5D4605F80E7F85F837004FF460
:10B7F00080506860E00068800120A5F8090098F892
:10B80000000028720520FFF771FF304602F0A8FC07
:10B81000284602F00DFD42F2B270CDF80E70ADF880
:10B820001270ADF80C0003A802F043FEFEF774FAA4
:10B83000724E40F6B800B047714D00F0EF0140F68F
:10B84000B800A84740F6B9000421A84740F69B007D
:10B85000B04700F0E30000F1080140F69B00A84764
:10B8600040F2D160B04740F0180140F2D160A847E3
:10B8700040F2AC60B04700F08F0000F1500140F2A0
:10B88000AC60A84700994FF4FA50484344E004469E
:10B890000020002702F0EEFD0B205E46CBF83C9026
:10B8A0008BF84400FEF784FA5D46139905F80E7F85
:10B8B00085F8370088F00100AF71E87141F60400A7
:10B8C000A8800F98C00068800120A872002918BFC6
:10B8D0006FF00D00687247480078287200F0CBFBCB
:10B8E0000020FFF703FF304602F03AFC284602F042
:10B8F0009FFCC120CDF807708DF80B708DF8060005
:10B9000049F2C140ADF8040001A802F0D2FDFEF7F3
:10B9100003FA4FF4FA506043B0FBF9F064E0009092
:10B9200000205D464FF0000B02F0A4FD32490120DB
:10B930002E4622468AF0010306F8380F0C2C11F827
:10B940000A10B77686F8189006F81A8C71766FF0A0
:10B95000040198BF0C2251FA89F10229169928BFD7
:10B96000224626F81C2C344689F00C0206F8171CD7
:10B97000139906F8181C1F49097806F8191CA9F133
:10B980000B01022938BF4FF0010BBAFA8AF104F813
:10B990002A0D1A434909B2FA82F201EA0B01AB46B9
:10B9A00052091143F17600F066FBFEF772F930465A
:10B9B00002F0D6FB204602F03BFC0098C0B202F039
:10B9C000B2FB16F8170C441E40F2367018BF012463
:10B9D00002F032FB00F0FB0040EA840140F23670D6
:10B9E00002F052FE4FF6FF70CBF8080005B0BDE83C
:10B9F000F08F00BF54010020A839010839E0000889
:10BA000089E6000870B5EB4E054601EB40000C4698
:10BA10004FF6FF7100220023B0654FF6FF7002F071
:10BA200067FB96F85600002102F02DFD28462146BE
:10BA3000BDE8704002F0D8BC3C1B00202DE9F0436B
:10BA400087B000279846154689460646CDE9047713
:10BA5000FFF758FAD74C002D18BF0125657018BFA5
:10BA6000B846012E40D0002E40F0B880D9F808002A
:10BA7000002800F0B180D9F80C00002800F0AC805C
:10BA800099F81E20082A00F2A780D9F8101004A8FF
:10BA900004F062FED9F80000002818BF012002F06F
:10BAA000E9FC002584F83850D9E90101E16399F8EF
:10BAB000201084F8441002F0B1F984F84500A57311
:10BAC00099F81F2099F8213099F81E1099F8220052
:10BAD000A2742375C900B9F80C20E174D2000028C3
:10BAE00022825CD0FF215CE0B9F83000002873D0DE
:10BAF00099F8320001280CBFD9F81450FF25D9F865
:10BB00002800002818BF012002F0B4FC5FFA88F07A
:10BB100002F009FB012084F8380099F82C1099F8FC
:10BB20002F0084F850100228B9F82D20A4F85120D5
:10BB300005D306D10B390020022938BF012084F833
:10BB40005300012004F80E0FB9F830006574E0814D
:10BB500099F832002074B9F83400608200F08BFA52
:10BB6000FEF797F804F12A0002F0FAFA204602F0F4
:10BB70005FFBE07C451E40F2367018BF012502F0E5
:10BB80005BFA00F0FB0040EA850140F2367002F0FB
:10BB90007BFD4FF6FF70002744F8060C1EE0D9F835
:10BBA0001410A17599F82410022918BF022819D180
:10BBB00099F82300A0F1F101022901D301280BD14A
:10BBC0008D4A0025CDF808908DF80C5052F81C1BBA
:10BBD00001A8FFF799F958B14FF0FF37384607B081
:10BBE000BDE8F083607599F823002176E07503E0E5
:10BBF00001206575A4F8170000F03DFA0020002729
:10BC0000FFF774FD04F1380002F0AAFA04F10E0007
:10BC100002F00EFB04A802F04CFCB9F81C0002F084
:10BC2000FBFCB9F8180002F043FA4FF4FA50D9F8C7
:10BC3000081008FB00F0B0FBF1F0A060CEE700BFF9
:10BC40002DE9FE4F1D46174688460446FFF75AF970
:10BC5000149EDDF830A0042C4DD0DDF84090DDE9D5
:10BC60000EB3012C55D0002C40F09980FB4E0B20D8
:10BC700086F844002846C6F83CA04FF0000A344637
:10BC80001D4604F838AF02F0C9F806F80EAF86F882
:10BC900037000120C6F83270B072B9F1000F18BF3A
:10BCA0006FF00D00707286F806A085F00100F0714B
:10BCB00041F60400B0804FEACB00708000F0DBF961
:10BCC0000020FFF713FD204602F04AFA3046149E8A
:10BCD00002F0AEFAC120CDF807A08DF80BA08DF8C8
:10BCE000060049F2C140ADF8040001A802F0E1FBF2
:10BCF000FEF712F853E00420FFF7F8FCE8480221B1
:10BD000000F8381F16210175C0F810A002F028FABB
:10BD100045E03746E24E012013990D9ABBF10C0F16
:10BD200006F80E0F86F84420234AF1742349337431
:10BD300086F842A086F8129085F001033446525DE1
:10BD4000097886F8432071746FF004015A4651FA5D
:10BD50008AF198BF0C22022928BF5A46F281AAF123
:10BD60000B0100220229B5FA85F138BF012204F83F
:10BD70002A0F490911408AF00C021A43B2FA82F2E2
:10BD80005209114386F8451000F075F9FDF781FF5F
:10BD9000204602F0E5F930463E4602F049FA4046B8
:10BDA00002F0E0FABE4C84F85600FFF7B8F866607F
:10BDB000BDE8FE8F3C1B0020A8390108540100207B
:10BDC000B0B514460D4602F0B1FA284602F0CAFAA0
:10BDD000012102F058FB4FF47A70444302F09CFBBF
:10BDE0009F482146051D284604F0D4FD2846BDE89D
:10BDF000B04004F0E7BD00BFAC0200202DE9F043E5
:10BE000087B0074600201C4615460E46CDE90400C3
:10BE1000FFF778F8032F00F21481DFE807F0024300
:10BE200084983068002800F0DF80B27C082A00F295
:10BE3000DB80B16804A804F08FFCF24F00200422DC
:10BE400087F838003168B873F963F17C87F84410DB
:10BE5000B1693964B188BA74C9003982B17C387566
:10BE6000C800F874B07D022803D0307D022840F06D
:10BE7000BE80707DA0F1F101022902D3012840F0BB
:10BE8000B380774A4FF0010801968DF80C8002CA02
:10BE900001A8FFF739F8002840F0A680A7F817801E
:10BEA0000020A9E0D74F012087F83800307887F8C4
:10BEB0005000707887F85100B07887F85200F07819
:10BEC000022807D308D13078A0F10B010020022905
:10BED00038BF012087F85300012007F80E0FB08803
:10BEE000F881B0793874F079B874307AF87400F069
:10BEF000C2F8FDF7CEFE07F12A0002F031F938460C
:10BF000002F096F997F8436040F6890002F094F841
:10BF1000062E0CBF00F0FB0140F0040140F6890042
:10BF200002F0B2FB8DE0306800285DD0B0F57A7F7A
:10BF30005AD80320FFF7DAFBB2480221162200F894
:10BF4000381F31680275016102F00AF979E0B27CAC
:10BF5000082A49D8B16804A804F0FEFB306800281C
:10BF600042D042F2107188420CD8A64803214FF00B
:10BF7000020880F8381081733168C163F17C80F861
:10BF800044100EE09F484FF0000880F8388080F899
:10BF90000E803168C163F17C80F8441031688908F3
:10BFA0000164B088974F0421B974C0000021388221
:10BFB000B07C3975C000F874B07D022802D0307DA5
:10BFC00002281ED1707DA0F1F101022901D30128C0
:10BFD0000AD1234A4FF0010901968DF80C9002CA4C
:10BFE00001A8FEF791FF90B14FF0FF3033E0707D74
:10BFF000F875B07D3876307D787500F03CF800201B
:10C000000CE0707DF875B07D3876307D02E0A7F8E1
:10C0100017900020787500F02EF84046FFF766FB79
:10C0200007F1380002F09CF807F10E0002F000F969
:10C0300004A802F03EFA308A02F0EEFAB08902F06B
:10C0400037F8284602F08EF96E4D85F85600FEF757
:10C0500066FF6C60002007B0BDE8F0833C1B002049
:10C06000AC02002080B5042002F0DAF90220BDE81D
:10C070008040F7F780B8002002F0E8B980B5614849
:10C08000002190F8560002F0FEF94FF4C0704FF412
:10C09000C071FDF700FBBDE8804001F0FFBF00BFAD
:10C0A0003C1B0020F0B50DF1140C089E01289CE803
:10C0B000901010D000285FD10CEB0400002E18BFA8
:10C0C00002302021002F18BF182101EBC0004FF4CF
:10C0D0007A71484352E019B9A2F10B00022804D347
:10C0E0000020012908BF0C2A00D101201425002FAF
:10C0F00018BF0025A5EB8205002E6FF0070618BFBC
:10C100001035072A05EBCC0528BF08359700002815
:10C1100018BF06EB82070C26072A38BF970038465F
:10C12000002DC8BF284401380C250C2C90FBF7F0DB
:10C1300088BF2646571F022F28BF2646072A38BF2A
:10C140000E25AC190433023A00FB03408000013095
:10C1500090404FF47A725043174A515C00220A29EA
:10C160000CD8DFE801F006101316191B1D0B1F2257
:10C17000250041F6846201E00122002010440138CC
:10C18000B0FBF2F0F0BD43F60952F7E747F6122292
:10C19000F4E74FF22442F1E70A4AEFE7084AEDE7F5
:10C1A000064AEBE742F6B102E8E745F26112E5E73D
:10C1B0004AF2C322E2E700BFA839010820A1070024
:10C1C00090D0030048E8010080B502F0CBF80121CF
:10C1D00002F059F9BDE8804002F09EB980B50948E7
:10C1E000012190F8560002F04EF94FF4D7602D214E
:10C1F00002F04AFA02F095F90348BDE8804002F0E7
:10C2000075B900BF3C1B0020FFFF0F0002F03CBAD5
:10C2100002F046BA10B50446FEF71AFE012818BF10
:10C2200010BD40F6231001F007FF00F0F90040EACE
:10C23000040140F62310BDE8104002F025BA0220A8
:10C2400070472DE9F04F87B0044650208DF8180054
:10C25000207A102802D16068C07B10B107B0BDE819
:10C26000F08F022700254FF064090DF1100A0DF13F
:10C2700008080DF1040B00260F2FEFD8072F17D257
:10C280006068815D30440491427841EA0221049162
:10C290008078059541EA004000FB09F1049158B10E
:10C2A00040468DF80C70CDF808A000F06FF808E05B
:10C2B0008DF81850CDE9045558468DF8047000F0FB
:10C2C000B9F801370336D7E710B514A403A3002843
:10C2D00008BF1C4604EBC100805C10BD00000000DC
:10C2E0000000010201000000000002030201000042
:10C2F000000003040302010000000405040302011E
:10C3000000000506050403020100060706050403F4
:10C3100002010707070605040302070702020202DB
:10C3200002020202020202020202020302020202EC
:10C3300002020304030202020202040504030202D1
:10C3400002020506050403020202060706050403AD
:10C3500002020707070605040302070710B5017963
:10C36000012905D079B9DD49096801F5587203E062
:10C37000DA49096801F55B7201681046012201245F
:10C3800000F09AFC00E00024204610BDF8B50579C5
:10C39000022D01D20620F8BD0F2D01D90320F8BDD2
:10C3A00004460068002107220026007A40F30300BB
:10C3B00000F0AAFFB0FA80F00021072247092068A8
:10C3C00090F90800001100F09FFF2168B0FA80F09A
:10C3D000400991F90820384342F30303B3EB221FCD
:10C3E000C8BF01260643086804F058FB0146062032
:10C3F000002918BF0520002E04BF05200420C6B95F
:10C4000091F0010115D1B54F05EB450621680C22CD
:10C41000386800EB860005F078FF3968002001EBF2
:10C420008602B1F8603350720122AA401A43A1F883
:10C430006023F8BD0178022901D200207047A74887
:10C4400001EB41020023006840F8223000EB820239
:10C4500000F5587013815360102200F010BC00BF2B
:10C46000FEB57B4F0D460728A8BF07201E46144681
:10C470005870394600F02AFD96F90110B07007296E
:10C4800003D1322000F089FC05E07048405C57F889
:10C49000211000F087FC07460748C06D804703461F
:10C4A00006F10C0006F108012246CDE900103846DD
:10C4B000294600F041FCFEBDC43A0108B0B504466F
:10C4C000406804F0EBFA0146DC480268207800EB93
:10C4D0004003022052F82350002918BF0320002DEA
:10C4E00008BF00F00100032803D102EB830162685A
:10C4F0004A60B0BDF8B501460078421E0020372AD8
:10C5000000F29780DFE802F022249595951C95951E
:10C5100095952A2C2E34953B3E4144474A95521C12
:10C5200054595E60639565686A959595959595955E
:10C530009595959595951E842095951E2095878BAC
:10C54000022076E0664874E0032072E0C87800E0DC
:10C550008878002818BF012040006AE0402068E089
:10C56000202066E091F90100897831B936495FE011
:10C5700091F901008978002959D0314958E040F6F5
:10C58000B83056E04FF47A7053E04FF4FA6050E060
:10C5900041F288304DE041F270704AE027484FF494
:10C5A0007A7105F03DFF00F5FA6042E04D4840E049
:10C5B000EF48006800F558703BE0ED48006800F572
:10C5C0005B7036E0102034E0E948006831E001207B
:10C5D0002FE04FF083402CE017482AE007208DF829
:10C5E000050010208DF80700487889788DF8040040
:10C5F000DF4800290068039000F55870029018BFCA
:10C60000012148008DF8060001A800F06FFC10E041
:10C6100040F211100DE091F901000C4908E091F988
:10C6200001000B4904B0BDE8804000F04FBC054953
:10C63000085C04B080BD00BF9A99094018FCFFFF58
:10C64000689101087091010860910108CC390108D6
:10C65000AC39010870B586B01F4991E87C00496982
:10C660008DE87C000591017B02291DD0012925D090
:10C6700081BB016871B3416861B3FA4C80681822CC
:10C68000C4E90010694605F040FE21680320144B00
:10C690000022A1F86C0350208882C1E9033208818E
:10C6A0001048C1E900020EE0EE480068B0F86C13D3
:10C6B000B0F860231143A0F860130BE0E94801686B
:10C6C00000200861486001F5587001F55B71012296
:10C6D00000F0F2FA06B070BD303901088002002087
:10C6E00040F7093700EA06372DE9F04F8FB00025F3
:10C6F000DFF8F094CDE901238B4607464FF0070A97
:10C700004FF00108ADF838500D95ADF832500DAC32
:10C71000387AE9B2814239D27868214650FA85F0F8
:10C7200000F09BFC90B3BDF8381005449DF837002D
:10C730004FF0060A51EA0002ADF83210E8D0421E6E
:10C740004FF0060A052AE3D34FF0060A0628DFD881
:10C75000D9F800204FF0070A0023102BD8D0062864
:10C7600008D116687EB108FA03F6B6B23143ADF8C7
:10C77000321008E021FA03F6F60704D01668002EFE
:10C7800008BF2AF0010A0C320133E6E702208DF8D7
:10C790002C00787A8DF82E000BA8FFF7ABFE8DF8F1
:10C7A00020000DF1320007218DF810A0A21C2346B5
:10C7B000079010208DF82110ADF82810F97A8DF827
:10C7C0001800B87A8DF81510611C8DF81100BDF8AD
:10C7D0003500ADF812009DF834008DF81400B889CA
:10C7E000ADF81600D9F8000009903868039003A846
:10C7F00000F0E2FB044607280DD1D9F80000002123
:10C800000C2200F5587005F094FDD9F80000BDF831
:10C810003210A0F860139DF835109DF836209DF871
:10C8200034008BF8001001990A700299087018986A
:10C83000057020460FB0BDE8F08F00BF80020020D9
:10C84000F8B501680A6892B1007902918DF80C0080
:10C8500002A8FFF79BFD062807D801460320DFE862
:10C8600001F0130404041012040000200CE000790D
:10C870008DF8040001A8FFF7DDFD002818BF032094
:10C8800002E0022000E0012004B080BD2DE9F04369
:10C8900097B007460020D34C164688460021012257
:10C8A00099460125CDE914008DF85B008DF85A00FA
:10C8B000CDE912000320ADF80E00206800F5587095
:10C8C00000F08AFA216828B9B1F8600340F003004B
:10C8D000A1F860030DF10E008DF831500990102081
:10C8E000ADF82000D7E90302CDE90D026268787A3D
:10C8F00007928DF8100097F908008DF81100D7E91C
:10C900000023069101F558710591CDE90A23397D7F
:10C91000BA7A8DF83C10F98A8DF83020F5F7AEFE22
:10C9200004A90DF15B03CDE910010DF15A00494650
:10C93000CDE900060AA812AE324600F0F3FA054629
:10C940000C280AD085B99DF85B00411E002005F037
:10C9500067FD305C88F8000006E02068B0F86013DE
:10C9600041F00301A0F86013284617B0BDE8F0833A
:10C97000800200202DE9F04F8BB0DFF8D0AB0646E7
:10C98000D0F804B090F901708846DAF804008047C6
:10C99000054600285FD1F07C5FFA87F960B99148BD
:10C9A0003178006801EB410150F821B000EB8100C3
:10C9B0004068002818BF8346DAF80C10DAF81840EF
:10C9C000584688478948B9F1070FC25719D1B17C39
:10C9D000A446308900240023CDE908410121CDE996
:10C9E0000644CDE90441CDE9020405204CF2503162
:10C9F00001901D4800904FF47A7042430020E047B8
:10CA000014E0B37CA64630890124B1784FF0080CBD
:10CA1000CDE908430023CDE9003CCDE90203CDE98F
:10CA20000433CDE9063301200123F047707C104A1E
:10CA30000E49002808BF0A46D05DDAF854200D30B0
:10CA4000C1B220469047F07C4FFA89F2594600F077
:10CA50001FFB88F80090B5FA85F040090BB0BDE8DF
:10CA6000F08F00BF80020020854501006091010821
:10CA70007091010870B50446406804F00FF805464F
:10CA800094F900000021072200F03EFC0626002D4C
:10CA900018BF0726002808BF06F0050694F9010014
:10CAA0000021072200F030FC002808BF06F0030632
:10CAB000304670BDBCB54B494278D1E900340178AD
:10CAC00001EB410103EB81014D7AD0E902130069CA
:10CAD000009005EB450004EBC00000F015FBBCBD69
:10CAE0002DE9F04F8BB0CDE909210646DFF8F4B00F
:10CAF000327896F90150DBE9000102EB420200EBCB
:10CB00008200407A00EB400001EBC00090F9021077
:10CB100096F9020000F04CFA074696F901003249F6
:10CB200000F0D4F9D6E901128246384600F042F905
:10CB300031780446DFF8148ADBF8000001EB41018C
:10CB4000D8F81C9050F82100D8F80C1088472748D6
:10CB500071784057072915D14FF47A614FF47A73F1
:10CB600000250522089158430121CDE90005CDE9B2
:10CB70000225CDE90415CDE906550020214646F2EF
:10CB8000A81210E04FF47A610125082208910021D3
:10CB9000CDE900050120CDE90221CDE90451CDE91F
:10CBA0000611214600225346C8473178DBF80000C1
:10CBB00001EB410150F8210096F9011000F0B4FAA0
:10CBC000B18996F90100F5F759FD0999D8F8542073
:10CBD0000860317B284690470A98077001200BB007
:10CBE000BDE8F08F80020020AC390108CC39010883
:10CBF0000020704780B5024600200A2924D8DFE8CB
:10CC000001F009232323230E11162306060092F9AF
:10CC1000000012E01068BDE8804003F03FBF1078CC
:10CC2000917806E092F900000021052207E01078D3
:10CC3000517840B209B1022100E00021072200F042
:10CC400063FB002818BF012080BD08B10020704799
:10CC500008461146FFF7F3BA00B170470846FFF7E0
:10CC6000F0BA08B1D0B27047084611461A46FFF72D
:10CC70002BBB08B1002070470846FFF76FBBB0B56B
:10CC800000230024914238BF01241209B2EB111F86
:10CC900028BF012304EA0302012A0BD10B0901F08A
:10CCA0000F01012530F8134005FA01F124EA0101D2
:10CCB00020F813101046B0BD38B131B12AB131F8A7
:10CCC000023B013A20F8023BF8E770472DE9F041BA
:10CCD0009A4202DB069B9A4202DD0020BDE8F08109
:10CCE000079B4FF0000E03F1080C00235FFA83F856
:10CCF0008045F2D208EB48030CEB83065FFA8EF313
:10CD000031F813700023102B0ED027FA03F4E40738
:10CD100007D0347804F00F059542D8BFB2EB141F4A
:10CD200007DD0C360133EEE70EF1010E08F11003BA
:10CD3000DCE70120BDE8F08170B54FF4FA6462438E
:10CD40006FF0070404EB410404FB0025DDE9044215
:10CD500055B14619013EB6FBF0F68E428CBF00215C
:10CD60000E46002D18BF31462160414385004C1C02
:10CD7000A5EB5404002908BF84004FF47A70002505
:10CD800003FB00F18C42C8BF40F2E73503FB1051B2
:10CD9000214491FBF0F0106070BD4FF4FA51B1FBEB
:10CDA000F0F07047024A02FA00F0B0FBF1F0704771
:10CDB00040420F00B0B5400014460D4606F05AFB45
:10CDC0000146284606F026FD214606F023FD05F023
:10CDD0002DFE06F0FBFAB0BDB8B1F0B50023CCB221
:10CDE00094420FD230F8144000250026102D06D0B2
:10CDF00024FA05F7FF0718BF01360135F6E733447B
:10CE00000131ECE7BDE8F04000E00023D8B2704704
:10CE10002DE9FE4F02914FF000084FF0010A00216A
:10CE200000244FF0000ECDE90023038A5FFA84F955
:10CE3000994543D209EB49035FFA8EFB00259C001C
:10CE4000102D36D043680AFA05F633F81B301E421F
:10CE50002CD087683B594BB30378E3B13E1990F966
:10CE60000130377A3A07B3EB227F1FDB7AB2B3EB9C
:10CE7000221F1BDC727AC36802EB420203EBC20280
:10CE8000127D92B1029E5FFA88F309EB050208F168
:10CE90000108F2540AE0D0F814C0BCF1000FDDD054
:10CEA0003CF81B301E42D9D100E001310C34013571
:10CEB000C6E70EF1010E09F11004B6E7009880F8FC
:10CEC000008001980170BDE8FE8F000051F820102D
:10CED0000448054A0844B0FA80F04009914208BF6E
:10CEE00002207047702FFCFF20A10700FEB50678D6
:10CEF0008778BE4214D004467DB2013EF0B2B842FB
:10CF00000DD0D4E9011294F90130E078CDE9003276
:10CF100072B22B46FFF7DAFE0028EED000E03E4664
:10CF200070B2FEBD2DE9F04F85B0074640689B46C4
:10CF300090460D4603F0D8FC3968DDF83C90DDF8EA
:10CF400038A0091AC9F8001001218AF80010002140
:10CF50008BF800107A6812B13A6882421FD82960B3
:10CF60003B7A7A7A3E7DD7E906C0D7E90354C16897
:10CF70000078CDE90065CDE9024C00F0EBF8C9F886
:10CF80000000F86941465A465346FFF741FF9BF8B7
:10CF9000000020B10020C9F80000002005E09AF848
:10CFA00000100B20002908BF0C2005B0BDE8F08F51
:10CFB0008842D8BF084670472DE9FE4F04460579E0
:10CFC00040798A46062198469146002808BF0921E3
:10CFD00014F801B04FF0070108BF0A216656082176
:10CFE000002808BF0B21675C2DB1BBF10F0F04D1E6
:10CFF00094F809B013E0002521E094F91520D4F845
:10D0000018C094F914302169207BCDE9002C4FFA27
:10D010008BF2FFF75BFE002808BF05F0FD050F2E21
:10D0200001D1A67A0BE094F91D00864201DA06468A
:10D0300005E094F91C008642C8BF05F0FB0585F0A9
:10D0400007008AF800B089F80060384308BF01275C
:10D0500088F800702846BDE8FE8F0278032A14D1B4
:10D060004278130902F00F024B708A7082788A802E
:10D07000C37842EA03228A80007900F00F02C0F3ED
:10D080000210C87005200A70704700207047000029
:10D09000F8B5052807D8CDE901120DA112A351F862
:10D0A0002000009002E003A3CDE90012FCF759FA3A
:10D0B0008FBD00BF5258206F6E20667265712025AB
:10D0C0006420487A2061742044522025640D0A00AF
:10D0D0003795010839950108419501083B950108EC
:10D0E000499501084395010852585F2573206F6EDA
:10D0F000206672657120256420487A20617420447E
:10D10000522025640D0A000070B51E46049B0C4693
:10D11000114605463246F5F70FFAE9686043081AEA
:10D1200038BF0020E86070BDE0B5CDE9000102A382
:10D13000FCF717FA8CBD00BF5458206F6E20667242
:10D14000657120256420487A20617420445220258E
:10D15000640D0A002DE9F04F8DB0664D0E4607466E
:10D16000624817991446624A01350844A9424FF0B3
:10D170000001B0FBF2F0039588BF00FB0221029191
:10D1800005935D4900FB0210019016981843049026
:10D1900087F001001843079003F09CFB4FF0FF3B22
:10D1A0004FF000090690002C00F096800894179C20
:10D1B000189D2046294602F001F88246304639463D
:10D1C00022462B46F5F7B8F980462FB105984B4C0F
:10D1D000A8BB4A4CF46032E0B8F1640F09D0B8F54E
:10D1E0007A7F07BFC6F808A0454CD6F808A0454C82
:10D1F00002E0424CC6F808A009A8514601F068FFB9
:10D20000DDE90930DDE9171200900BA801F0C6FF37
:10D2100004990C9831B13169A14203D10B99344A78
:10D2200091420CD31799334AF460914207D94FF6D3
:10D23000FF7120EA0101019801F0C0FFB060706841
:10D2400000B9F460346137B103F04EFBD6E9031442
:10D250000844F06000E0F068A04284BFF46020461B
:10D26000002206997160199908FB01F1814228BFDB
:10D270000122079B134227D000228C42327588BFBF
:10D2800009F101090A1A934538BF5A468C4288BFF2
:10D290009346EFB91898B8F57A7F179B00900398DA
:10D2A00008BF49F6B020B8F1640F08BF4FF46160C1
:10D2B0000299002201440BA801F070FFDDE90B0187
:10D2C00001F07CFF834603E0012009F1010930757C
:10D2D000089C1836013C66E75FEA096108BF4FF019
:10D2E000FF3B58460DB0BDE8F08F00BFD013FEFFE6
:10D2F000805101002FEC010030EC010040771B0051
:10D3000080A81201002E9302884201DB904201DDC9
:10D31000002070470120704700B1704710B5029C93
:10D32000FCF71AF9BDE81040FFF79AB808B10020E1
:10D3300070470846FFF7C2B808B10020704708469A
:10D34000FFF7D8B8004870470100010200B17047EC
:10D350000846FFF77FB9B0FA80F04009704708B17E
:10D36000002070471CB5DDE904400090FCF7F4F89C
:10D37000FFF7BAF91CBD08B1002070470846FFF757
:10D380005FBA08B10920704710B5029CFCF7E4F8B9
:10D39000BDE81040FFF77ABA08B100207047084690
:10D3A0001146FFF7E7BA08B1002070470846FFF7BB
:10D3B00061BB00B170470846FFF77CBB08B1002095
:10D3C0007047084611461A46FFF78ABB08B100208D
:10D3D00070470846FFF70CBC08B1002070470846AC
:10D3E0001146FFF707BC0000F0B58FB0584C00267F
:10D3F0000121584D8DF80C10A4F80C1184F81C6113
:10D40000A66284F8076104F1A80704F1640C694678
:10D41000C5F89C64A5F81C6485F81E648DCFACE843
:10D420008D00A4F8096184F83A60B4F8CC0094F84F
:10D43000B920208794F8A50084F8752084F861004D
:10D4400094F8B80084F8740094F84000D4E92F23CD
:10D45000C4E91E232E4A029204F5F472019204F5E7
:10D46000F2720092FFF772FF4FF4807085F8D0637C
:10D4700085F81F64CDE90D66A5F8E20394F8750000
:10D48000D5F8D01385F8E00394F8800085F8E1031F
:10D4900094F81C0185F8E403606EC5F8D403D5E95F
:10D4A000F6C2D5E9F837C5E9FA1040F20120C5E91E
:10D4B000FCC2C5E9FE37A5F8FA03D5F8480318B150
:10D4C00041680069CDE90D1004F58E7004F26452D4
:10D4D0000C9004F1D8000B9004F144000A9004F180
:10D4E0004000099004F1D400089005F2954007909F
:10D4F00005F58B60069005F22440059005F26C401E
:10D50000049004A80DA9F9F7E6F90FB0F0BD00BF2B
:10D51000A01A0020F8B50C4603F08AFA0B4D286BD0
:10D5200080470B4F0B4E214697F8400006F5856269
:10D53000FFF732FF48B196F82804696B86F86E044D
:10D54000F86C8847E07C86F89404F8BDC43A01087A
:10D550007C8500207C14002000210D4AB0F5803F1E
:10D5600038BF012138BF00040901B0F1807F3CBF02
:10D5700008310002B0F1805F38BF043138BF0001CC
:10D58000000F81F01F01105C081AC0B2704700BF85
:10D59000483B0108F4F788BAD248811C021DF4F711
:10D5A00065BA00BFF8B5044600200D46002600F01D
:10D5B00093FAF6F7BFFA01F04DFEFBF7F1FCFBF72B
:10D5C00059FDFBF7D1FD5348F6F74BF800F0CEF8C4
:10D5D000F4F7A0FA3220F5F7CEFDC24FAE4229D2C1
:10D5E000FFF7DAFF00F05AF8388A2188084461888A
:10D5F0002080B8890844A188608038890844A080C8
:10D60000F86905F0E3FEE18801360144E1802189F3
:10D61000014421816189084439886081A0890844D6
:10D62000E189A08178880844218AE081B88808448B
:10D630002082D3E7B4F90000B4F90210B4F9042051
:10D64000B4F9063090FBF5F0208091FBF5F0608096
:10D6500092FBF5F0A08093FBF5F0E080B4F90800B0
:10D6600090FBF5F02081B4F90A0090FBF5F06081A1
:10D67000B4F90C0090FBF5F0A081B4F90E0090FB1A
:10D68000F5F0E081B4F9100090FBF5F02082F4F79A
:10D690000BFA924800210170F8BD00BF70B51D481B
:10D6A000F5F7DFFFF4F736FA02F014F8FDF73EFB6A
:10D6B0008C4E308AB16A0844716AB062B0890844FD
:10D6C00031897062D6E90702D6E905451144316215
:10D6D000B16B0131B16305F079FE05F0CBFE014677
:10D6E000706B05F0E5FC7063284605F06FFE05F0F1
:10D6F000C1FE0146306B05F0DBFC3063204605F0CF
:10D7000065FE05F0B7FE0146F06A05F0D1FCF06257
:10D7100070BD00BF784C0020BCB504463020F4F743
:10D720008FF90546C00601D4002006E0684601F0E6
:10D7300009FD6C480099816401202070280701D4FC
:10D74000002006E0684601F0FDFC6648009941644F
:10D7500001206070BCBD00BF10B50020002400F0A7
:10D76000BBF9F4F7A1F95D48047010BD5D480021D4
:10D77000632280F84C1080F84F10A0F85010A0F8E9
:10D780005210A0F85410A0F85610A0F85810A0F8A5
:10D790005A1080F85E20C163C0E90A11C0E90C117B
:10D7A0008163C0E90211C0E90411C0E90611C0E9B2
:10D7B00008110164704700BF2DE9F843494C4FF050
:10D7C000010984F84C90E06B84F84F0044480078DD
:10D7D00068B3A06BD4E90923D4E90761D4E90585CE
:10D7E000B3FBF0F3B2FBF0F2B1FBF0F1A4F8503070
:10D7F000A4F85220A4F8541005F03CFE0746304629
:10D80000394605F0EDFC05F0E1FDA4F85600284688
:10D81000394605F0E5FC05F0D9FDA4F8580040466E
:10D82000394605F0DDFC05F0D1FDA4F85A000020D2
:10D83000E063C4E90800C4E90A00C4E90C00A0637D
:10D84000C4F84090BDE8F883264991F84C20027056
:10D8500091F84F20C270B1F850208280B1F8522068
:10D86000C280B1F854200281B1F856204281B1F84B
:10D8700058208281B1F85A10C1817047BCB5174C4D
:10D88000207850B301A8FFF747FF9DF8040068B166
:10D89000FFF782FEFFF76AFF1148007830B10025DC
:10D8A000022D03D8FFF7FAFE0135F9E79DF80500D0
:10D8B00078B1FFF771FE0B4D686CA96C401AFA2124
:10D8C000B0FBF1F202FB1100E863FFF775FF0120E6
:10D8D000286400202070F4F7E7F8BCBD0C4E00204F
:10D8E000B0330020CC010020B0B590B06C46402190
:10D8F000FBF75CFE35492046402202F02DFF9DF8E3
:10D900000000B8BB9DF801005A2833D19DF80200F1
:10D9100001282FD187489DF804109DF805209DF817
:10D9200006309DF8075080F8281080F8292080F8EC
:10D930002A3080F82B5000229DF8081080F82C1017
:10D940009DF8091080F82D109DF80A1080F82E100F
:10D950009DF80B1001F03F0180F82F1004F10B012E
:10D9600090F82F309A4215D28D5C8318013283F8DB
:10D970003050F5E7FCF79EFC884800211422103057
:10D9800002F0F3FE4FF47A70F5F7F5FBFCF730FB8D
:10D9900010B0B0BD9DF828109DF829209DF82A30C0
:10D9A0009DF82B5080F84C1080F84D2004F12C018C
:10D9B000002280F84E3080F84F50142AE6D08C5C5C
:10D9C0008318013283F85040F7E700BF00F80308DE
:10D9D000B0B58EB006A81A210630F3F7A5FE304880
:10D9E000012500248DF81C508DF817400690F4F79F
:10D9F00079FDFD280DF1170088BF63248DF81D40C7
:10DA000000F050F800283FD001AC12211225FBF79E
:10DA1000CDFD20460A21FFF7C5FDBDF80610BDF873
:10DA2000040009BA8DF82000000A090CADF8211095
:10DA3000BDF8081009BA090CADF82310BDF80A109A
:10DA400009BA090CADF82510BDF80C1009BA090C7B
:10DA5000ADF82710BDF80E1009BA090CADF8291061
:10DA6000BDF8101009BA090CADF82B10BDF8121052
:10DA700009BA090CADF82D10BDF8141009BA090C3B
:10DA8000ADF82F10192101E0082158208DF81F0052
:10DA90008DF81E5006AAFBF765FF0EB0B0BD00BFA3
:10DAA00053005A0110B50446F3F7AAFF2070E52889
:10DAB00018BF002010BD0000022888BF70470A4828
:10DAC00010210122F5F770BD022888BF7047064873
:10DAD00010210022F5F768BD022888BF7047024870
:10DAE00010210122F5F760BD0004004802A20120C8
:10DAF000052100F005B800BF5056585858000000E6
:10DB000070B50C4B0024A14204D0155DDE6835557C
:10DB10000134F8E703F8080F00225970D97A184643
:10DB2000F8F7B4FB063018BF70BDBDE87040F8F7D9
:10DB3000D9B900BF0000002010B5184C207C58B1A6
:10DB400004F03AFD002818BF012040002071207920
:10DB5000022801D10020207410BD00BF10B50F4C69
:10DB6000207C00B110BDE068022807D3E0680428DB
:10DB700004D80BA201200421FFF7C2FFE0680528AA
:10DB8000F0D304F019FD002818BF012040002071D7
:10DB900020790228E6D10020207410BD84030020E3
:10DBA0005246414300000000074940F441700A68B2
:10DBB00022F040020A6008604FF4B85048600868DC
:10DBC00040F040000860704700000158B8B54E4C66
:10DBD00064232268FBF7F1FF294B0092009A3AB1C7
:10DBE000009A013A00921A689207F7D5002201E0E4
:10DBF00001228260FF251D7164252468C4EBC404E2
:10DC0000C4F34C446C430094009C34B1009C013C30
:10DC100000941C68E407F7D001E001228260586894
:10DC200008701046B8BD00BF18B5374C6423226891
:10DC3000FBF7C3FF124B0092009A3AB1009A013AE7
:10DC400000921A689207F7D5002201E00122826053
:10DC5000197121686424C1EBC101C1F34C416143D6
:10DC60000091009931B10099013900911968C907F3
:10DC7000F7D001E0012282605868104618BD00BF4D
:10DC80000800015881B00179012915D11E490968A0
:10DC900001EB4101C1F34F31009109490A6822F4B7
:10DCA00000420A60009A013A0092009A002AF9D1D3
:10DCB0000A6842F400420A6001B000F007B800BFF1
:10DCC00090040058E948F6F701BF00BF81B00E4943
:10DCD0006422096801EB4101C1F34B4151430091BA
:10DCE0000A490A68009B53B1009B9208013B0093CC
:10DCF0000B6802EA5302D207F3D1002002E00221AE
:10DD00008160012001B070475801002014040058C0
:10DD1000E0B500F07F000DF1070101228DF807004A
:10DD2000892000F0A3FC8CBDE0B51849884204D3DB
:10DD3000E1208DF80600E9201EE01549884204D351
:10DD4000D7208DF80600DB2016E01249884204D364
:10DD5000C1208DF80600C5200EE00F49884204D38B
:10DD600075208DF80600812006E00C49884205D315
:10DD70006B208DF806006F208DF807000DF106016D
:10DD80009820022200F072FC8CBD00BF01E9A4358E
:10DD900081F8A9328144E52D010B6B1B41FC54191C
:10DDA0002DE9F843194C814640F607008846A04704
:10DDB00006464FF4D660A047074600F00F0540F234
:10DDC000B160A0473A0740EA0520114948BF08431F
:10DDD000C6F3C1010FA20123515C06F00702013A0C
:10DDE00091400D4AB2FBF1F1B1FBF9F2082A38BFBC
:10DDF00002235A43042A38BF04235943490948439C
:10DE0000C011C8F80000BDE8F88300BF39E0000881
:10DE100000F0FFFF04080A0C0048E80160B1074A5F
:10DE20000021B02907D0535808318342F9D950183E
:10DE300010F8040C7047FEE71F207047D439010822
:10DE4000F1484078704700BF1CB504460DF105014C
:10DE50001420032200F0E2F8EB48817801292170B8
:10DE600010D009BB9DF805009DF806109DF807200D
:10DE700020710020A06048424008A0715042400834
:10DE800060711CBD40689DF8071020619DF8050079
:10DE90004042400820739DF90600023080086073FC
:10DEA00048424008A0731CBD20460021142202F005
:10DEB0005CFC0F2020701CBD7CB50E460446002083
:10DEC0000DF1070115468DF80700304600F04CF8BB
:10DED0003278AA4201D901207CBD9DF80700214675
:10DEE00000F08EF800207CBD0A2070477CB5002031
:10DEF000019040F6E20000F09FF8144E044600F056
:10DF0000FE0140F6E200B04740F6E50000F094F86C
:10DF1000054600F07F0140F6E500B0476FF07F4016
:10DF200000F034FA01A940F61900042200F090F83C
:10DF3000002000F08BFA40F6E2002146B04740F6A0
:10DF4000E5002946B04701987CBD00BF89E600087E
:10DF5000E0B50DF107011520012200F05FF89DF8F2
:10DF60000700404240108CBDBCB50C4605460DF183
:10DF700006011320022200F051F8E04881780129BF
:10DF800007D1C078012804D140F2027000F054F8A3
:10DF900001E09DF8060028709DF807002070BCBDC8
:10DFA00010B508B1ED498860FBF7D0F80220FEF704
:10DFB00031F9EA4C00202070002000F047FAFCF70D
:10DFC00049FF01280DD101204FF4207100F07AFAA9
:10DFD00040F61110002100F057FB7F20FFF798FE5C
:10DFE00009E040F61110102100F04EFB40F612102F
:10DFF000102100F049FBFCF7F9FE0120607010BD14
:10E0000010B5FBF744FBEFF31084EFF3108072B60A
:10E010001648F6F70FFE84F3108810BD10B5FBF715
:10E0200036FBEFF31084EFF3108072B60F48F6F76B
:10E03000DFFC84F3108810BDE0B501460B480DF1FC
:10E0400007020123F6F722FE9DF807008CBD00BFF2
:10E0500010B5FBF71CFBEFF31084EFF3108072B6E2
:10E060000248F6F713FE84F3108810BD144D00200B
:10E0700010B5144600F044F92046BDE8104000F009
:10E0800035BAE0B58DF807108DF806000DF10601E0
:10E090008F20022200F0EAFA8CBD000080B5C52076
:10E0A0000021002200F0E2FAF1480721417080BD12
:10E0B000E0B540BAADF80600ED48807800B18CBDFF
:10E0C0000DF1060140F2BE60022200F0E9FA8CBDBB
:10E0D000E0B540BAADF80600E548807800B18CBDE7
:10E0E0000DF1060140F2BC60022200F0D9FA8CBDAD
:10E0F000E0B58DF80520120A8DF80310090A8DF895
:10E100000100000A8DF807301B0A8DF804208DF8F5
:10E1100002108DF800006946082008228DF80630AC
:10E1200000F0A4FA8CBDE0B58DF807000DF10701F1
:10E13000A020FBF79DFB9DF8070040280ED3410867
:10E140000020CAB2202A02D301309108F9E700EB7F
:10E15000C100C1B240F2067000F096FA8CBD00001A
:10E160001CB5EC4904460020CDE9000020788978F0
:10E17000814202D000F0B0F82178032942D8DFE8CC
:10E1800001F00222262DA089204A0023ADF80300C9
:10E19000D4E90101B2FBF0F0020A8DF80200000C94
:10E1A0008DF801206E4A8DF800004806C909F3F782
:10E1B00071F9010A8DF80700000C08228DF806108D
:10E1C0008DF805001AE0A0690422009016E0207D79
:10E1D0000E4904228DF80300206905E0A0890B494F
:10E1E0000522ADF803006068B1FBF0F0010A8DF87C
:10E1F0000200000C8DF801108DF8000069468B209C
:10E2000000F034FA1CBD00BFA00200200000093D50
:10E21000E0B58DF806208DF804008DF807308DF8F4
:10E22000051001A99520042200F020FA8CBD000001
:10E230007FB504460020B74D8DF80C00CDE90100F4
:10E240002078A978814202D000F046F8217803298D
:10E2500040D8DFE801F0020D1A02667AF12E19D0DB
:10E26000F22E21D1062641F2210541F60F5016E08B
:10E27000207C617C0622E8708DF806008DF807107E
:10E28000608AADF80800E0891CE0207B01228DF84F
:10E2900004001BE0022648F205054FF6FF70FFF769
:10E2A00017FF2846FFF704FF20798DF80B6009223D
:10E2B0008DF80600D4F80500CDF80700A07A8DF897
:10E2C0000C00608800BA000CADF8040001A98C2095
:10E2D00000F0CCF97FBD00BFE0B5DC498DF8070048
:10E2E000887020B940F2AC60002100F0CDF90DF14A
:10E2F00007018A20FBF7BCFA8CBD00BFA0020020FA
:10E300000A460146002000F0A3B9E0B5FCF7A0FDE5
:10E3100001380DF107010122B0FA80F040098DF8B3
:10E320000700962000F0A2F98CBD0000BCB5C74DD7
:10E330000446287820B92046FFF7F6FC0120287013
:10E34000074A6006E1090023F3F7A4F800BA0422A3
:10E35000019001A9862000F089F9BCBDA00200202F
:10E360000048E801B0B50446FCF73EFD022805D0A0
:10E37000012520B90F2CC8BF022500E00225284640
:10E380002146022200F0D2F82846B0BDE0B5AF49E0
:10E3900005228DF807004A70010A000C03228DF84F
:10E3A00006108DF805000DF10501822000F05EF9E0
:10E3B0008CBD00BF1CB50446A4480521417040F641
:10E3C000AC00972100F060F9200A0DF1050103224D
:10E3D0008DF807408DF80600200C8DF8050082208E
:10E3E00000F044F91CBD00BF1CB50A0A8DF80710E7
:10E3F000090C8DF8040006248DF80510010A000CA4
:10E400008DF8062006228DF803108DF802000DF11C
:10E410000201942000F02AF98C4844701CBD00BF12
:10E42000BCB5044600200025FCF7BAFC0220FDF72D
:10E43000F1FE04F007000DF1070101228DF807003D
:10E44000842000F013F981484570BCBDE0B58DF81B
:10E4500007000DF107018020FBF70AFA9DF807106D
:10E4600002200029794908BF012048708CBD00BFF7
:10E47000A0020020E0B58DF807000DF107019F20F4
:10E48000FBF7F6F98CBD012908D110B50446012827
:10E4900007D10420FDF7BEFE022003E00120FCF7B7
:10E4A0007FBC0120022C08BF0320BDE81040FCF710
:10E4B00077BC80B501464FF4D860082200F0F0F830
:10E4C000002080BDE0B500F007008DF807100422A1
:10E4D0008DF80400080A8DF80600080C8DF8050078
:10E4E00001A9972000F0C2F88CBD0000E0B55749A3
:10E4F00004228DF807004A70010A000C03228DF8EF
:10E5000006108DF805000DF10501832000F0AEF82E
:10E510008CBD00BFA0020020D1200021002200F00D
:10E52000A5B8D2200021002200F0A0B87CB5144686
:10E530000D46012810D10020FCF750FCA842B8BFBE
:10E5400005460A2826D006460E282AD10420002196
:10E550000122FBF717F82CE040F6D800FFF76CFD1E
:10E5600040F01E0140F6D80000F08EF80120FCF7C4
:10E5700035FCA842B8BF05460E2822D00646112811
:10E5800025D0142E2AD1032005210022FAF7FAFF04
:10E5900002352BE0012000210122FAF7F3FF0335B9
:10E5A00007E0062000210122FAF7ECFFA81B00F18A
:10E5B0000E0568B210F1110FD8BF6FF010051821C9
:10E5C0001BE0022002210022FAF7DCFF0EE002200D
:10E5D00003210022FAF7D6FF053507E004200721C2
:10E5E0000022FAF7CFFFA81B00F1160568B210F160
:10E5F000090FD8BF6FF00805382140F6E70000F09A
:10E6000043F80DF106018E2002228DF807408DF8A7
:10E61000065000F02BF87CBD10B504460B488078FE
:10E6200000B110BD4FF4D760FFF706FDC4F3002121
:10E6300000F0FE0001444FF4D76000F025F8E1B28D
:10E6400040F2B960BDE8104000F01EB8A002002002
:10E6500010B5FBF71CF8EFF31084EFF3108072B6DF
:10E660001648F6F757FB84F3108810BD10B5FBF77A
:10E670000EF8EFF31084EFF3108072B60F48F6F740
:10E68000E1F984F3108810BDE0B503460B488DF81E
:10E6900007100DF1070219460123F6F761FB8CBD47
:10E6A00010B5FAF7F4FFEFF31084EFF3108072B6B1
:10E6B0000248F6F755FB84F3108810BD144D002076
:10E6C0007047000080B50B48F3F766F978B10A4946
:10E6D00040F6E4424FF6FF7309884A43994204BF6B
:10E6E00040F6D802C0F24C02B2FBF0F000E000208D
:10E6F00080B280BD004000B8AA75FF1F1CB5002085
:10E70000ADF80600FFF7DEFF04461448F3F744F9BE
:10E71000134960430A88098C891A07D040F6E443FC
:10E72000B0FBF3F0801A642250430AE040F6FF7118
:10E730004FF47A72B0FBF1F00A4900FB021040F688
:10E74000C41190FBF1F01E30ADF80600BDF80600D4
:10E750000002ADF80600BDF906001CBD001000B0B7
:10E76000A875FF1F4067F4FF014802490160704728
:10E77000B44B002000240140F0B58FB00446F8F7F8
:10E78000ADF808B10E2514E1AA4F97F8040101284D
:10E7900007D1F8F7A9F810B9F8F7A4F808B10F25D0
:10E7A00007E1386B38B9A449B7F80C01D1F8201447
:10E7B0004843401A3863A04E96F80401042807D055
:10E7C000002840F0F58006F58470FAF794FA03E02B
:10E7D00006F58470FAF728FA08B11125E9E096F8F1
:10E7E0000C013080386B039097F839008DF81400D5
:10E7F00097F808018DF8160001A800F0A3FCD7E9EE
:10E800004430DDE9011200900AA800F0C7FCDDE900
:10E810000A01FA6ACDE9060104923288002001213A
:10E820008DF820008DF81510ADF8222097F81C21E6
:10E830001AB98DF815008DF8201007F1300197F8FE
:10E84000400006F21F4206F59363009103A9FEF70C
:10E8500098FDB0B105460B2840F0AB80002C47D0A6
:10E86000D6F8981459B1D6F8400306F55A7440F01A
:10E870002000C6F84003FAF731FFFAF746FF0025FB
:10E8800097E097F8404097F9613097F9392097F869
:10E8900075102046FEF7E5F906F56E717B6C97F86A
:10E8A0004820009141B22046FEF736FD7B6C97F878
:10E8B000482097F9681097F8400006F574740094A2
:10E8C000FEF72AFDD7E91423D6F8C403D6F8DC13E3
:10E8D00002440B44C6E9EC2397F81C2152B10020F6
:10E8E0000A900AA8F8F77EF8002865D0132560E0A2
:10E8F0000B255EE0D7E9162310441944C6E9EC0164
:10E9000000210A9197F8382097F8393096F81F447B
:10E9100097F840008DF829308DF82A20D7E91E237A
:10E920008DF82840CDE90B238DF83610318806F597
:10E9300084630DF12702ADF8341000218DF8271003
:10E940000AA9FEF73BFD0120C6F8544486F84504A9
:10E9500097F8390086F846049DF8270086F84704A2
:10E96000D6F82004C6F85C04C6F84C04F7F7B8FFE4
:10E9700030B1D6F82004F7F7B9FF08B1102518E038
:10E9800097F80401012808BFF7F7C2FFF7F7A2FFC5
:10E99000002096F81F4497F839500E9096F804011D
:10E9A00004281AD020B906F58470F8F761FA26E039
:10E9B000032528460FB0F0BD96F837029DF82810C1
:10E9C0000C1897F93900F3F735FE0825FF2C98BF8E
:10E9D0008442EED897F81C1194E70EA8F8F7B8F91E
:10E9E00008B11225E5E796F81C140E9809B1013814
:10E9F0000E9006F5847329462246F8F763FA00283C
:10EA00007FF4EBAED6F84003C14A96F80C1100250E
:10EA1000C6F89C5440F00200926A3180C6F8400368
:10EA200096F81C04013086F81C0486F84904B01CD2
:10EA30009047BEE77C8500207C1400202DE9F0473C
:10EA4000BEB040B11C4633B106460D46080708D09B
:10EA50004FF0050A01E04FF0020A50463EB0BDE813
:10EA6000F087174601A80021F02203F062FC6946F6
:10EA70003846F3F7A3FD82460028EED100980DF149
:10EA8000040810214FF010094246013003F0B0FB9A
:10EA900000272804E1D056FA87F054FA87F142465D
:10EAA00003F04AFA59FA87F7103DF2E77E2B98BF38
:10EAB000F3F782B9032070471FB5A0B114460A4688
:10EAC0007F2C01D1042A10D100216B46CDE902111F
:10EAD000CDE900111021FFF7B1FF38B96946204692
:10EAE00000F032F902E0022000E0032004B010BD83
:10EAF000AE480068704700BFAC48006808307047F7
:10EB000010B5AA4A0023126803F11104BB2C06D0E9
:10EB100013441B7C83422346F6D1FAF7A0BD0320A1
:10EB200010BD00BFB0B558B10C46A04D0549C0227C
:10EB3000286003F0EAFB0CB12868A0470020B0BDB4
:10EB40000220B0BD00E503082DE9F04389B01E4B5B
:10EB5000DFF87880FAF7FCFC1D4D0020A847012063
:10EB6000A8471C4BFAF7F4FC0320A8470220A8474B
:10EB7000194BFAF7EDFCDFF86490D9F80000017842
:10EB800042788378C678077944798579C0798DE8A9
:10EB9000CE00CDE90545079011A3FAF7D9FCD9F8C5
:10EBA0000000017A427A837AC47A057B467B877BB0
:10EBB000C07B8DE8FE00079019A3FAF7C9FC00207E
:10EBC00009B0BDE8F08300BFD0940108BD0501087D
:10EBD000A9A60008A6940108BB940108381B0020D0
:10EBE000232323232323204465764575693A202077
:10EBF00020202020253032583A253032583A25300E
:10EC000032583A253032583A253032583A25303287
:10EC1000583A253032583A253032580D0A00000053
:10EC2000232323232323204170704575693A202034
:10EC300020202020253032583A253032583A2530CD
:10EC400032583A253032583A253032583A25303247
:10EC5000583A253032583A253032580D0A00000013
:10EC600010B5054C0420A0477F20A0470220A047F4
:10EC70000320A047002010BDA9A60008F8B543B1A5
:10EC8000079C34B1089F27B1069D212D03D905208B
:10EC9000F8BD0220F8BD204619462A461E4603F05C
:10ECA00034FB691E701C631C012289B2FFF7C6FE8B
:10ECB00008B10720F8BDE07AC10940B200283970D8
:10ECC00017D4281F2A19215C12F8033C12F8025CA1
:10ECD00012F8012C41EA0321012341EA054141EAEE
:10ECE000026281B2204600F063F8002818BF0120BC
:10ECF000F8BD0420F8BD000038B110B50446E7485F
:10ED0000406980472060002010BD0220704700BF8E
:10ED1000C43A010840B180B5014624480822006881
:10ED200003F0F3FA002080BD0220704748B180B59F
:10ED300001461E4808220068083003F0E6FA002069
:10ED400080BD0220704700BFF0B585B009B3174EF3
:10ED50000023326803F11107BB2F1CD013441B7C26
:10ED600083423B46F6D1802817D100207F22CDE98F
:10ED70000300CDE9010001AD084610212B46FFF745
:10ED80005DFE0446306829461022384403F0BDFA7F
:10ED900008E0022406E0032404E0D019102203F066
:10EDA000B4FA0024204605B0F0BD00BF381B002097
:10EDB000A0B11CB514460A4601460020019001A8E6
:10EDC00000900020F2F7F8FF01460198A0420846A3
:10EDD00018BF0120002918BF08461CBD022070473B
:10EDE000F0B585B0F3F77EFB04466846FEF72CFDD0
:10EDF000684D674E142028727079E9680870707841
:10EE000060B11520FE210227287200207070632057
:10EE10006043B0FBF1F0E968487000E0012740482A
:10EE2000017800295AD000210D220170E868C155EF
:10EE30005A21E868384441700121E86838448170FB
:10EE40006320FE216043B0FBF1F0E9683944C870EB
:10EE5000381DE9680A54E9689DF8032001444A70A6
:10EE6000E9689DF8052001448A70E9689DF804204E
:10EE70000144CA70E9689DF8072001440A71E968F5
:10EE80009DF8062001444A71E9689DF80920014473
:10EE90008A71E96808449DF80810C17107F10C01F6
:10EEA0001237E8689DF80B204254E8689DF80A2064
:10EEB00008444270E8689DF80D2008448270E868B4
:10EEC0009DF80C200844C270E8689DF80F200844A3
:10EED0000271E86808449DF80E104171307996F887
:10EEE0005D100128384688BF0020687251B1F7F7DD
:10EEF000B5F8012806D106F1540001F099FD21482A
:10EF0000FAF794FA022F09D3E97C05F108000022F0
:10EF1000F7F7BCF9063008BFF6F7E4FF05B0F0BD1F
:10EF20000C02002070B5174C174E4FF4004101221F
:10EF300001252046B04720464FF400710122B0471A
:10EF400020464FF400610122B0471048FAF74EFC0A
:10EF5000F7F713FA80B90F480D4E1030F570F6F739
:10EF600097FEF1780220002918BF01200121F7F750
:10EF700021F8204601F026FD0448BDE8704001F06C
:10EF800021BD00BF00040048A9350008F00300209F
:10EF90008403002000000020414890F89514890760
:10EFA00003D590F89314022909D33B4991F806211F
:10EFB0002AB18A6A013228BF4FF0FF328A620021EB
:10EFC00080F81E14A0F81C14D0F8401321F00201A0
:10EFD000C0F84013704700BFF7F754B8F8B52E4E8D
:10EFE000054696F8040102280CD001280DD050B92E
:10EFF000022D1AD0012D4CD02DB9D6E91901C6E940
:10F000001B0100E055B1032441E02846F7F781FCDD
:10F010000446E0BB86F80451002438E01F48002471
:10F0200086F80441C06A804731E01D484FF0020C69
:10F0300086F804C100F5747700F57A7EBECFAEE89D
:10F04000BE0096F8DA1080F8FBC3C1B140F201317E
:10F0500096F8F420A0F8FA13D6F8F01086F870208D
:10F0600096F88020F166C0F8EC1390F81F1480F831
:10F07000F92380F8E81396F8751080F8F813002447
:10F0800080F81E440548C06A8047FBF715FA204601
:10F09000F8BD01250120B9E77C850020C43A0108AC
:10F0A0007C1400207047000010B51944029B002416
:10F0B000C0E90014054C1A4413048280A34204DB07
:10F0C000A2F57A7201318280016010BD0100E70370
:10F0D000F8B5054646480C464768C068804706466E
:10F0E000B8470346B0B200904FF47A70B4FBF0F129
:10F0F000034801FB004082B22846FFF7D5FFF8BD68
:10F1000018FCFFFF70B586B0394904460020CDE9F0
:10F11000040004A84E68D1E90351043088470490E4
:10F12000A8470546B0470146DDE90430AAB2009081
:10F1300002A8FFF7B9FFDDE90201C4E9000106B04A
:10F1400070BD00BF10B500210446016040F8041FE7
:10F15000274909698847206010BD00BFF0B587B016
:10F160000C46234905460020CDE9040004A80E689A
:10F170008F6809690430884703460490059829463A
:10F180002246009002A800F009F80298BDF90C4050
:10F19000B0472046B84707B0F0BD00BF10B5C91A48
:10F1A000029B0024C0E90014D21A1304828004D503
:10F1B00002F57A7201398280016010BDFEB5054604
:10F1C0000B480C464768C06880470646B847034668
:10F1D000B0B229462246009001A8FFF7DFFFBDF933
:10F1E0000810019A4FF47A7002FB0010FEBD00BFB8
:10F1F000883B010880B51348016821F40041016093
:10F2000001F0C2FB104801210170F2F727FE01F066
:10F2100029FA0E4801F046FA0D484FF4004101600A
:10F22000002001F043FAFFF79FFAF2F7A0FFFEF784
:10F2300093FA01F05DFA01200121BDE8804001F060
:10F240005DBA00BF08000058341B002015F8000804
:10F2500010400058B0B59AB008AD4421281DF2F70F
:10F2600085FA02AC18212046F2F780FAF4F702FD85
:10F27000164817490A5822F018020A500120109027
:10F280000A6860F34A220A600868B02100F4C0608E
:10F29000019000201390CDE9110181200B902420D2
:10F2A000089001982846F4F737FF60B94F201421E1
:10F2B0000290201DF2F75AFA20460221F4F7B2FD1F
:10F2C00008B91AB0B0BDF2F76FFF00BF90FCFFFFA6
:10F2D00000040058704700006148F5F7E9B900BF25
:10F2E0000148F5F760BE00BF204D00205C480221B8
:10F2F000F5F7B6B95A480021F5F7B2B958480121D7
:10F30000F5F7AEB9024656480221F5F7ADB900BF90
:10F31000024653480021F5F7A7B900BF02465048FE
:10F320000121F5F7A1B900BF4FF47A71A0FB0101EB
:10F33000800A40EA8150704780B5FAF76FF880BDC7
:10F34000B0B5FAF76BF80446F3F7C8F90546F3F7DA
:10F35000C5F9401BA04228BFB0BD00BFF7E703209E
:10F36000704770B50446F3F7B9F905466FF39F206F
:10F370004FF47A714843860AFFF7B8FFA90A26803E
:10F3800041EA805070BD00002D480068704700BF02
:10F3900080B5F3F7A3F92A490968401A80BD00BF78
:10F3A00011480078012808BFF3F798B9002070478A
:10F3B00070B50D4D2878A0B9294C4FF0FF36266363
:10F3C000F9F78AFE00F03EF8FAF7EBF820462663DC
:10F3D000F5F750F90020FFF795FF00F007F801203E
:10F3E0002870002070BD00BF9E19002080B5F3F783
:10F3F00075F91349086080BDB0B58CB001AD044605
:10F4000028212846F2F7B2F900F01CF84FF4807179
:10F41000002001220B914FF000510890CDE9060128
:10F420000748294600682044C04302900C48F5F77D
:10F4300045FA08B1F2F7B8FE00200CB0B0BD00BF2D
:10F44000301B002010B50548054C01210160FAF77A
:10F45000A8F84FF0FF302063002010BD5C2800406A
:10F46000DC4C002070B5184A0368904218BFB0F118
:10F47000804F05D14C6823F070032343904208D09D
:10F48000B0F1804F05D0114CA04202D0104CA042E8
:10F4900003D1CC6823F4407323434E6923F08003E7
:10F4A0000C688D68334390420360C562846205D066
:10F4B000064A904202D0064A904201D1096901638E
:10F4C0000121416170BD00BF002C01400048014096
:10F4D0000044014010B5036A046A24F00104046288
:10F4E000846924F0F00444EA0212826123F00A02E3
:10F4F0001143016210BD036A23F0100303628369A4
:10F5000023F4704343EA0232036A826123F0A002CB
:10F5100042EA011101627047F0B5EFF31082EFF398
:10F52000108372B66A4B1E8A5C8AA6420CD1C4F55F
:10F530008066B5B2854216D8844214D900250126CA
:10F540001C805D829E7010E00CD2C4F58067BDB255
:10F5500085421BD8864219D900251C8001245D8272
:10F560009C7001E0361B25463446A4B2844207D97C
:10F570000D80598A08446FF39F205882002001E0D3
:10F580004FF6FF7082F3108800B2F0BD25463C466E
:10F59000EBE700BFEFF31080EFF3108172B64C4938
:10F5A000CA8A0132CA8280F310887047B0B5484DCC
:10F5B000EFF31084EFF3108072B6E88A10B184F391
:10F5C000108809E0FFF7E6FF688A298A814205D1A1
:10F5D00000F072F884F310880020B0BDAA786AB1F8
:10F5E000012A13D12B880222AA7000225B1A2A80DA
:10F5F000AB821B040AD12A82AA7000E00A46114697
:10F60000904294BFC2F58060801AA882284884F393
:10F610001088441801F042F82648A98AC26820469A
:10F62000BDE8B040104700BFB0B5EFF31080EFF376
:10F63000108172B626498C78022C03D10024002256
:10F640008C7004E00A8A8B8A1A446FF39F224B8ADB
:10F650000A829A4211D0CD8A012D0ED1ACB1012C73
:10F660001BD10D8802248C700024AD1A0C808D8271
:10F670002D0412D10C828C7008E080F3108801F008
:10F6800009F8BDE8B04000F017B81446A34294BF93
:10F69000C4F580621A1B8A82224680F310880448CF
:10F6A000898A1044034AD268BDE8B040104700BFC1
:10F6B00038040020C83B0108EFF31080EFF31081FD
:10F6C00072B60349CA8A013ACA8280F31088704729
:10F6D00038080020F8B50120F2F748FA0520F3F7C2
:10F6E0004AFD2049204A214B214C224D224E002028
:10F6F0000027B7F5006F07D0C851D051D851E0515D
:10F70000E851F0510437F4E71C4C2046F3F7ACFF06
:10F710002046F3F7A6FFF2F773F9194C2046F5F7E8
:10F7200089FB2046F5F7A8FB2068164C002500262B
:10F73000016841F0010101602580B0B2B5EB502FA6
:10F7400007D121880029FCD0F6F702F9258001367F
:10F75000F3E70020F2F70AFA0948BDE8F840F5F7A8
:10F76000B1BB00BFA4230020A41B0020A42B0020B9
:10F77000B4330020B43B0020B4430020784C002078
:10F78000204D0020981B0020124A116819B101F188
:10F7900014028142F9D1002918BF0121084670479F
:10F7A0000C4A116809B100230B721060416100F02E
:10F7B00013B800BF10B5074909680A46496921B165
:10F7C0000B6804689C42F8D800E000215061416158
:10F7D00010BD00BF9C1B00202DE9F041DFF83080F8
:10F7E0000446D8F82000D8F8187080470546012054
:10F7F00026682072B8472844864203D2B847284476
:10F80000206000E02068D8F80810BDE8F041084703
:10F810009C3B0108BFB5054602A80C46FFF772FCE9
:10F82000BDF90C00029B0090284602F0E9FE284634
:10F83000F1F7D4FE2080BFBDB0B5416E91B1026832
:10F840000C4B0D4D91689268C1F34261520F5C5CA4
:10F85000695C9B5CAA5CC900D200B1FBF4F1B2FB0D
:10F86000F3F201E001220121A0F86810A0F86A205B
:10F87000B0BD00BF589101085091010810B5816AD0
:10F88000CA0706D00268C36A546824F400342343CC
:10F8900053608A0706D50268036B546824F48034E9
:10F8A000234353604A0706D50268436B546824F427
:10F8B0008024234353600A0706D50268836B54688B
:10F8C00024F4004423435360CA0606D50268C36B80
:10F8D000946824F48054234393608A0606D5026812
:10F8E000036C946824F40054234393604A060FD5B4
:10F8F0000268436C546824F480141C43B3F5801FE1
:10F90000546005D1836C546824F4C00423435360CD
:10F91000090606D50168C06C4A6822F4002210432B
:10F92000486010BDBCB504460020C4F88C00F3F755
:10F9300041FE05462068016809070BD56FF07E403F
:10F940004FF4001100222B460090204600F0B0FB3F
:10F9500070B92068006840070CD56FF07E404FF406
:10F96000800100222B460090204600F0A1FB08B148
:10F970000320BCBD2020C4F88400C4F88800002007
:10F9800084F88000E066BCBD806A0021A0F85E10AB
:10F99000A0F85610F5F751BCB0B5846A2068D4F8C9
:10F9A0008420D4F888508168212A09D111F080017F
:10F9B00006D00020A4F85600204600F053F8206836
:10F9C0008068222D08D110F0400005D00020A4F856
:10F9D0005E00204600F02AF8D4F88C0040F01000B9
:10F9E000C4F88C002046BDE8B040F5F726BC01689D
:10F9F000806A0968890648BFF5F7AEBE0021A0F805
:10FA00005610016851E8021F026821F0800142E8A7
:10FA10000213002BF5D14DF808EDFAF74FF85DF819
:10FA200008EBF8D17047806AF5F7A4BE10B50168FD
:10FA3000F9F790FEFBD1E549026852E8022F03680E
:10FA40000A4043E80224002CF6D1C16E012902D1FC
:10FA5000FAF7A1F9FCD12021C0F888100021016734
:10FA6000C16610BD016851E8001F026821F0C001A5
:10FA700042E80013002BF5D14DF808EDF9F718FE18
:10FA80005DF808EBF8D12021C0F8841070470168B8
:10FA9000D0F88820222A39D1B0F860204B6A1A4069
:10FAA000836D23F8022BB0F85E20013AA0F85E20A7
:10FAB0008365B0F85E200AB1704701684DF808ED23
:10FAC000F9F748FE5DF808EBF7D14DF808EDFAF7C5
:10FAD00012F95DF808EBF8D12021C0F88810002158
:10FAE0000167C26E012A18BFF5F7CEBDC1664DF899
:10FAF00008EDFAF750F95DF808EBF8D10168CA692A
:10FB0000D20601D510220A62F9F7C4BEF9F7F4BE95
:10FB10002DE9F84FF9F7FFFD63D1B4F86870AB4EEB
:10FB2000F9F77DFF002F61D01AF020005ED0206829
:10FB3000A16D426A2A4021F8022BB4F85E20013AF6
:10FB4000A4F85E20A165D0F81CA05FEA4A711ED01F
:10FB50005FEACA7218BFB8F1000F01D0F9F791FE41
:10FB60005FEA8A7204D5B9F1000F01D0F9F735FECA
:10FB7000002904D5B9F1000F01D0F9F718FED4F827
:10FB80008C0020B12046F5F758FBC4F88CB0B4F8CF
:10FB90005E000028C6D1206850E8000F216820F4DC
:10FBA0008070FAF710F8F6D1206850E8020F21684B
:10FBB0003040F9F7EAFEF7D1F9F773FE0DD1C4F83A
:10FBC0006CB0F9F798FCFCD12068C169C90601D571
:10FBD00010210162F9F7BEFEA4E72046F5F754FDB7
:10FBE000A0E7816941F0080181611AE0B4F85E0084
:10FBF000B8B1B4F86810884213D2206850E8020FF8
:10FC0000216820F08050F9F7C0FEF6D10648206741
:10FC1000206850E8000F216840F02000F9F7D3FF7A
:10FC2000F6D1BDE8F88F00BF8FFA00080168D0F860
:10FC30008820222A3AD1B0F86020496A1140826DAA
:10FC40001170B0F85E100139A0F85E10816D0131BD
:10FC50008165B0F85E1001B1704701684DF808ED9C
:10FC6000F9F778FD5DF808EBF7D14DF808EDFAF7F4
:10FC700042F85DF808EBF8D12021C0F88810002187
:10FC80000167C26E012A18BFF5F7FEBCC1664DF8C8
:10FC900008EDFAF780F85DF808EBF8D10168CA6959
:10FCA000D20601D510220A62F9F7F4BDF9F724BE95
:10FCB0002DE9F84FF9F72FFD65D1B4F86870434E80
:10FCC000F9F7ADFE002F63D01AF0200060D0206855
:10FCD000A16D406A28400870B4F85E000138A4F8AD
:10FCE0005E00A16D20680131A165D0F81CA05FEA1B
:10FCF0004A711ED05FEACA7218BFB8F1000F01D076
:10FD0000F9F7BFFD5FEA8A7204D5B9F1000F01D09F
:10FD1000F9F763FD002904D5B9F1000F01D0F9F717
:10FD200046FDD4F88C0020B12046F5F786FAC4F8D9
:10FD30008CB0B4F85E000028C4D1206850E8000FF1
:10FD4000216820F48070F9F73EFFF6D1206850E872
:10FD5000020F21683040F9F718FEF7D1F9F7A1FD3D
:10FD60000DD1C4F86CB0F9F7C6FBFCD12068C169AD
:10FD7000C90601D510210162F9F7ECFDA2E7204682
:10FD8000F5F782FC9EE7816941F0080181611AE084
:10FD9000B4F85E00B8B1B4F86810884213D2206895
:10FDA00050E8020F216820F08050F9F7EEFDF6D1FF
:10FDB000BE482067206850E8000F216840F020000E
:10FDC000F9F701FFF6D1BDE8F88F00BFFEFFFFEFA6
:10FDD00070B5016804468068674ED4E903230D6856
:10FDE0001843E369354066693043654E184328433C
:10FDF000624D0860486820F4405010434860A942B2
:10FE0000A0691CBF226A10438A6832401043886090
:10FE1000626AC86A20F00F001043C86259488142E4
:10FE200008D0A9420AD05848814210D1574859A653
:10FE3000006807E055480068800802E05348006801
:10FE4000800A534E00F0030056F8206000E01026B0
:10FE50005448A94210D00121B3F5004F1AD1082E01
:10FE600000F28180DFE806F00546507F497F7F7F02
:10FE70004E00F4F7C1F842E00121082E00F2738031
:10FE8000DFE806F005711C71147171711A00F4F746
:10FE9000B3F80DE0082E66D8DFE806F00549536593
:10FEA0004C6565655100F4F7A7F845E0F4F7C0F834
:10FEB000002855D0626A01E04FF400403A4931F819
:10FEC00012106268B0FBF1F002EB4201884249D3A4
:10FED000B0EB023F46D8010E000210EB520041F198
:10FEE00000010023F1F7D6FA304AA0F540719142A3
:10FEF00034D937E0F4F78CF801E0F4F799F878B3E7
:10FF0000626A01E04FF40040274931F81210B0FB5B
:10FF1000F1F061684A0802EB4000B0FBF1F04FF6E7
:10FF2000F07101401ED0C0F34200084316E0F4F720
:10FF30006FF801E0F4F77CF890B1626A01E04FF4E9
:10FF40000040194931F81210B0FBF1F0616800EB84
:10FF50005100B0FBF1F080B2102803D32168C860D3
:10FF6000002100E001210020C4E91C004FF0011035
:10FF7000A066084670BD00BFF369FFCF0080004057
:10FF8000FFF4FF1100440040003801408800005891
:10FF90004091010801000000040000000200000080
:10FFA000080000000024F400583B0108FFFC0F008B
:10FFB00010B5A0F85E2081650021A0F85C200167E3
:10FFC000816851B1B1F1805F0BD0B1F5805F0CD188
:10FFD000016921B940F2FF110AE0016939B9FF2135
:10FFE00006E0016919B13F2102E0002100E07F2114
:10FFF000A0F860100021C0F88C102221C0F88810F1
:020000040801F1
:10000000016851E8021F036841F0010143E802144E
:10001000002CF5D1416EB1F1005F03D1B0F868104A
:10002000914221D982680021204BF9F710FD1E4A28
:1000300008BF1346036718BF00290AD1016851E8B9
:10004000001F026841F0200142E80013002BF5D1A7
:1000500024E0016851E8001F026841F4907142E811
:100060000013002BF5D119E0826800210D4BF9F740
:10007000EEFC0B4A08BF1346036718BF002903D0E4
:100080000168F9F7A7FCFBD1016851E8021F02687B
:1000900041F0805142E80213002BF5D1002010BD41
:1000A00011FB0008B1FC00088FFA00082DFC0008C5
:1000B0002DE9F843DDF8209004460068984616467E
:1000C0000F4609F10105C1693940C91BB1FA81F137
:1000D0004909B1421ED1002DF5D0F3F76BFAA0EB20
:1000E0000800484519D8B9F1000F16D020680168FA
:1000F0004907E8D5C1690905E5D54FF400610162FA
:1001000050E8000F216820F4D070F9F75CFD1CD096
:100110002068F5E70020BDE8F883206850E8000F6C
:10012000216820F4D070F9F74EFDF6D1206850E830
:10013000020F216820F00100F9F727FCF6D12020FA
:10014000C4F8840004F188000FE0206850E8020F32
:10015000216820F00100F9F718FCF6D12020C4F83E
:100160008400C4F8880004F18C00002184F8801019
:10017000202101600320BDE8F88300000148F5F765
:100180005DB800BF6C4D00202DE9F04190B00446F1
:100190000078052940D859283ED16078A0F1440163
:1001A0000B2900F2BC80DFE811F00C00B500E6007E
:1001B000B500EE00B500B500B500B500F600B5001D
:1001C0000D01A078A0F13001092900F2A380E278A6
:1001D000A2F13001092900F29D802179A1F14803A3
:1001E0000B2B00F29780012505FA03F340F6210559
:1001F0002B4200F08F8000EB8000DE4D4D2902EB9A
:100200004000A0F50470A86000F07681482940F015
:1002100077814FF4616070E1032977D3502875D15D
:10022000A078A0F13002022A80F095806078312811
:1002300040F0D9800A292FD1E078202521796279F0
:10024000A37900EB800005EB4006CE4806700678E7
:1002500031443039017002EB8201CB4A05EB410198
:10026000117011781944C94B30391170E17901EBE3
:10027000810105EB41011970217A1D78294430393B
:100280001970C34B617A3039197001781278914234
:1002900002D8017802310170FDF77CF9DFF8E4E261
:1002A000DFF8E482B94CDFF8E8C2B44E0020032244
:1002B0009EF8001098F8003025789CF8007086F8B9
:1002C00024005A2086F82500012086F8260086F8AA
:1002D000270086F82F209EF8002086F8302098F816
:1002E000002086F83120227886F83220A44A107146
:1002F000A84851719371D571177210609CF8000075
:1003000086F83300F9F7D6FF09216FE0412808BFCE
:10031000162923D010B0BDE8F041FDF7E7BB562801
:1003200067D05A28F6D1A078432800F0BE80532821
:1003300000F0CE80482840F0C8809AA20120142105
:10034000FDF7DEFB41F28830F2F715FF10B0BDE893
:10035000F041FAF71FB83228DCD1B6E060784328C4
:10036000D8D1844DA01C002114294FD0425C6B18B9
:1003700001311A74F8E7A0783928CBD83038C0B2E8
:10038000FDF7A2FB25E0A0783928C3D83038C0B2E9
:10039000FDF792FB1DE0A0783038C1B2092900F2C8
:1003A00094807449754A0871087982F82D00744A5E
:1003B00044F6595010800879032130309070F9F7D5
:1003C000D1FAD1E0A0783928A4D83038C0B2FDF7EE
:1003D00083FB20786178A378694A1070517093701C
:1003E0000120032183E0FDF781FB0321644A012002
:1003F0007DE0A078432830D0482866D1604A66481E
:100400006649C2E900100120082170E0FDF794FB65
:100410005948407D01280AD158480021142909D0A3
:100420006B18421801311B7C82F85030F6E702202D
:10043000287106E000212971297980F82D10F9F73B
:1004400039FF4F490020162803D0225C0A5401309E
:10045000F9E74B4A0120162149E06C464021F9F7A3
:10046000A5F82046F9F72AFE454C2F21302204F149
:100470001100F1F749F943201121224620709DF81F
:1004800000006070DDF80100C4F80200DDF805002E
:10049000C4F80600DDF80900C4F80A00BDF80D0034
:1004A000E0819DF80F0020740DE000208DF8000021
:1004B0006846F5F703FD324A3948052110609DF87A
:1004C000000041301071F9F74DFA10B0BDE8F0812D
:1004D0002B4C402130222046F1F71EF9FDF778FA27
:1004E00041F28830F2F747FE01201521224610B074
:1004F000BDE8F041FDF704BB3C20A9684843A86073
:10050000A8684FF47A711D4E484370603060F9F767
:1005100093FF20781A4A6178A378E77810702079E1
:1005200051700521D770937001271071F9F71AFAED
:10053000002086F824005A2086F8250086F82670C8
:1005400086F82770A078E17800EB800001EB40008E
:10055000103886F82800207986F82900287886F84F
:100560002C00287986F82D0010B0BDE8F041F9F78D
:10057000A1BE00BF84030020C44C00200000002066
:10058000104E00206400002065000020660000205E
:10059000B033002050005A010318031A56005A01C4
:1005A0004C005A012159756E486F726E2053545396
:1005B00020526576697665210000000070B586B02E
:1005C0001C460023ADF802303A4B1D7A854201D219
:1005D000FB2042E0D868084088422AD132B15A68EC
:1005E00022B10DF105000DF1020190471C480AAB44
:1005F0004FF400712246059302F016F80546FEF707
:10060000C9FFBDF802006946284480B2FEF784FFA6
:1006100001301FD0BDF80220BDF800101A4B0DF1BB
:10062000050042B110F8015B8EB2013A01319D55CF
:10063000F7E7FA2011E013FA81F0059BADF80010FE
:100640004FF40071224601F0EFFFFFF735F8FEF797
:10065000ADFF02E0FFF730F8FD2040B206B070BDFC
:100660006C4E002080B513480021182200F07DF860
:10067000054800214FF4806200F077F803480168D4
:100680000348BDE88040084738040020C83B010803
:1006900029F600080220002100F046B802200121BE
:1006A00000F042B803494860704700BF0149087232
:1006B000704700BF38080020B0B5EFF31084EFF3A7
:1006C000108072B62348016819B10848D0E90015B6
:1006D00007E04068002805480CBFD0E90415D0E9C0
:1006E00002158847A84784F31088B0BD703B010805
:1006F00018480021C0E90011704700BFEFF31082D5
:10070000EFF3108372B629B1012909D11149496863
:10071000084303E00F49496821EA00000D49486099
:1007200082F31088704700BFEFF31082EFF310835D
:1007300072B629B1012909D106490968084303E0C5
:100740000449096821EA00000249086082F3108820
:10075000704700BFE0020020130408BF704711F883
:10076000013B013A00F8013BF6E7130408BF70476C
:1007700000F8011B013AF8E7FFF79EBF704770478A
:10078000B0B5EFF310851446EFF3108172B6FCF7A5
:10079000E3FE424901EB8000846185F31088B0BD1F
:1007A0002DE9F047DFF8CCA03C4E4FF0FF39012592
:1007B000DAF8048006F1080400EA0800CAF8040028
:1007C00033687168DAF800201040B268184230D0FF
:1007D00011402ED1274657F8081F0842FBD0396830
:1007E00008407968084208BFC7F804907968084053
:1007F000FCF7B2FEF06005FA00F0796821EA00002B
:100800007860EFF31080EFF3108172B63168F26810
:1008100005FA02F29143316031699143316180F30D
:100820001088F06806EB800080698047DAF80400E1
:10083000C6E74FF0FF30F060FFF7A1FFEFF3108441
:10084000EFF3108072B631687068DAF8002011405A
:10085000DAF80420114204D1B168014208BFFFF761
:100860008BFF84F31088FFF789FFCAF80480BDE886
:10087000F08700BFC000002010B5EFF31082EFF347
:10088000108372B6054B1C6803EBC10104431C6066
:100890000B691843086182F3108810BDE80200203C
:1008A0002DE9F041012490B11F4683B10024064692
:1008B0001546DDF8188004607648426A084690477D
:1008C000B47234817060C6E903787461F5722046B1
:1008D000BDE8F08110B56F48C169846A8847214638
:1008E000BDE81040084700BFF8B504466948C16933
:1008F000D0E90967884705462046B047281A394697
:10090000BDE8F840084700BF2DE9F843614EEFF31A
:100910001088EFF3108072B6D6E904408047054690
:10092000A0475B4F3C6854B1401B21460A684B69A5
:10093000121A38BF00220A60002B1946F6D1B56999
:100940004FF00009E4B126681EB1A8473C68864212
:1009500010D2A4F808906269D4E903103A6088477D
:10096000E07A012804D1A07A10B9204600F02AF8D4
:100970003C68E7E724B1207A10B92046FEF72CFF47
:1009800088F31088BDE8F8834148002101604148A0
:100990000068004710B588B104463E48426A0846E0
:1009A000904760602046FEF7EFFE48B1204600F019
:1009B0003FF82046BDE8104000F004B8012010BD0B
:1009C000002010BDF8B528B10446FEF7DDFE08B9D9
:1009D000607A08B10120F8BD2E4EEFF31085EFF3D9
:1009E000108072B66768306A80470021A1724FF4A8
:1009F00080718742218138BF07462760244F3868BD
:100A000060B1B0698047216808443968206009688E
:100A1000884205D32046FEF7CDFE04E030698047CA
:100A20002046FEF7BDFE85F310880020F8BD00BF0C
:100A3000012158B3B0B5164DEFF31084EFF31082D7
:100A400072B681722968E1B100228142427207D0F8
:100A50000A46B2B182420AD0536911461A46F8E7F3
:100A60000272406940B12860FEF7B6FE09E04069B5
:100A700000B90020486104E00648C06880470020B3
:100A8000286084F310880021BDE8B0400846704714
:100A90009C1B00209C3B0108FEE7000010B50446AB
:100AA0000748016A2046884728B10648844202D395
:100AB0000548844201D9002010BD012010BD00BFAF
:100AC000C43A0108C0CA89360028503710B5074C0F
:100AD00000F00F03B0F1FF3F034A2344C8BF83185F
:100AE0000801187010BD00BF00E400E014ED00E044
:100AF0000648BFF34F8F064A016801F4E0611143D5
:100B00000160BFF34F8F00BFFDE700BF0CED00E0B9
:100B10000400FA05F0B500238B4228BFF0BD02EBBC
:100B2000430632F813400233768824F0030426F09B
:100B300003060559875907518551044406446568E1
:100B4000776867607560E7E72DE9F04105889846AA
:100B500016460C460746012A09D1201D294631B107
:100B60000268013982F0004240F8082BF7E7102DA7
:100B700014D0202D1ED0402D15D0802D0ED0B5F5CF
:100B8000807F17D0B5F5007F0DD0B5F5805F0AD016
:100B9000B5F5006F0ED0B5F5806F0FD13846214600
:100BA00000F078F80AE07A6820462946012300F030
:100BB00077FC03E03846214600F086F9B8F1000FD3
:100BC00004D0BA68B9892046FFF7A4FF012E16D1D8
:100BD000284602F04FFC01464FF07E5002F000FB29
:100BE000064665B1D4E90017F8F792FD206087F05A
:100BF0000041F8F78DFD60600834013DF1E7BDE884
:100C0000F0810000002201801029426016D02029C6
:100C100016D0402916D0802916D0B1F5807F15D086
:100C2000B1F5007F14D0B1F5806F13D0B1F5805FBE
:100C300012D0B1F5006F18D1154B0EE00D4B0CE042
:100C40000D4B0AE00D4B08E00D4B06E00D4B04E0A8
:100C50000D4B02E00D4B00E0054B4DF808EDF8F7A9
:100C60004FFF5DF808EB40B27047FF20FBE700BF85
:100C700010910108D09001080091010830910108FD
:100C8000C0900108F090010820910108B09001087F
:100C9000E09001082DE9F04F9DB00388059101EB2C
:100CA00083024FEA830B02925A0801920390406834
:100CB000970007EB83020490D8080023002800F077
:100CC000F1801590059800EB0B0500EB0308C419A3
:100CD00086180498296818440B90D8F800000990E9
:100CE0000891CDE91727149302F0E2F97168D6F85C
:100CF0000CA0D4F80890E7686A681A91B1681C9152
:100D00006168CDF848A00C961B912946CDF8449017
:100D100013970A950692AD683268C9680E951091CE
:100D200007922268C8F80000D8F80C001992CDF894
:100D300058B0D8E901B60D960F9002F0B9F9C8F88D
:100D40000C003046F8F712FD069DC8F8080058461A
:100D5000F8F70CFDC8F804003846F8F700FE1C99B7
:100D6000E060484602F0A4F9A060DDE91A1002F044
:100D70009FF9DDF81C8060601998F8F757FE206035
:100D8000DDE9081002F046FD07465846F8F79DFCDD
:100D9000DDF82CA00546DAE90094F8F7AAFD06462E
:100DA0003846F8F7D4FDF8F793FDDDF828B049464A
:100DB000CBF80400F8F733FF06462846F8F7C7FDDE
:100DC000F8F718FE1999CBF80000F8F7CBFE0546A6
:100DD000DDE91A0102F01EFD2146064602F0C6FBBF
:100DE00007462846F8F785FDF8F748FD0C9F214691
:100DF0007860F8F7ECFD04463046F8F77AFDF8F72E
:100E0000CCFB3860B946DDE90D0102F003FD064672
:100E1000DDE90F0102F0FEFCDAE902850746F8F78A
:100E2000D9FC04463046F8F778FDF8F7B6FBCBF866
:100E30000C003046F8F7CEFC04463846F8F76DFD56
:100E4000F8F7BAFDCBF808001C98119902F0E2FC03
:100E50000446DDE9120102F0DDFC2946064602F0F7
:100E600085FB07462046F8F7B5FCF8F707FDC9F8FB
:100E70000C0020462946DDF858B002F077FB044606
:100E80003046F8F7A7FCF8F788FBDDE91727149B35
:100E9000C9F8080015980BF1100B103710321033F9
:100EA00001380BE7019C0598049A0223214600F0C3
:100EB000F7FA039821460223426802981DB0BDE864
:100EC000F04F00F0EDBA00002DE9F04FA9B004900A
:100ED000008889464FEA500B279001EB8B0858F8A1
:100EE0002B102291D9E900562846219602F0E0F80D
:100EF00059F82B102890259102F0DAF808EB8B04B2
:100F000054F82B10239102F0D3F8D4F804A0C9F8B8
:100F100000003046F8F723FDD8F804602690F8F773
:100F2000A3FD04EB8B014F680391F8F7A7FC22990E
:100F3000C9F80400F8F738FC3146229002F0B8F8FE
:100F4000F8F7AAFECDF8909049F82B005146219869
:100F500002F060FCDDF894900546F8F714FEDDF829
:100F60008CA0F8F7FCFCC8F804002898F8F70BFEF2
:100F7000F8F777FDCDF8088048F82B003146269821
:100F800002F048FCF8F788FE60602298F8F744FD0C
:100F9000F8F774FC44F82B0028464946019402F007
:100FA00087F8F8F75EFD03994FEA8B0648606FF00B
:100FB000030000EB8B0100EBCB0020911F906FF042
:100FC000070000EB0B1126910BEB4B0100EB8100AE
:100FD0008F0028906FF00100279A00EB92004008E4
:100FE000239004984068059090084FEACB02009047
:100FF000002027900020229000202190249D2798F7
:101000002C18A818D4E9029A1392D0F808801A90E4
:10101000C06819904846F8F709FD05EB060B2590C6
:101020001296DBF80810DBF80C201E911C9202F0DF
:101030003FF8EE191197B168F7681D9102F038F882
:10104000199DA0605046F8F791FBDBF80C10CDF825
:101050005CB0834602F02CF8F1681B9602F028F889
:10106000E0604846F8F7D3FD1C9C8146F8F758FE2F
:10107000F8F712FE16905046F8F727FBDDF878A037
:101080000646F8F7EEFC1D9DF8F770FB15905146EB
:10109000259802F0BFFBF8F718FB19905846F8F7AF
:1010A00008FCF8F7F9FD80464846F8F702FCF8F727
:1010B000E5FB18903046F8F752FCF8F706FB0546BA
:1010C000059821994418229901441491279900EB1D
:1010D000010B2398002800F03881CDF82C8024994A
:1010E000CDE90E451F9889460F18099720980E18CC
:1010F00028980A1805460D92289026980C188246C2
:101100003068516810940890079101F0D1FF396858
:101110000C901E9101F0CCFF61681D9101F0C8FF99
:1011200059F80A2059F8051056F8045CCDF898A033
:101130004C461C9257F8042C3060284625920691A4
:1011400001F0B6FF57F8041C0A9001F0B1FF59F8FE
:101150000A1001F0ADFF46F8040CDDF85490DBF8FE
:1011600008604846F8F7E1FBDBF80CA0169F8046C4
:101170003846F8F7ECFA0146F8F7F4FC179C3146CC
:10118000E060F8F74CFD07464846F8F7E0FA0146FC
:10119000F8F748FD0699A060F8F706FB169004469C
:1011A000DDE9071002F036FB17900546DDE91D105A
:1011B00002F030FB01461590204601F079FF259999
:1011C0000446F8F7F1FADDF870B0594601F070FF07
:1011D00005462046F8F7BBFA07462846F8F7A5FB70
:1011E000F8F74CFB099F514647F8040CF8F7EFFB62
:1011F00005462046F8F799FBF8F773FA149D386016
:101200000B9FD5F810903846F8F773FBD5F814808B
:10121000199E04463046F8F7DDFAF8F7BEF91A9D34
:101220004946E860F8F774FA04463846F8F7D2FA07
:10123000F8F7C2FBA8600A98259902F0EBFAF8F7D4
:101240008EFC04460C981E9902F0E4FA1D9902F0F7
:10125000E1FA05462046F8F74CFB06462846F8F723
:10126000B9FAF8F7D9FBDDF890B028994BF80100EE
:1012700085F00041484602F079F905462046F8F726
:10128000A9FAF8F72EFA0D990E9C0F9F4860384680
:10129000D4F81880F8F79EFAD4F81CA0189D0646DA
:1012A0002846F8F754FAF8F713FB1B9C4146E06018
:1012B000F8F78DFB06463846F8F749FAF8F79AFB37
:1012C000A060DDE9150102F0A5FA81461C98259978
:1012D00002F0A0FA179902F09DFA07464846F8F77F
:1012E00036FA04463846F8F775FAF8F719FD269EDF
:1012F00051464BF80600F8F792FC04464846F8F7CA
:1013000069FAF8F74AF9109948602098083820904F
:101310001F9808381F902898083828903046A6F162
:1013200008002690279808302790229810302290A5
:101330002198183021902398119F139A129E0138FA
:10134000083708320836239058E6DBE902A7DDF8B3
:1013500054904846F8F7FBF9169E83463946F8F74D
:10136000D7F90146584602F055FADDF85CB051460F
:10137000CBF80C00F8F7CCF906464846F8F78EFA99
:10138000F8F738FBCBF8080014984746D0E904A9D1
:101390004046F8F7DCF9199E80464946F8F7B8F957
:1013A0000146F8F7DFFBDDF868805146C8F80C000D
:1013B000F8F7AEF906463846F8F79BFAF8F71AFB45
:1013C000C8F808002846D4E90679F8F767FA189CA7
:1013D00006464946F8F7B0FBF8F77AFA1B9E3946FD
:1013E000F060F8F7A9FB04462846F8F782FAF8F708
:1013F000E3FA009DB0600D4E2498059A0423294617
:10140000B047049C0298294604236268B04762688A
:10141000019829460423B0476268039829460423AB
:10142000B44629B0BDE8F04F604700BFA1140108E1
:101430002DE9F04114468846064674B1F8F7D5FB0D
:10144000F8F759FB0146284601F032FE01F02CFB6B
:1014500048F8040B0836013CEFE7BDE8F0812DE9C0
:10146000F84FF8F7ADFA00925BF8047BC24513D051
:101470005BF8045B3846294601F09FFE0646384675
:10148000294601F09AFE002818BF444608F10108D9
:10149000002E18BF2F46E9E70098F8F753BA00006E
:1014A0002DE9F04FC1B00E4600F10C01CDE902323A
:1014B00004303346009101900B96D908DA00DDF82C
:1014C00004A0C8004FEA01190591CDE90C2380461C
:1014D000A0EBD300C0003A9048013E9001EB8100A0
:1014E000C50001EB4100C1004FEA001B40913BA841
:1014F0000021CDF8FCB080E82003399129465AF844
:1015000008004F46DDF8F89045465AF801102F9034
:101510002E9101F0CDFD0446329040985AF80020FB
:101520003A985AF80010104627922B9101F0C0FD0E
:1015300001463190204601F0BBFD04465AF80910DF
:10154000DAF800002D912C9001F0B2FD06465AF811
:1015500007005AF80B103690359101F0A9FD0146AD
:101560003090304601F0A4FD2146074601F0A0FD71
:10157000CAF800003846F8F79CF94AF809000AEB67
:101580000800349050F8048C3B98504450F804BC48
:1015900038904046594601F08BFD0546269040980C
:1015A0005044379050F8044C3A98504450F8047C1A
:1015B00033902046F8F762F901462590F8F7F4F8E1
:1015C00030998146304602F025F94946054602F039
:1015D00021F93D994AF801004846F8F7C7F83F99C4
:1015E0004AF801004046F8F7BAFA05462A90204624
:1015F000F8F752FB01462990F8F7A1FA70490D4619
:1016000001F0B4FF04463090DDE92E1002F002F93B
:101610000646289027982B9902F0FCF8014627905F
:10162000304602F0F7F8F8F778F907462E903D9823
:101630000AEB000B3F985BF8045C504450F8046CD4
:1016400024902846F8F7E8F921462F9001F030FD64
:1016500004462B90DDE92C0102F0DCF839462D9090
:1016600001F026FD21462C9002F0D4F83C994AF86E
:101670000100DDE9251001F01BFD07463E985AF8F0
:10168000049C0AEB0008484658F8041C269101F017
:101690000FFD04462846F8F7E7F905462046F8F717
:1016A00065F83946064601F003FD4AF8040C304659
:1016B000F8F7F2FA48F8040CDDE9311002F0AAF864
:1016C00006462046F8F701F83146044601F0F0FCE2
:1016D0004BF8040C2046F8F79FF9249941F8040CC4
:1016E000DDE9291002F096F8354CF8F730F9054697
:1016F000DDE9271001F0DCFCF8F729F9269983468B
:101700004846DDF8F08002F085F82946044601F0ED
:10171000CFFC0746DDE9351002F07CF859468146DA
:1017200001F0C6FC06463846F8F79EF9349941F8B0
:10173000040C314638460B9E02F06CF8339941F8A0
:10174000040C2046F7F7C1FF044648463B9DDDF8F0
:10175000F490F8F704FA07462046F8F78FF838991E
:1017600041F8040C2046F8F797FA379941F8040C31
:10177000DDE92B0101F09CFC3A994AF80100DDE912
:101780002F0102F047F80446DDE92D0102F042F88E
:101790002146074602F03EF84AF805002046394641
:1017A000DDF8FCB001F084FC4099DDE90C234AF837
:1017B0000100399992441944B142FFF49EAE01E010
:1017C000F304353F402BC0F06A820298DDF80090A8
:1017D0000023012480B204900598C0EBC0004FEABA
:1017E000C008CDF8B88004980399034451F8330039
:1017F000C3EBC30603EB830C5D0103EB430E0893BD
:101800003A9051F83600399051F83C0038904859D8
:10181000379051F83E000A9018010A5836922A1D56
:101820008A583592021D8858DA000432349088585C
:101830004FEA0E12339088583290F0000430085866
:101840003190101D085830904FEACC0004300858F1
:101850002F904FEACE0004300858CDE90694099045
:101860003C993B9A2D9459F801000C4659F8021006
:1018700017461990189101F01BFC054621904098DD
:1018800059F8081059F800001691179001F010FC53
:1018900001462090F8F753F9054625903E9859F8EF
:1018A0000010D9F800001D911C9001F001FCDDF83A
:1018B000F4A059F80B1006461F9059F80A001A9127
:1018C0001B9001F0F5FB01461E90304601F0F0FB45
:1018D0002946834601F0ECFBC9F8000009EB04003F
:1018E00009EB0701299050F8040C2B9151F8041CC6
:1018F0001190109101F0DCFB0546409809EB0801BE
:101900002A9151F8041C48442C9050F8040C0E9174
:101910000F9001F0CDFB80462846F8F787F8074680
:1019200024903E98484450F8041C269059F8040C22
:101930001391129001F0BCFB064609EB0A0050F827
:10194000042C27903F984844159250F8041C289086
:101950001046149101F0ACFB82463046F7F7FFFFCA
:101960003946239001F056FF2599074622905846A4
:1019700001F050FF01462590379801F0F7FD04462D
:101980003598F7F78BFFF7F708FE3E9949F8010005
:101990002846F8F73CF98046DDE9201001F03AFFCF
:1019A00083463046F8F75DF85946064601F080FB5D
:1019B00005462090DDE91E1001F02CFF4146074648
:1019C00001F028FF01462190369801F0CFFD044632
:1019D0003498F7F7A2FFF7F7E0FD3D9949F80100C9
:1019E0003046F8F7BCF805461E904046F7F746FF2C
:1019F00001461F90329801F0B9FD04463098F7F780
:101A00008CFFF7F7CAFD3F9949F80100DDE9101096
:101A100001F000FF8246DDE90E1001F0FBFE80467A
:101A20005046F8F7F4F89F490E4601F09FFD054631
:101A30001190DDE9181001F0EDFE0746DDE9161002
:101A400001F0E8FE04463846F8F76AF9F7F76DFF4B
:101A500006461890DDE9120101F0DCFE29461990D6
:101A600001F026FB05461290DDE91A1001F0D2FEC6
:101A70003146179001F01CFB01461A90F8F75FF809
:101A800083461B905046F7F7D1FF864EF7F74DFF80
:101A9000054616903846F7F70CFFF7F746FF044661
:101AA0001390DDE9141001F0B5FE2946159001F000
:101AB000FFFA0646DDE91C0101F0ACFE2146824634
:101AC00001F0F6FA3146074601F0A4FE01461D90EA
:101AD0003A9801F04BFD05463398F7F762FEF7F7A9
:101AE00000FE3C9949F8010012981A9901F092FE03
:101AF00004461A903046F7F7C1FE01461C9039980B
:101B000001F034FD05463198F7F721FFF7F7E9FDBD
:101B10002E9949F801001998119901F07BFE83462E
:101B2000DDE9170101F076FE80465846F7F77EFFA3
:101B300007461890DDE9150101F06CFE1399054682
:101B4000504601F067FE2946044601F063FE014657
:101B50001990389801F00AFD06462F98F7F79EFE77
:101B6000F7F7B6FE3B9949F801005846F8F74FF8E9
:101B700007462846F8F7D4F80A9E82465146F7F7FA
:101B8000C7FD099D04463946F7F721FFF7F705FD24
:101B9000409949F80100DDE9230101F089FA49F88B
:101BA000040C3798229901F0E1FC044635982599F8
:101BB00001F0DCFCF7F700FF269941F8040C369899
:101BC000209901F0D3FC04463498219901F0CEFC11
:101BD000F8F7A6F8279941F8040C32981E9901F0FD
:101BE000C5FC044630981F9901F0C0FCF8F798F83E
:101BF000289941F8040C3A981B9901F0B7FC044667
